:020000040800F2
:1000000000000220F12E0108F9920008FB9200087E
:10001000FD920008FF920008019300080000000014
:100020000000000000000000000000000393000832
:1000300005930008000000000793000809930008DA
:10004000352F0108352F0108352F0108352F0108FC
:10005000352F0108352F0108352F0108352F0108EC
:10006000352F0108352F0108352F0108A17600082A
:10007000352F0108352F0108352F0108352F0108CC
:10008000352F0108352F0108352F0108352F0108BC
:10009000352F0108352F0108352F01083995000843
:1000A000352F0108352F0108352F0108352F01089C
:1000B00005950008352F0108352F0108352F010857
:1000C000352F0108352F0108352F0108352F01087C
:1000D000352F0108352F01084D960008352F0108EE
:1000E000352F0108352F01080D930008352F010821
:1000F000352F0108352F0108352F0108352F01084C
:10010000352F0108352F0108352F0108352F01083B
:10011000352F0108352F0108352F0108352F01082B
:10012000352F0108352F0108352F0108352F01081B
:10013000352F0108352F0108352F0108352F01080B
:10014000352F0108352F0108352F01083D93000890
:10015000352F0108352F0108352F0108352F0108EB
:10016000352F0108352F0108352F0108352F0108DB
:10017000352F0108352F0108352F0108352F0108CB
:08018000352F0108352F01089D
:1001880074B2050800000020080C0020080C0020AC
:10019800A43C002008B5074B186809F04BF80DF08F
:1001A80043FE054B054806221A70BDE8084001F0D9
:1001B800C4BB00BF10260020A4250020800F00200B
:1001C80008B5034801F0B9FB024B00221A7008BDBC
:1001D800D4170020A425002008B5054B01220020D3
:1001E8001A7005F053FD0348BDE8084001F0A5BBAF
:1001F800242C0020441500202DE9F041144C204601
:1002080003F0A3FE00201349134A03F055FC1349D9
:10021800134A0746002003F04FFC1249124A0646CB
:10022800002003F049FCD22105463A4623460A201D
:1002380003F05AFDD22132462346FA2003F054FD3A
:100248005A20D2212A462346BDE8F04103F04CBD8E
:1002580058130020E69E0508C9010008EF9E05080E
:10026800E1010008F79E05089D01000808B5054B47
:10027800012200201A7005F009FD0348BDE8084076
:1002880001F05BBB242C00204415002008B503486E
:1002980001F053FB024B00221A7008BDD41700204E
:1002A800A425002008B5054B07221A700DF0BCFDE7
:1002B8000348BDE8084001F040BB00BFA42500206A
:1002C800581300202DE9F041144C204603F03DFE60
:1002D80000201349134A03F0EFFB1349134A07465A
:1002E800002003F0E9FB1249124A0646002003F0F9
:1002F800E3FBD22105463A4623460A2003F0F4FCE4
:10030800D221324623465A2003F0EEFCAA20D221FD
:100318002A462346BDE8F04103F0E6BC800F0020E2
:10032800E69E050895020008009F0508AD02000832
:10033800099F050875020008014801F0FEBA00BFD0
:100348006C11002010B5094C204603F0FEFD00207A
:100358000749084A03F0B0FBD221024623464FF46E
:100368008270BDE8104003F0BFBC00BF8C160020AF
:10037800129F05084103000870B50C4C0C4D20680D
:100388004FF6E076314602F0DBFE2068294602F09F
:1003980085FE6068314602F0D3FE6068294602F0A7
:1003A8007DFEBDE8704004F009B800BF080C0020CD
:1003B80001A5050838B52B4CFFF7DEFF002005F036
:1003C80065FC237A23B90A203221274A05F06CFDFF
:1003D800637A23B90A206421244A05F065FD214C7B
:1003E800A37A23B90A209621214A05F05DFDA37A54
:1003F8001C4DFBB16B7AEBB12B7ADBB100232B726E
:100408006B72AB721B4B286801221A704FF6E071B1
:1004180002F096FE2868184902F040FE68681749FD
:1004280002F03CFE0BF0FDF903F0C8FF144804F09D
:1004380009F80DE00B4C4FF47841206802F080FE7B
:100448002068104902F02AFE60680F4902F026FE73
:10045800FFF792FF00200BF0A7F90C48BDE83840E1
:1004680001F06BBA080C0020199F0508279F0508A2
:10047800369F0508A4250020449F050802A5050805
:1004880080969800589F050804A50508D4170020F1
:1004980008B500200BF088F90248BDE8084001F0D3
:1004A8004CBA00BFD417002038B5FFF765FF0DF030
:1004B800D3FC3C213F220023DF2005F0D7FC4FF47A
:1004C80080600EF005FA124C3E223C21DF2000230A
:1004D80005F0CCFC012323720E4B4FF6E07518682B
:1004E80008F0A8FE2068294602F02AFE20680A497A
:1004F80002F0D4FD6068294602F022FE60680749D0
:1005080002F0CCFD03F05AFF054B00221A7038BDEB
:10051800080C0020102600206A9F05087D9F05080A
:10052800A425002038B5FFF727FF0DF095FC6E21B4
:100538003F220023DF2005F099FC4FF486400EF09F
:10054800C7F9124C3E226E21DF20002305F08EFCF5
:10055800012363720E4B4FF6E075186808F06AFEC7
:100568002068294602F0ECFD20680A4902F096FD51
:100578006068294602F0E4FD6068074902F08EFDD4
:1005880003F01CFF054B00221A7038BD080C002030
:1005980010260020909F0508A19F0508A42500208B
:1005A80010B5FFF7E9FE0DF057FCA0213F2200230C
:1005B800DF2005F05BFC4FF402400EF089F9114C86
:1005C8003E22A021DF20002305F050FC0123A37266
:1005D8000D4B186808F02EFE20684FF6E07102F007
:1005E800AFFD2068094902F059FD6068084902F02A
:1005F80055FD03F0E3FE64200AF0B0FF054B00222E
:100608001A7010BD080C002010260020B29F0508A3
:1006180002A50508A42500202DE9F74F3A4D3B4EC9
:100628000024284603F091FC224623464FF6FF712A
:1006380037480094019402F047FD4FF6E07804270C
:10064800F06041462246234632480097019402F062
:100658003BFD23463060414622462F4800970194CF
:1006680002F032FD2D4970602D4A204603F024FA2D
:100678002C492D4A0746204603F01EFA2B492C4ADE
:100688008046204603F018FA2A492B4A814620461C
:1006980003F012FA29492A4A8346204603F00CFA45
:1006A80021468246F2682B46204603F01DFB5A215C
:1006B80032682B460A2003F017FB6E2172682B461E
:1006C8000A2003F011FB9B213A462B46FA2003F03F
:1006D8000BFB692142462B46FA2003F005FB372124
:1006E8004A462B46FA2003F0FFFAC82152462B4609
:1006F800AA2003F0F9FAF020C8215A462B4603B085
:10070800BDE8F04F03F0F0BAFC130020080C0020FD
:10071800C69F0508CE9F0508E19F0508F09F0508BC
:10072800A9050008F89F05082D050008E89F050899
:10073800B104000800A005089904000807A00508EE
:10074800BD03000838B50C4C4FF6E0752068294603
:1007580002F0F6FC2068094902F0A0FC606829460E
:1007680002F0EEFC6068064902F098FC03F026FEF1
:10077800BDE8384003F022BE080C0020CE9F0508D3
:100788000EA0050870B52DED028B9FED248A88B068
:100798000A26F0EE488A03E0B0EE608AF0EE418A5D
:1007A8000CF093FA8DED000ACDED010A9DE80300E7
:1007B80004AB83E80300F0EE680AB0EE480A9DED4A
:1007C800041ADDED051A8DED028ACDED038A0CF0D1
:1007D8001FF8CDED010A8DED000A9DE8030002AD7A
:1007E80085E80300013E6C46DDED020A9DED031A23
:1007F800D2D19FED0B0A0CF05FFA8DED000ACDED1A
:10080800010A9DE8030085E80300DDED030A9DED7C
:10081800020A08B0BDEC028B70BD00BF00000000EA
:10082800CDCCCC3D2DE9F74F564D574CDFF86491B0
:10083800DFF864814FF6E07005F0FCF9286811F0E4
:100848005BFA064668680F4611F056FA3246CDE95B
:1008580000013B464946204616F0C4F822460023CC
:100868000520372105F020FB2869484F484E11F034
:1008780043FA824668698B4611F03EFA5246CDE942
:1008880000015B463946204616F0ACF822460023A4
:100898000520692105F008FB286B11F02DFA824626
:1008A800686B8B4611F028FA5246CDE900015B4689
:1008B8004146204616F096F8002305209B21224643
:1008C80005F0F2FA31462A6C204616F08BF82246DB
:1008D80000239B21A22005F0E7FA4FF4FC6005F005
:1008E800A9F9A86811F008FA8246E8688B4611F061
:1008F80003FA5246CDE900015B464946204616F008
:1009080071F8224605205021002305F0CDFAA86988
:1009180011F0F2F98246E8698B4611F0EDF952467A
:10092800CDE900015B463946204616F05BF82246C1
:1009380000230520822105F0B7FAA86B11F0DCF935
:100948008246E86B8B4611F0D7F95246CDE9000193
:100958005B464146204616F045F800230520B421A1
:10096800224605F0A1FA31466A6C204616F03AF89C
:10097800A220B4212246002303B0BDE8F04F05F0C1
:1009880093BA00BF303A0020180C002033A00508A5
:1009980056A0050821A0050845A0050808B50020AF
:1009A80005F074F90A4B1B780B2B0BD8DFE803F022
:1009B8000A0A0A0A0A0A08060A0A0A0A054802E08E
:1009C800054800E00548BDE8084000F0B6BF00BF94
:1009D800A425002058130020800F0020D4170020E1
:1009E8002DE9F14F2D4C204603F0AFFA00202C4999
:1009F8002C4A03F061F82C492C4A8146002003F068
:100A08005BF82B492B4A0746002003F055F82A4982
:100A18002A4A0646002003F04FF82949294A054684
:100A2800002003F049F82849284A8046002003F0AE
:100A380043F82749274A8246002003F03DF8D2218F
:100A480083464A462346E62003F04EF928203A46D4
:100A58002346014603F048F946213246234628201A
:100A680003F042F964212A462346282003F03CF982
:100A7800822142462346282003F036F9524623466F
:100A88002820A02103F030F928205A46BE21234609
:100A980001B0BDE8F04F03F027B900BF44150020AE
:100AA8005BA00508A509000864A0050875120008E0
:100AB8006FA005085112000879A005082D1200083A
:100AC80084A00508091200088FA00508E511000890
:100AD80099A00508C1110008023810B50A2800F2CB
:100AE8003C83DFE810F00B000F006400D2008A019D
:100AF8002001170231023A03A102F502BDE81040B5
:100B08000AF0FCBE00204FF6E0710BF057F86320A6
:100B18004FF6E0710BF052F8B3204FF4F0610BF090
:100B28004DF8C7204FF6E0710BF048F84FF6FF700C
:100B380005F080F8DC2100237D20D34A05F0B4F9C4
:100B48004EF29C7005F076F8052001210023CF4A6B
:100B580005F0AAF9052052210023CD4A05F0A4F991
:100B6800B62100230520CB4A05F09EF94FF4F0602A
:100B780005F060F80121002340F21310C34A05F084
:100B880093F9002340F213105221C24A05F08CF960
:100B9800B621C14A40F21310002305F085F94EF240
:100BA8009C7005F047F80520A221BC4A68E00020A7
:100BB8004FF6E0710BF002F831204FF6E0710AF0C1
:100BC800FDFF63204FF6E0710AF0F8FF95204FF61D
:100BD800E0710AF0F3FFC7204FF6E0710AF0EEFF6C
:100BE8004EF29C7005F026F8052001210023AC4A3E
:100BF80005F05AF9052020210023AA4A05F054F9E6
:100C0800052052210023A84A05F04EF90520842129
:100C18000023A64A05F048F9B62105209D4A00237D
:100C280005F042F94FF4F06005F004F8012140F2B4
:100C3800131000239A4A05F037F940F213102021C7
:100C48009B4A002305F030F940F213105221914AD3
:100C5800002305F029F940F213108421954A002356
:100C680005F022F9B621944A40F21310002305F04A
:100C78001BF94FF6FF7004F0DDFF904A7D20DC2160
:100C88000023BDE8104005F00FB900204FF6E071D1
:100C98000AF094FF27204FF6E0710AF08FFF4F20EB
:100CA8004FF6E0710AF08AFF77204FF6E0710AF0FC
:100CB80085FF9F204FF6E0710AF080FFC7204FF6AE
:100CC800E0710AF07BFF4EF29C7004F0B3FF052040
:100CD800012100236F4A05F0E7F8052016210023BB
:100CE800774A05F0E1F805203E210023754A05F012
:100CF800DBF8052066210023734A05F0D5F88E211C
:100D080000230520714A05F0CFF80520704AB62166
:100D1800002305F0C9F84FF6FF7004F08BFF7D2023
:100D2800DC216C4AACE700204FF6E0710AF046FF80
:100D380031204FF6E0710AF041FF63204FF6E07171
:100D48000AF03CFF95204FF6E0710AF037FFC72004
:100D58004FF6E0710AF032FF4EF29C7004F06AFF21
:100D68000520012100235C4A05F09EF8052020217A
:100D780000235A4A05F098F8052052210023584AC2
:100D880005F092F8052084210023564A05F08CF8D6
:100D9800B62105203F4A002305F086F84FF4F0609D
:100DA80004F048FF012140F2131000234E4A05F0D9
:100DB8007BF840F2131020214C4A002305F074F808
:100DC80040F213105221334A002305F06DF840F227
:100DD80013108421464A002305F066F8B621454AD7
:100DE80040F21310002305F05FF84FF6FF7004F08F
:100DF80021FF7D20DC21404A42E700204FF6E071C8
:100E08000AF0DCFE31204FF6E0710AF0D7FE6320CD
:100E18004FF6E0710AF0D2FE95204FF6E0710AF025
:100E2800CDFEC7204FF4FC610AF0C8FE4EF29C705C
:100E380004F000FF052001210023304A05F034F8B2
:100E48000520202100232E4A05F02EF805205221E6
:100E580000232C4A05F028F88421002305202A4A7B
:100E680005F022F84FF4F06004F0E4FEB621052006
:100E7800264A002305F018F84FF6FF7004F0DAFE52
:100E88008720234ADC21FBE66FA00508A3A00508FC
:100E98009EA0050851A60508A2A00508D0A005082F
:100EA800BCA00508A7A00508B7A00508ACA00508C0
:100EB800B1A00508B6A00508BBA0050879A00508DB
:100EC800BFA00508C3A00508C7A00508CBA0050852
:100ED800CFA00508D3A00508DFA00508E3A00508F2
:100EE800E7A00508EAA00508F3A00508EFA0050893
:100EF800EEA00508F2A00508F7A0050802A105085C
:100F0800C8A00508C0A0050812A1050868A705081B
:100F180099A0050800204FF6E0710AF04FFE632003
:100F28004FF4FC610AF04AFE4FF6E071C7200AF060
:100F380045FE4FF6FF7004F07DFE002004F07CFFB4
:100F4800A520D721854A9BE6042004F075FF0020E0
:100F58004FF6E0710AF032FE31204FF6E0710AF0E8
:100F68002DFE63204FF6E0710AF028FE95204FF61B
:100F7800E0710AF023FEC7204FF6E0710AF01EFE6A
:100F88004EF29C7004F056FE052001210023744A9D
:100F980004F08AFF052020210023724A04F084FF10
:100FA800052052210023704A04F07EFF0520842189
:100FB80000236E4A04F078FF0520B6216C4A00230E
:100FC80004F072FF4FF6E07004F034FE40F20B10AC
:100FD8000121684A002304F067FF40F22B1020210A
:100FE800654A002304F060FF40F223105221634A4F
:100FF800002304F059FF40F21B108421604A0023AB
:1010080004F052FFB6215F4A002340F2131004F0A7
:101018004BFF4FF6FF7004F00DFE002004F00CFFAC
:101028006E20D221584A90E0042004F005FF0020E9
:101038004FF6E0710AF0C2FD27204FF6E0710AF082
:10104800BDFD4F204FF6E0710AF0B8FD77204FF64E
:10105800E0710AF0B3FD9F204FF6E0710AF0AEFD93
:10106800C7204FF6E0710AF0A9FD4EF29C7004F01B
:10107800E1FD052001210023444A04F015FF052065
:1010880016210023424A04F00FFF05203E210023C9
:10109800404A04F009FF052066213F4A002304F076
:1010A80003FF05208E213D4A002304F0FDFEB621F2
:1010B8003B4A0023052004F0F7FE4FF6FF7004F0CA
:1010C800B9FD002004F0B8FE6420D221354A3CE086
:1010D800042004F0B1FE00204FF6E0710AF06EFD26
:1010E80043204FF6E0710AF069FD85204FF6E07164
:1010F8000AF064FD4FF6E071C7200AF05FFD4EF27A
:101108009C7004F097FD05200121274A002304F074
:10111800CBFE05204521254A002304F0C5FE052005
:1011280087211F4A002304F0BFFEB621204A00236E
:10113800052004F0B9FE4FF6FF7004F07BFD002097
:1011480004F07AFE1B4A7D20D221002304F0ACFE75
:101158000420BDE8104004F06FBE10BD1AA50508B4
:1011680006A1050812A1050811A1050814A1050882
:1011780018A105081DA10508BCA0050824A105089B
:1011880028A105082DA1050833A1050839A10508DE
:10119800EFA00508F4A005083EA1050841A105082F
:1011A800D0A0050844A105084DA1050802A105081D
:1011B80051A60508C5A5050810B5064C064806231E
:1011C800237000F0BAFB2078FFF786FCBDE81040DA
:1011D8000DF04CBB242C00203017002010B5064C15
:1011E80006480723237000F0A8FB2078FFF774FC5B
:1011F800BDE810400DF03ABB242C00203017002029
:1012080010B5064C06480523237000F096FB20789D
:10121800FFF762FCBDE810400DF028BB242C00202D
:101228003017002010B5064C06480423237000F040
:1012380084FB2078FFF750FCBDE810400DF016BB8A
:10124800242C00203017002010B5064C0648032334
:10125800237000F072FB2078FFF73EFCBDE81040D9
:101268000DF004BB242C00203017002010B5064CCC
:1012780006480223237000F060FB2078FFF72CFC5F
:10128800BDE810400DF0F2BA242C002030170020E1
:1012980038B5094C05464FF6E071206801F050FF5B
:1012A80020680DB1054900E0054901F0F7FEBDE8E9
:1012B800384003F083B800BF340C002051A1050862
:1012C80064A105081A4B10B51C78012C14BF102412
:1012D8000024002C14BFD820C82006F033FA154982
:1012E8000246154815F07EFB002C14BFDC20CC20EC
:1012F80006F028FA0F490246104815F073FB002C37
:1013080014BFE020D02006F01DFA0A4902460C4816
:1013180015F068FB002C14BFE420D42006F012FA64
:10132800044902460748BDE8104015F05BBB00BF02
:10133800F40D002056A00508E02500200426002012
:10134800162C0020CC25002010B5E82006F0FAF96C
:101358000F4C024621460F4815F044FBEC2006F0DE
:10136800F1F9214602460C4815F03CFBF02006F046
:10137800E9F921460246094815F034FBF42006F045
:10138800E1F9024606482146BDE8104015F02ABB9F
:1013980056A00508E025002004260020162C002071
:1013A800CC2500200E4A012310B513700D4A0024E5
:1013B80014700D4A204613700AF0F6F9204604F01E
:1013C80065FC0A4B03221A700AF032FD0BF019FA79
:1013D800074B08481C70BDE8104000F0AEBA00BFCB
:1013E800242C00204F0D00204D0D0020A4250020A6
:1013F800043800201012002038B50D4B0D4D002484
:101408001C700D4B28681C700C4B4FF6E0711C705B
:1014180001F096FE28680A4901F040FE02F0CEFF6E
:10142800204604F033FC0748BDE8384000F085BA90
:10143800AC0D0020340C00204F0D0020A425002006
:1014480006A50508D417002007B50E4B0E481A78D4
:10145800D2F1010238BF00221A700C4B05221A7013
:1014680000F06BFA022201238DE80C00B020602105
:10147800102232230DF09EFB03B05DF804EB02F05E
:101488009DBF00BFAC0D0020C8100020A42500207F
:101498002E4A002310B513702D4A13700CF0DEFF8E
:1014A8000446002842D02B4C4FF6E071206801F02A
:1014B80047FE2068284901F0F1FD60684FF6E071A9
:1014C80001F03EFE6068254901F0E8FDA0684FF68E
:1014D800E07101F035FEA068214901F0DFFD02F05E
:1014E8006DFF4FF47A600AF039F820684FF6E07122
:1014F80001F026FE20681B4901F0D0FD60684FF618
:10150800E07101F01DFE6068164901F0C7FDA06892
:101518004FF6E07101F014FEA068124901F0BEFD1B
:1015280002F04CFFBDE8104002F048BF0CF07CFC14
:10153800204604F0ABFB0C4B0C4804221A7000F058
:10154800FCF9BDE81040FFF7FDB800BFAC0D002066
:101558004F0D0020340C002077A105088BA1050849
:101568009BA1050805A50508A4250020FC1300205B
:101578002DE9F04F6A4DDFF8F4916A4E85B00024EA
:101588004FF6FF78284602F0E0FC41462246234603
:1015980065480094019401F097FD042703904146A3
:1015A8002246234648460097019401F08DFD4146A6
:1015B80030602246234648460097019401F084FD96
:1015C800414670602246234648460097019401F040
:1015D8007BFDA8F50048B0604146224623465348A3
:1015E8000097019401F070FD4146F06022462346C1
:1015F8004F480097019401F067FD4146306122464B
:1016080023464C480097019401F05EFD2346706123
:101618004146224648480097019401F055FD474944
:10162800B061474A204602F047FA4649464A804692
:10163800204602F041FA4549454A8246204602F0D2
:101648003BFA4449444A0746204602F035FA4349E2
:10165800434A8146204602F02FFA4249424A8346CD
:10166800204602F029FA21468446039ACDF808C09C
:101678002B46204602F038FB052132682B46A02075
:1016880002F032FB692172682B46782002F02CFBAD
:101698007D21B2682B46782002F026FB2821F268CB
:1016A8002B46052002F020FB4B2132692B460520F2
:1016B80002F01AFB052072696E212B4602F014FB1A
:1016C8009121B2692B46052002F00EFBD2213A4641
:1016D8002B46052002F008FBD22142462B4660200B
:1016E80002F002FBD2214A462B46B02002F0FCFA57
:1016F800D22152462B464FF4807002F0F5FAB421FD
:101708005A462B46052002F0EFFADDF808C06020A3
:10171800B42162462B4605B0BDE8F04F02F0E4BAAA
:10172800A0140020340C0020ABA10508B5A10508C1
:10173800BCA10508C2A10508C8A10508CEA10508D5
:1017480099140008D6A1050801140008DEA10508AF
:1017580051140008E7A10508AD130008EFA105081A
:1017680051130008F8A10508CD12000802A50508C4
:10177800544A00232DE9F0471370534ADFF860916B
:101788001370524B1D780127BD4214BF1025002548
:10179800B842044689F8007003D0022840F08C80D3
:1017A8000BE021464FF4747005F0B3FF0AF066FAB7
:1017B800204605F0BBF920467CE0002D14BFD82058
:1017C800C82005F0BFFF0446002D14BFDC20CC2044
:1017D80005F0B8FF8046002D14BFE020D02005F0AA
:1017E800B1FF0646002D14BFE420D42005F0AAFF5F
:1017F80005460AF043FA364B36491A68A24218469B
:1018080002DB0B68434513DD334B04601E60334B2A
:10181800C1F800801D6009F087FF314B01221A7062
:10182800304A0520B4210023BDE8F04704F03CBB52
:10183800944218D1984516D1274B1B689E4212D165
:10184800264B1B689D420ED14FF47470394689F8B7
:10185800007005F05EFF244B00221A60234B4FF006
:101868007E521A6028E01E4B02251D7029464FF44F
:10187800747005F04EFF164B1B6806EE906A1C1B31
:10188800F8EEE67A06EE904AB8EEE67A164B87EE60
:10189800277A284683ED007A0F4B1B6806EE903AAC
:1018A800B8EEE67A114BC7EE277AC3ED007A05F059
:1018B8003DF90020FFF7ECFC0AF09FF9BDE8F0477E
:1018C80002F07CBDAC0D00204F0D0020F40D00206F
:1018D80018260020302C00200C2C0020C8250020C1
:1018E800B501002001A20508A0250020D825002068
:1018F80008B500F0A5FEFEF77FFC00F04FF800F0F9
:101908006FF8FEF789FEFEF7DDFCFFF769F801F0D6
:10191800A7FAFFF72DFE01F079F8FEF713FD01F0A5
:101928009BF900F06DFB00F081FD00F013FE00F064
:101938005FFABDE8084000F02DBB10B5044628B991
:101948000F48104A104B532102F060FF0F4B1868E4
:10195800844213D010B1C36900219847002004F0D5
:1019680095F9002004F07CF94FF6FF7004F062F955
:10197800E369204601219847044B1C6010BD00BF55
:1019880015A20508D41F040831A20508500C002030
:101998000048D2E7D41700200CF020BD10B5084C41
:1019A800204602F0D2FA00200649074A02F084F8DD
:1019B800D22102462346FA20BDE8104002F094B92D
:1019C800380E00204FA20508A1190008024B034851
:1019D80001221A70FFF7B1BFA4250020A01400202F
:1019E8002DE9F743374D384F384E0024284602F08A
:1019F800ACFA2246234647F6FF7135480094019415
:101A080001F062FB4FF6FF788146414622462346A5
:101A180038460094019401F057FB41463060224655
:101A2800234638460094019401F04EFB414670600D
:101A38002246234638460094019401F045FB23468C
:101A4800B0604146224638460094019401F03CFBC0
:101A58002049F060204A204602F02EF81F49204A0B
:101A68000746204602F028F8214680464A462B467B
:101A7800204602F039F93C2132682B46192002F041
:101A880033F95A2172682B46192002F02DF9782172
:101A9800B2682B46192002F027F99621F2682B46E6
:101AA800192002F021F9D2213A462B46EC2002F007
:101AB8001BF99C20D22142462B4603B0BDE8F043D7
:101AC80002F012B91012002002A50508540C0020DB
:101AD80041A205084EA20508D519000857A2050815
:101AE800A51C000870B5474E474C327847492DED84
:101AF800028B142592B005FB02420C320FA814F099
:101B080071FF33780D2B05FB03F504EB050332D881
:101B1800D3ED016A9B6807EE103A6359B8EEE68A7E
:101B280006EE903ADFED3A7AF8EEC78AB8EEE67A32
:101B380088EE278AC8EEA78AC7EE277A17EE900A9A
:101B480010F0DAF802460B466846324914F04AFFAC
:101B580018EE100A10F0D0F802460B4605A82E49D8
:101B680014F040FF18EE900A10F0C6F802460B4633
:101B78000AA82A4929E093ED017A9B6807EE903A72
:101B8800635906EE903AF8EEE78AF8EEE67AB8EE90
:101B9800C78A17EE900A10F0AFF802460B4668465F
:101BA8001F4914F01FFF18EE100A10F0A5F802469E
:101BB8000B4605A81B4914F015FF18EE900A10F003
:101BC8009BF80B46184902460AA8184C14F00AFF5D
:101BD8002068174901F062FA20680FA901F05EFA3F
:101BE8006068694601F05AFAA06805A901F056FA3A
:101BF800E0680AA901F052FA02F0E0FB12B0BDEC6D
:101C0800028B70BD162600200000002060A2050887
:101C180000007A446BA205087CA205088DA205087D
:101C28009EA20508AFA20508C0A20508540C002012
:101C38000BA5050808B5114B114A1B780D2B8CBF55
:101C480000210121117014225A430E4988588B181B
:101C58004FF47A720C495043086059684A430B495B
:101C68000A609A680A4B1A6009F05EFD094B0A4837
:101C780001221A70BDE80840FFF75FBE1626002053
:101C8800F40D00200000002018260020302C002031
:101C98000C2C0020A4250020A0140020CAE700BFB7
:101CA8004FF6FF7070474FF6FF7070471FB5002959
:101CB80047D04FF2DE7003F0E9FF002004F0BCF8D3
:101CC8000F2003F0B7FF1F4C1F4A412101230A20B0
:101CD80004F0EAF8042004F0AFF8236828209621DD
:101CE800042B24DC0123194A04F0DEF803A90DF1C2
:101CF8000E02206804F060FB0F2003F09BFFBDF884
:101D08000C00BDF80E1014380F242822002380B2CE
:101D1800009403F0BFFFBDF80E10BDF80C0000944E
:101D2800143989B22822012303F0B4FF09E0084AD4
:101D3800012304F0B9F81E20A521064A012304F066
:101D4800B3F81FBD640C0020D1A20508E4A2050861
:101D580000A3050816A3050837B51E4C2368042BF5
:101D680005462BDC01A80DF1060104F023FBBDF8A4
:101D78000630BDF80420184904200DF071F82368D6
:101D8800002B04DA1548164A164B592105E0042B96
:101D980005DD1248124A144B5A2102F037FD04EBB4
:101DA8008302BDF8041001339180BDF8061023604A
:101DB800052BD18008D1201D04F07EFB00230B48A1
:101DC8002360FFF7BAFD03E028460121FFF76EFF05
:101DD8003EBD00BF640C00202DA3050872A30508B2
:101DE800E61F040894A30508ABA30508E81500201E
:101DF80037B50B4C204602F0A8F80A4B0A49009365
:101E080000250120094A0A4B019501F046FF2946A1
:101E180002462346284603B0BDE8304001F064BFBF
:101E2800B4120020B51C0008A91C0008AF1C00084B
:101E3800611D00084FF6FF7070474FF6FF7070473E
:101E480030B54FF6E07087B003F020FF002003F0B4
:101E5800F3FF0F2003F0EEFE00212C4A2C4C012347
:101E68000A2004F021F8002003F0E4FE042003F027
:101E7800E3FF0A201921274A012304F015F8252138
:101E8800254A01230A2004F00FF81F2003F0D2FE90
:101E980001230A203721214A04F006F82378002B71
:101EA80031D001231E2096211D4A03F0FDFF6288D0
:101EB8001C4902A814F096FD01231E20A22102AAA3
:101EC80003F0F2FFA288184902A814F08BFDAE2196
:101ED80002AA01231E2003F0E7FF0F2003F0AAFE49
:101EE8006088A188143880B20F2528220023009525
:101EF80003F0D0FEA18860880095143989B22822A1
:101F0800012303F0C7FE07B030BD00BFD9A3050801
:101F18007C0C0020EBA305080BA405082BA40508DE
:101F28004EA4050860A405086DA4050801B187E75B
:101F3800704713B50DF1060101A804F0EFF9144B31
:101F480001221A705988BDF80420891A0E311C29FB
:101F580019460AD89C88BDF80600201A0E301C289D
:101F680003D899680131996001E000238B60084B20
:101F78009968012905DD00229A601A70FFF708FDAB
:101F880005E05A80BDF806209A80FFF759FF1CBD6E
:101F98007C0C002037B50B4C204601F0D6FF0A4BCD
:101FA8000A49009300250120094A0A4B019501F0CE
:101FB80074FE294602462346284603B0BDE8304051
:101FC80001F092BEE8150020351F00083D1E0008EC
:101FD800431E00083B1F000808B5064B00221A7074
:101FE800054B186814F094F90448BDE80840FFF759
:101FF800A4BC00BFA4250020F0350020D417002081
:102008002DE9F04F514D524E85B00024284601F07D
:102018009CFF2246234647F6FF714E4800940194E0
:1020280001F052F84FF6FF770390394622462346CF
:1020380049480094019401F047F839463060224637
:10204800234646480094019401F03EF84FF00108F9
:102058007060224623464FF6E0714148CDF8008073
:10206800019401F031F82346B060394622463D48D4
:10207800CDF80080019401F027F83B49F0603B4A15
:10208800204601F019FD3A493A4A0746204601F030
:1020980013FD3949394A8046204601F00DFD38497B
:1020A800384A8146204601F007FD3749374A8246BB
:1020B800204601F001FD3649364A8346204601F0A4
:1020C800FBFC21468446039ACDF808C02B462046DF
:1020D80001F00AFE3C2132682B46142001F004FE70
:1020E8003C2172682B46EC2001F0FEFDB421B26859
:1020F8002B460F2001F0F8FDD2213A462B46E62068
:1021080001F0F2FD642142462B46052001F0ECFD6A
:102118004A462B460520872101F0E6FD52462B460C
:102128000520D22101F0E0FDD2215A462B4650204D
:1021380001F0DAFDDDF808C09B20D22162462B466B
:1021480005B0BDE8F04F01F0CFBD00BFDC0E0020A8
:10215800880C00207AA4050884A40508FEA10508B7
:1021680000A5050802A505084EA20508E11F0008FC
:10217800E89F0508C9210008F89F0508C92200083A
:102188008DA40508D123000895A405088D2300080F
:102198009DA405084923000808B50BF05DFE4FF41F
:1021A80041400CF095FB044B186807F043F8034BCB
:1021B80009221A7008BD00BF10260020A42500209F
:1021C80010B50C4CFFF7E8FF0B4A0023B42005219B
:1021D80003F06AFEA0684FF6E07100F0B1FFA06856
:1021E800064900F05BFF0BF037FEBDE8104002F037
:1021F800E5B800BF880C002008A50508A5A40508B7
:10220800264B2DE9F7431888C00014F079F80546E5
:1022180028B90520B421224A2B4603F045FE214B5C
:10222800DFF878801D6000240BF016FE26461E4F4E
:10223800DFF8889023E009F0CFF83B68D9F8000070
:1022480045F8083C7B6845F8043C184B1B68C018E7
:1022580006F0F0FF164B186809F080F9B8F800008E
:1022680094FBF0F080B24FF4FC63009328210246FF
:10227800322303F06BFC04F59E7401360334B8F87E
:1022880000300835B342D6DA0A4B186806F0D2FF98
:10229800094B09221A70BDE8FE8300BFFC390020F3
:1022A800BEA40508F0350020BC3700209C2500207E
:1022B800C825002010260020A4250020F83500207D
:1022C80010B5094CFFF79CFFA0684FF6E07100F0CD
:1022D80037FFA068054900F0E1FE0BF0BDFDBDE841
:1022E800104002F06BB800BF880C0020CCA4050891
:1022F80010B5074C4FF6E071A06800F021FFA06808
:10230800044900F0CBFEBDE8104002F057B800BF0A
:10231800880C0020E6A4050810B5074C4FF6E071BC
:10232800A06800F00DFFA068044900F0B7FEBDE802
:10233800104002F043B800BF880C0020FCA4050838
:1023480010B50C4C0B2323700B4B01221A70002084
:1023580002F06AFF0948FFF7F0FA2078FEF7BCFBA5
:10236800074B032093ED000A0BF085FDBDE81040F4
:10237800D2E700BF242C0020500D00203017002089
:102388000C03002038B50C4D0C232B700B4B01248B
:102398001C70002002F048FF0948FFF7CEFA2878A1
:1023A800FEF79AFB074B204693ED000A0BF063FDFE
:1023B800BDE83840B0E700BF242C0020500D0020B5
:1023C800301700200C03002010B50C4C0923237093
:1023D8000B4B01221A70002002F026FF0948FFF774
:1023E800ACFA2078FEF778FB074B022093ED000A41
:1023F8000BF041FDBDE810408EE700BF242C002003
:10240800500D0020301700200C0300200CF0ACB851
:10241800034A044800231370034A1370FFF78DBA68
:1024280004380020D4170020A42500202DE9F74304
:10243800384D394EDFF8FC800024284601F085FD30
:102448002246234647F6FF7134480094019400F071
:102458003BFE4FF6FF7781463946224623463048F1
:102468000094019400F030FE39463060224623463D
:1024780040460094019400F027FE394670602246D9
:10248800234640460094019400F01EFE2346B060A7
:102498003946224640460094019400F015FE214931
:1024A800F060214A204601F007FB2049204A0746F0
:1024B800204601F001FB214680464A462B4620462D
:1024C80001F012FC3C2132682B46282001F00CFC5C
:1024D8005A2172682B46192001F006FC7821B2684F
:1024E8002B46192001F000FC9621F2682B46192092
:1024F80001F0FAFBD2213A462B46EC2001F0F4FB1E
:102508000520D22142462B4603B0BDE8F04301F036
:10251800EBBB00BF24100020980C002016A505086E
:102528001EA505084EA205081924000829A50508B6
:102538001524000802A50508034A0448002313705F
:10254800034A1370FFF7F9B904380020D4170020A4
:10255800A42500202DE9F743324E334DDFF8DC8007
:102568000024304601F0F1FC2246234647F6FF716D
:102578002E480094019400F0A7FD4FF6FF7781469E
:102588003946224623462A480094019400F09CFDCF
:10259800394628602246234640460094019400F0BC
:1025A80093FD3946686022462346404600940194CC
:1025B80000F08AFD2346A86039462246404600942A
:1025C800019400F081FD1B49E8601B4A204601F098
:1025D80073FA214607464A463346204601F084FBF3
:1025E8003C212A683346192001F07EFB5A216A688B
:1025F8003346192001F078FB7821AA683346192060
:1026080001F072FB9621EA683346192001F06CFB51
:10261800EC20D2213A46334603B0BDE8F04301F03E
:1026280063BB00BF78180020A80C002031A505085E
:102638003FA505084EA205084125000802A5050882
:1026480010B50B4C204601F080FC002001462246C4
:1026580000F09AFD00200749074A01F02DFAD2211F
:10266800024623464FF48270BDE8104001F03CBB9F
:10267800301700204CA50508A926000870B5C92404
:102688000AE0A8B200223146013502F05DFCF02DC7
:10269800F7D10134EF2C02D00025A6B2F1E770BDC6
:1026A80010B51A4C2378092B08D1194A0023137046
:1026B800184A1370FFF7E2FF174823E00A2B0ED1E0
:1026C800164B186813F024FE154A00231370114A9C
:1026D8001370144A1370FFF7D1FF134812E000205B
:1026E80002F0A2FD114A00231360114A13800D4B1A
:1026F80002221A700F4B186806F09CFD22780E4BC8
:102708000E481A70BDE81040FFF717B9A42500203D
:10271800500D00204F0D0020DC0E0020F035002069
:10272800510D002004380020241000209C0D0020AA
:10273800AA0D002010260020C22500206C110020C0
:10274800034B01224FF4FC601A7003F073BA00BF08
:102758004F0D0020044B054800221A70044B0C2230
:102768001A70FFF7EAB800BF4F0D00207818002054
:10277800A425002007B50A4A0023137004228DE817
:102788000C00C6201022232356210CF013FA054B07
:1027980005480A221A7003B05DF804EBFFF7CDB8BC
:1027A8004F0D0020A42500202410002007B50A4A58
:1027B8000023137004228DE80C0097201022232395
:1027C80056210CF0F7F9054B054809221A7003B099
:1027D8005DF804EBFFF7B1B84F0D0020A4250020E9
:1027E800DC0E002007B50B4B00221A7008220323C9
:1027F8008DE80C004920102223233D210CF0DAF942
:10280800054B064801221A7003B05DF804EBFFF788
:1028180094B800BF4F0D0020A4250020A01400206C
:1028280008B501214FF080400EF015FB0A4B00203F
:1028380018700A4B18700A4B18700A4B08221A7045
:10284800094B187003F022FA084B094801221A7044
:10285800BDE80840FFF771B8C3250020AC0D002083
:102868004F0D0020A4250020242C0020083600202D
:10287800380E002070B51F4C1F4E20684FF6E075CB
:10288800294600F05DFC20681C4900F007FC6068E0
:10289800294600F055FC6068194900F0FFFBA06864
:1028A800294600F04DFCA068164900F0F7FB01F03E
:1028B80085FD4FF47A6008F051FE2068294600F043
:1028C8003FFC2068314600F0E9FB6068294600F0CB
:1028D80037FC6068314600F0E1FBA068294600F04B
:1028E8002FFCA068314600F0D9FBBDE8704001F02C
:1028F80065BD00BFB80C002005A5050877A105082F
:102908008BA105089BA105080C4B10B500241C7071
:102918000B4B01221A70204608F046FF204603F0B0
:10292800B5F9084B0B221A7009F082FA09F069FF11
:102938000548BDE81040FFF700B800BF4F0D002064
:10294800242C0020A4250020441500200F4A002331
:1029580010B513700E4A13700BF080FD044628B1B1
:10296800FFF788FFBDE8104001F028BD03F08EF99D
:1029780009F084F9074B1C70074B07221A7009F0FD
:1029880077F90648BDE81040FEF7D7BFAC0D002028
:102998004F0D0020242C0020A425002058130020CF
:1029A80010B54FF0804001210EF055FA114A00236E
:1029B8001370114A1370114A13700BF04FFD04463F
:1029C80028B1FFF757FFBDE8104001F0F7BC03F04E
:1029D8005DF909F053F906F085FC094B1C70094BA9
:1029E80006221A7009F044F90748BDE81040FEF7BE
:1029F800A4BF00BFC3250020AC0D00204F0D002050
:102A0800242C0020A4250020800F00202DE9F04F61
:102A18006D4DDFF810928BB000244FF6FF782846F2
:102A280001F093FA414622462346684800940194EF
:102A380000F04AFB4FF6E076042704903146224620
:102A4800234663480097019400F03EFB3146059009
:102A5800224623465F480097019400F035FB414623
:102A680006902246234648460097019400F02CFB26
:102A7800594E414630602246234648460097019405
:102A880000F022FB234670604146224648460097E4
:102A9800019400F019FB5149B060514A204601F0F9
:102AA8000BF85049504A0746204601F005F84F49AF
:102AB8004F4A8046204600F0FFFF4E494E4A814665
:102AC800204600F0F9FF4D494D4A8246204600F065
:102AD800F3FF4C494C4A8346204600F0EDFF4B4932
:102AE8004B4A84462046CDF80CC000F0E5FF494922
:102AF8000790494A204600F0DFFF48490890484AB5
:102B0800204600F0D9FF21460990049A2B4620461A
:102B180001F0EAF82146059A2B46C82001F0E4F8AE
:102B28000A21069A2B46C82001F0DEF855213268A2
:102B38002B46782001F0D8F8692172682B46782056
:102B480001F0D2F87D21B2682B46782001F0CCF84C
:102B580005203A4628212B4601F0C6F8D2214246E4
:102B68002B46052001F0C0F8D2214A462B465620B4
:102B780001F0BAF8D22152462B46A62001F0B4F84B
:102B8800B4215A462B46052001F0AEF8DDF80CC0FA
:102B9800B42162462B46562001F0A6F8B421079AC4
:102BA8002B46A62001F0A0F8B421089A2B46F6205F
:102BB80001F09AF8099AF620D2212B460BB0BDE80D
:102BC800F04F01F091B800BFD417002051A50508B7
:102BD8005AA5050867A50508B80C002072A50508C0
:102BE800ED2700087AA505081129000883A505081E
:102BF800A92900088CA505085529000895A50508E8
:102C0800292800089EA50508B5270008A7A50508D6
:102C18007D270008B0A505085D270008B8A50508A8
:102C28004927000802A5050807B5032308228DE8EF
:102C38000C004920102223233D210BF0BBFF044B3D
:102C4800044801221A7003B05DF804EBFEF775BE64
:102C5800A4250020A01400202DE9F743314E324F5F
:102C6800324D0024304601F070F92246234647F6DB
:102C7800FF712F480094019400F026FA4FF6FF7870
:102C8800814641462246234638460094019400F086
:102C98001BFA414628602246234638460094019490
:102CA80000F012FA414668602246234638460094EE
:102CB800019400F009FA2346A860414622463846A6
:102CC8000094019400F000FA1A49E8601A4A204674
:102CD80000F0F2FE214607464A463346204601F0F8
:102CE80003F83C212A683346192000F0FDFF5A21D9
:102CF8006A683346192000F0F7FF7821AA6833463E
:102D0800192000F0F1FF9621EA683346192000F0F7
:102D1800EBFFEC20D2213A46334603B0BDE8F0433E
:102D280000F0E2BFC810002002A50508C40C00206E
:102D3800C0A505084EA20508312C00081C4B1A78BE
:102D48001C4B10B51A7009F079F81B4B1B4A00246C
:102D58001C6002202346CA2103F0A6F8204608F08A
:102D680023FD174B1C80174B1C70174B1B78023B1D
:102D7800052B1CD8DFE803F003070B13170FBDE87A
:102D88001040FEF773BABDE81040FEF75DBABDE823
:102D98001040FEF747BABDE81040FEF71FBABDE87D
:102DA8001040FEF72DBABDE81040FEF705BA10BD79
:102DB800C2250020A42500209C0D002001A505089F
:102DC8000436002004380020242C002008B5084BC5
:102DD800186806F02FFA002002F058FF09F028F8CA
:102DE800044B05480B221A70BDE80840FEF7A5BD44
:102DF80010260020A425002044150020114B10B5F2
:102E080000241C70104B186806F014FA204602F0D3
:102E18003DFF0E4B1B780B2B0ED8DFE803F00606A0
:102E28000D0D0D0D0A080D0D0D06094802E00948A3
:102E380000E00948FEF781FD084B1C70BDE8104012
:102E480008F0F6BF242C002010260020A42500201E
:102E5800D417002058130020800F002004380020C9
:102E68002DE9F041144C204601F06FF80020134979
:102E7800134A00F021FE1349134A0746002000F0C8
:102E88001BFE1249124A0646002000F015FED22108
:102E980005463A462346E62000F026FF4B213246F7
:102EA8002346642000F020FF642069212A46234637
:102EB800BDE8F04100F018BF6C1100205BA00508C8
:102EC800052E0008C8A50508D52D0008D4A50508B5
:102ED800452D000808B508B143682BB90348044AD2
:102EE800044B9B2101F092FC586908BDE1A5050837
:102EF800F81F040803A6050808B5FFF7EBFF80686C
:102F0800123080B208BD08B5FFF7E4FF406806300C
:102F180080B208BD2DE9F84F04468846FFF7DAFF6E
:102F28006689E589074606F1030905F10F0AB8F134
:102F3800000F1FD01F2002F07DFE2046FFF7DCFFA8
:102F480083462046FFF7DFFF294603465FFA8BF2E8
:102F5800F0B202F0AFFE042002F06EFF0B364FF61F
:102F6800FF70033502F066FEB0B2A9B23A680123D9
:102F780002F09AFF3D69204641464A465346A84713
:102F8800BDE8F88F13B504460DF1060101A803F05A
:102F9800C5F92046FFF79EFF6389BDF80410BDF808
:102FA8000620C91AE389D21A0339C3680F3A2046A2
:102FB80098471CBDF7B5044614200D4616461F4613
:102FC80013F09EF9089BC7600361064B0649074A40
:102FD80080E8700000930190054B002000F05DFE32
:102FE800FEBD00BF1D2F00080F2F0008012F00088D
:102FF8008D2F0008704708B508B143682BB90448FD
:10300800044A054BAD2101F001FC586908BD00BF19
:1030180022A605081020040803A60508F8B50546E9
:103028000E46FFF7E8FF836B04461BB1284631467E
:10303800984700E018466F8994F83C30ED890EB93E
:10304800034310D0208E02F0F5FD608E02F008FEDA
:1030580094F8350002F0F0FE94F8343038462946EA
:10306800224602F021FF002384F83C30F8BD08B561
:10307800FFF7C1FF90F83500BDE8084002F0F1BE47
:1030880038B5FFF7B8FF044613F032FD054694F84B
:10309800350002F0E1FE684380B238BD38B50D4610
:1030A800FFF7A9FF29462E22044613F051FD50B11F
:1030B800204629462E2213F09DFD002384F82E3049
:1030C800012384F83C3038BD2DE9F74307464020FA
:1030D8000E461546984613F013F9044628B91148C8
:1030E800114A124B4E2101F091FB114B114A124922
:1030F8008DE818000020114B00F0CFFD39468146BD
:10310800FFF7CCFF9DF82830268684F835300B9BD6
:103118006586A363002384F8348084F83C304846ED
:10312800BDE8FE8322A605082820040840A6050855
:10313800253000087730000889300008FD2F000886
:1031480010B50C46FFF757FF0123048680F83C3082
:1031580010BD00BF4FF4A0707047C820704770477B
:10316800074B1B78022B07B508D1064B1B78022B9F
:1031780004D001A80DF1060103F0D0F80EBD00BF80
:1031880004380020242C002073B50A4B06460D464F
:103198001446009300200849084A094B019000F0A2
:1031A8007CFD294602462346304602B0BDE8704001
:1031B80000F09ABD673100085D31000863310008EE
:1031C8006931000813B502AB03E90600436843B14F
:1031D800027C0124082A9C7004D11B692146984767
:1031E80000E01C4620461CBD30B500282BD0058BBE
:1031F800002425E0036A1A7C012A05D15B681A8835
:103208008A421BD1187F30BD052A06D15B681A880F
:103218008A4213D193F82C0030BD032A06D15B688B
:103228001A888A420AD193F8250030BD062A05D1AA
:103238005B681A888A4201D1D87A30BD01340430DB
:10324800AC42D7D3002030BD08B18175012070474A
:10325800F8B504460D46D0B1E175D0F898309847D6
:10326800012D0DD12746002606E0F86900F1080275
:10327800436906CA98470136238B04379E42F4D324
:10328800D4F898302046294698470120F8BDF8BD63
:10329800F8B50546084617460E4613F029FC013FC7
:1032A800B84234BF04463C463CB128463146224623
:1032B80013F0A0FC00232B55F8BD2C70F8BDF7B512
:1032C800044600200090019000296CD00E8B68E025
:1032D80000F1080351F823301D7C042D04D15D68EA
:1032E8002D88954247D0013000F1080351F823306A
:1032F8001D7C012D04D15D682D8895423BD001309D
:1033080000F1080351F823301D7C052D04D15D68B8
:103318002D8895422FD0013000F1080351F8233051
:103328001D7C032D04D15D682D88954223D0013082
:1033380000F1080351F823301D7C022D04D15D688B
:103348002D88954217D0013000F1080351F8233039
:103358001D7C072D04D15D682D8A95420BD0013064
:1033680000F1080351F823301D7C062D08D15D6853
:103378002D88954203D103F10801204615E001305C
:1033880000F1080351F823502B7C082B09D16F68F2
:103398003F88974204D105F1080120461A4605E006
:1033A8000130B04294D320466946082213F058FAF7
:1033B8002046FEBDF8B505460F461646002830D013
:1033C8004388032B2FD0202012F09AFF04460028B0
:1033D8002BD040F80C5B39460C22FFF759FF182018
:1033E800E66112F08DFF0646B8B10223037401238B
:1033F80063760F4B446063600E4BA3600023237613
:103408006B8805EB830201339BB2012B50606B8004
:103418000CD16A685268137608E0204612F078FFEB
:1034280004E0064602E0002600E006463046F8BD05
:10343800749F0408129C040837B5456802AB03E979
:1034480006003DB3037C0124042B85F8314022D1CA
:10345800688E02F0EFFB95F8300002F0EDFC95F86D
:10346800343043B9BDF80200BDF80610AA1C234643
:1034780002F01AFD0FE0012B03D1084840F2395140
:1034880004E0022B07D1054840F24151044A054B9C
:1034980001F0BCF92C4620463EBD00BF53A60508E6
:1034A800E86A040851A60508F8B504460F4616460A
:1034B80010B3838A0A2B20D0202012F021FF054662
:1034C800E8B14460102200F108003946FFF7E0FE39
:1034D8004FF6FF73A08A2B801F236B8000232B7667
:1034E800831D013080B20128EE6144F82350A08288
:1034F80007D1A3691876F8BDF8BD0020F8BD0120F2
:10350800F8BD0120F8BD2DE9F3471D464B1C984234
:1035180082460C461746BDF828600DDD95420BDC47
:1035280001320AF101035B1A521BC8B2D2B29BB234
:103538002946009602F0B6FBAAF1020A3046C4EB0F
:103548000A0A02F077FB4FF000084FF001091FFA52
:103558008AFA0BE0601C08EB050180B289B252467A
:103568000023009602F096FB09F101097B1B08F184
:10357800010899451FFA88F8ECD3BDE8FC87F8B52F
:10358800C7B2144638461E460D4602F095FB621E29
:1035980092B23846294602F08FFB304602F04AFBC9
:1035A800022606E0A21B92B23846294602F084FBA6
:1035B8000136A642F6D3F8BD73B504460E4600F1AF
:1035C8001E001546009200233C2280B21E3E02F0E7
:1035D80061FBB1B220463C220123009502F05AFB60
:1035E8007CBD73B504460E4601381546009200238B
:1035F800032280B2013E02F04DFBB1B22046032205
:103608000123009502F046FB7CBDF7B5089D2E7B93
:10361800EF7A1C463604AB7A06EB0726F618431AEF
:10362800687B06EB00602D1800200190121B0846ED
:103638002146009501F026FFFEBD30B5456885B0EE
:1036480004AB03E906007DB101242C736D68BDF855
:103658000800BDF80A109DF80C209DF80E30009562
:10366800FFF7D3FF204600E0284605B030BD2DE91E
:10367800F04385B004AB03E906004468BDF8086070
:10368800BDF80C70002C41D0012384F8263094F842
:1036980025300BB9A26800E06268FFB2BDF80A10D5
:1036A8009DF80E30009230463A46FFF7AEFF04F11F
:1036B8000C08022002F0C0FB404613F019FA054638
:1036C80000B1451E0F3F0024153E1FFA87F90DE093
:1036D80002F0BCFB02F0C0FB04FB106189B2484653
:1036E8002022002302F0FAFB0134E4B2AC42EFD30B
:1036F800002002F09FFAB8B2B1B24246012302F0AC
:10370800EDFB002002F098FB012000E0204605B008
:10371800BDE8F0832DE9F04385B004AB03E906006A
:103728004568BDF80860BDF80C70002D3CD0012339
:103738006B762B7EBDF80A10012B0CBF6A68AA684D
:103748009DF80E300092FFB23A463046FFF75DFF13
:103758000C35022002F070FB284613F0C9F90E3F21
:1037680081460024163E1FFA87F80DE002F06EFB32
:1037780002F072FB04FB106189B24046202200234C
:1037880002F0ACFB0134E4B24C45EFD9002002F062
:1037980051FAB8B2B1B22A46012302F09FFB0020C9
:1037A80002F04AFB012000E0284605B0BDE8F0839E
:1037B8002DE9F04F85B00546DDF840900291484666
:1037C8009046039313F094F9DDF838A0DDF83CB087
:1037D8000646294600242F4611E024B1B4420CBF06
:1037E8005B46534600E0039B01F10805ADB2009328
:1037F8002846029A4346FFF708FF01342946B44297
:10380800EBDD002002F016FA022002F015FB7D1D08
:1038180008F10508A8B21FFA88F14A46012305B045
:10382800BDE8F04F02F040BB70B5406886B006AB0B
:1038380003E9060000282ED0012380F82D30866881
:10384800164BF21A534243EB020390F82C205AB15C
:10385800002B134D134B144A08BF1D46134B00F1A0
:103868001C0418BF13460AE0002B0D4D0D4B0E4AE1
:1038780018BF1D460D4B00F10C0408BF1346BDF8D8
:103888001200BDF81410BDF8162000960195029498
:10389800FFF78EFF012006B070BD00BF5874040802
:1038A800947004083A760408767204081C780408B0
:1038B80070B5446886B006AB03E9060004B301237B
:1038C8006377A668104B227FF11A4B4243EB010342
:1038D8000AB10BB904E01BB966680C4D0C4B01E04A
:1038E8000C4D0D4BBDF81200BDF81410BDF8162094
:1038F80000960C3401950294FFF75AFF012000E06E
:10390800204606B070BD00BFA47F0408E07B040811
:10391800C27D04087A810408508304082DE9F04325
:1039280085B004AB03E906004468BDF80860BDF83B
:103938000A90BDF80C50BDF80E80002C00F08C8069
:103948000123A3740220676802F076FA4FF6FF702D
:1039580002F086F9002002F06DF9EDB25FFA88F8FE
:10396800A6F1160189B230462A4643460097FFF76A
:103978004CFE277A002F2ED1A28A234600E0013779
:10398800974204D29969097E04330029F7D002F0DE
:103998005DFA02F061FAA9F116091FFA89F90E21F8
:1039A80001FB10914FF6FF7208F101085FFA88F3E6
:1039B80089B2009248462A46FFF7A5FD022002F088
:1039C8003BFA1F2002F036F9A38A002B38D0103DAD
:1039D800E8B2303E2CE0E3685C68A28A2346013AEC
:1039E800002700E00137974204D29969097E043321
:1039F8000029F7D002F02AFA02F02EFA0E2101FB74
:103A080010914FF6FF7208F101085FFA88F389B246
:103A1800009248462A46FFF776FD022002F00CFA8B
:103A28001F2002F007F9A38A53B1103DE8B21A3EED
:103A38000637B1B254F827200123083202F04EFAB3
:103A4800002002F0F9F94FF6FF7002F009F91F2083
:103A580002F0F0F8012000E0204605B0BDE8F08350
:103A68002DE9F04105463620884614461F4612F0D7
:103A780047FC0646E0B120F8025B41462E22FFF7DC
:103A880007FCBDF8183086F83440738618200123E7
:103A980086F8307086F8313012F032FC044618B1DE
:103AA80004234660037404E0304612F031FC00E061
:103AB80004462046BDE8F081F8B5064624200F46A6
:103AC800154612F01DFC0446D8B10F4B06808360E2
:103AD8000E4B39464360102200F10C00FFF7D8FB6B
:103AE80001260023182025622377667712F008FC48
:103AF800054610B14460067404E0204612F008FC44
:103B080000E005462846F8BDA47F0408FE790408AD
:103B1800F8B506462C200F46154612F0F1FB044670
:103B2800E8B120F80C6B39461922FFF7B1FB0D4BB1
:103B3800A562A3600C4B6360002384F8253018202D
:103B4800012384F8263012F0DBFB054618B1032365
:103B58004460037404E0204612F0DAFB00E00546F6
:103B68002846F8BDB09804084E95040810B50446D8
:103B7800142012F0C5FB20B100234380014B0480C0
:103B8800036110BDBD33000838B50546442012F066
:103B9800B7FB0446C0B10E4B058243600D4B036072
:103BA800012383740023037283820B4B0364182060
:103BB80012F0A6FB054618B107234460037404E01D
:103BC800204612F0A5FB00E00546284638BD00BF98
:103BD800449104083A8D0408B13400082DE9F041F5
:103BE80005463420884614461F4612F089FB0646CF
:103BF80020B3144B05808360134B41464360102269
:103C080000F10C00FFF744FB214606F11C001022CE
:103C1800FFF73EFB002386F82C301820012337637A
:103C280086F82D3012F06CFB044618B10523466067
:103C3800037404E0304612F06BFB00E004462046B3
:103C4800BDE8F08158740408B26E04082DE9F0410B
:103C5800044614200D461646984612F051FB0746B6
:103C6800B8B1069B048003610023C3720123456039
:103C7800068180F80A800373182012F041FB04467D
:103C880018B106234760037404E0384612F040FB7D
:103C980000E004462046BDE8F0812DE9F0410446E5
:103CA80018200D461646984612F02AFB0746B8B16A
:103CB80001238370069B04800361079B456086602F
:103CC800C0F80C804361182012F01AFB044618B1A2
:103CD80008234760037404E0384612F019FB00E03B
:103CE80004462046BDE8F0812DE9F34198461B8B38
:103CF8001D2B05460C4617464FF0000000F2B48015
:103D0800B5F5A07F0090019000F2AE80F02900F296
:103D1800AB80127CADF80610511EADF80250072991
:103D280000F28A80DFE801F045595E04456A14769E
:103D38007B684E4A7A611A8893F834303A80013B9E
:103D4800DBB2012B7FD8ADF80240ADF806507AE01F
:103D580005F11602ADF8002004F11602ADF80420B2
:103D680002AE434A16E903007A6107F1080282E8C5
:103D7800030003F10802013348F82270A8F818304C
:103D88007B681A8A187A3A8000286CD1FFF7FCFE03
:103D98003849436859603849DF600126163D196083
:103DA80002461E72A8B2E1B24346FFF79DFF3046B5
:103DB8005AE0012A0CBF314B314B78687B6130F8EF
:103DC8000C3B3B8012F094FE431CDB001A34ED18C8
:103DD800ADF80440ADF8005035E07B68294A1B680F
:103DE8007A6102E0284A7B687A611B8814353B8037
:103DF800ADF800501434ADF8044024E07B68234A41
:103E08007A611A883A801A899B7AAD18ADF8005001
:103E1800E418F0E77E681E4B7B61338838463B80A8
:103E280073689847013D4519ADF80050B3683846A6
:103E38009847013C0419DEE71648174A174B40F229
:103E48001A3100F0E3FC02AA12E9030007F10803A3
:103E580083E80300B8F8183003F10802013348F882
:103E68002270A8F818300120BDE8FC814134000810
:103E7800253900083089040826850408B93800085F
:103E8800313800081D370008773600084336000827
:103E9800CD31000853A60508F86A040851A605089C
:103EA800F8B51646002834D01378002B2ED0028B94
:103EB800002327E0046A257C042D21D165682F881A
:103EC8008F421DD195F8313053B16F8E01F0D8FE75
:103ED80004F1080268866369204606CA98476F8617
:103EE800A81C31462E22FFF7D3F995F831307BB163
:103EF80004F108026369204606CA98470120F8BD04
:103F0800013304309342D5D30020F8BD1846F8BDDC
:103F18000120F8BD70B5B8B1068B0446002310E047
:103F2800256A287C04280AD16D682888884206D129
:103F38001046A91C2E22FFF7ABF9012070BD0133F2
:103F48000434B342ECD3002070BD38B5044620B326
:103F5800134BC361134BC0F89830134BC0F89C3017
:103F6800124B00257822C0F8A0308575C5750583E9
:103F7800294600F1200012F0B5FCD4F8983020460C
:103F8800294698470A4A1388312B07D8094941F826
:103F9800234001331380012038BD38BD284638BD81
:103FA8005932000851320008F1310008C7320008C0
:103FB800D40C00201C1900202DE9F04104460028EB
:103FC80000F0B380078B02460025A8E0136A1E7C28
:103FD800042E00F08780012E23D1586803888B4275
:103FE80040F09B8005F1080712F092F954F8270079
:103FF8004FF00008C0F8048012F08AF9228B531E93
:104008009D4208D00732238354F8221044F8271021
:1040180044F8228002E044F8278025833046BDE832
:10402800F081052E5ED0032E5CD0022E13D15B6882
:10403800186803888B4270D14388013B9BB2438048
:104048000BB912F065F905F1080654F826305868DE
:1040580012F05EF94EE0072E21D15E68338A8B425A
:104068005BD1002706E0BB1D013756F8230012F08C
:104078004FF9FFB2B38ABB42F5D80027B78205F1E2
:10408800080654F82630586812F042F954F8260009
:1040980033E044F8267025830120BDE8F081062E20
:1040A8001ED1586803888B4237D105F1080612F0F3
:1040B8002FF954F826000027476012F029F9228BBF
:1040C800531E9D4209D00833013A54F82310228325
:1040D80044F8261044F82370DEE744F826701AE006
:1040E800082E1AD1586803888B4216D112F010F99D
:1040F80005F1080654F826000027476012F008F971
:10410800228B531E9D42C4D0073254F8221044F823
:10411800261044F822702383BEE701350432BD42DD
:10412800FFF454AF0020BDE8F081BDE8F08170B520
:10413800044600282AD0068B751E083600EB860632
:104148001EE056F8043D1A7C042A13D0012A11D027
:10415800052A0FD0032A0DD0022A02D15B681B68FA
:1041680009E0072A02D15B68198A05E0062A01D00E
:10417800082A04D15B6819882046FFF71DFF013D16
:10418800681CDED100232383012070BD70BDF0B50B
:1041980028B30023068B1A461EE0046A257C072DE7
:1041A80018D16468258A8D4214D1A78A002504EBAA
:1041B80083040DE004EB050C0435DCF818C09CF80A
:1041C80018C0BCF1010F03F1010301D1D8B2F0BD51
:1041D800BB42EFD301320430B242DED30020F0BD3F
:1041E80070B508B3048B00231BE0026A157C072D09
:1041F80015D15268158A8D4211D10023958A11462E
:104208001C46012007E013B99669307601E08E69F3
:10421800347601330431AB42F5D3012070BD01334C
:104228000430A342E1D3002070BD2DE9F04128B34A
:104238000023078B1A461EE0046A257C072D18D137
:104248006468258A8D4214D1B4F814C0002504EBA3
:1042580083040CE066190435B66996F81880B8F13D
:10426800010F03D106F10800BDE8F0810133634571
:10427800F0D301320430BA42DED30020BDE8F08129
:104288002DE9F04700282FD00023B0F818C01D46AC
:1042980027E0046A267C072E21D16468268A8E428C
:1042A8001DD1B4F81480002604EB830915E009EB4E
:1042B8000604A7693C7E012C0DD192F800A0BAF142
:1042C800000F08D007F1080011461022FEF7E0FFA2
:1042D8002046BDE8F087013304364345E7D301356E
:1042E80004306545D5D30020BDE8F087F0B5B0B1FE
:1042F800068B002510E0046A277C062F0AD1646823
:1043080027888F4206D123819DF814306260A372FA
:104318000120F0BD01350430B542ECD30020F0BDDA
:1043280010B500210446FEF793FF20460121BDE8A1
:104338001040FEF78DBF38B598B1048B02460023B4
:104348000CE0106A058804328D4206D100F108029B
:10435800436906CA9847012038BD0133A342F0D308
:10436800002038BD10B50C460021FEF771FF20462D
:104378000121BDE81040FEF76BBF13B502AC04E99C
:104388000C00BDF80230834206D8BDF800308342E5
:1043980034BF0020012000E00020BDF806308B4229
:1043A80006D8BDF804308B4234BF0021012100E05B
:1043B8000021002818BF0846C0B21CBD38B5114BF3
:1043C800114A1988002319E052F8045FA87D0128D2
:1043D80012D100240CE004F1080355F82300037CF3
:1043E800082B03D1436800211B6998470134A4B204
:1043F8002B8BA342EFD838BD01339BB28B42E3D15C
:1044080038BD00BFD40C002018190020704770B5C3
:10441800094CA5787DB9094B1E78012E0BD163682C
:10442800013363606268064B9A4204D9284601F05A
:10443800C5FCA670656070BDD40C00208401002006
:1044480040420F00054A9060134602E0996801391E
:10445800996091680029F9D1704700BFD40C0020F9
:10446800F0B585B001F058FF002800F0498100251B
:1044780002A80DF10A01ADF80850ADF80A5001F094
:104488004DFF03A80DF10E01ADF80C50ADF80E501C
:1044980001F090FFBDF80C10BDF808200091BDF8A0
:1044A8000E10BDF80A3001912C46964D9649082009
:1044B8000AF0D6FCA878012803D101F07FFCAC7083
:1044C80019E1924B5B78012B40F01581AB78002BFA
:1044D80040F011816B6029888D4A09E152F8046F18
:1044E800B07D012840F002810025FAE005F10803BB
:1044F800BDF8080056F82340BDF80A1004F1080377
:104508000CCBFFF73AFF002800F0E980237C013B41
:10451800062B00F29F80DFE803F00429159D1F9DFC
:104528004C006668012304F10805337795E8060016
:10453800636920469847002333772046636995E8E6
:10454800060086E0636893F8252012F1FF3218BF51
:10455800012283F8252077E0636893F82C2012F174
:10456800FF3218BF012283F82C206DE06268137EA9
:104578001568002B6ED16E882F462946184606E02E
:1045880051F804EFDEF804E001338EF81800B34266
:10459800F6D301231376002607E057F8040F00F13D
:1045A8000802436906CA984701366B889E42F4D3CD
:1045B80050E0656820892E68A37B227B0096A0F1D5
:1045C800160189B2FFF721F81420FFF73BFF2B7A79
:1045D800C3B9AF8A29461A461E4609E0886990F889
:1045E80018E00676BEF1010F08BF13460431013208
:1045F800BA42F3D301220BB9AB6924E0053355F86D
:10460800233020E06368DB685A680023908A1546E7
:1046180019461F4609E0AE6996F818E03776BEF1EC
:10462800010F08BF0B46043501318142F3D3411E07
:104638008B4203D1053052F8203003E004D207330F
:1046480052F8233001221A7604F1080206CA636977
:1046580020469847237C013B072B4CD8DFE803F022
:104668000410074B0A0D123A63681B6A34E063684A
:104678009B6A2DE063681B6B2AE063681B6927E06F
:10468800636824E063681A7A7AB9988A1946013807
:1046980000E00132824204D28C69247E0431002C6D
:1046A800F7D0063253F8223011E0DB685A68908A56
:1046B80011460138002300E00133834204D28C699B
:1046C800247E0431002CF7D0063352F82330DB69FE
:1046D800984710E06368DB68204698470BE001358F
:1046E800ADB2338BAB423FF601AF04E001339BB26E
:1046F8008B427FF4F3AE01F055FE0F20FFF7A2FEC8
:1047080005B0F0BDD40C002079A60508840100206E
:1047180018190020034B9A6812B19A68013A9A60F6
:10472800704700BFD40C00202DE9F3470120DFF8C3
:10473800D080DFF8D09001460BF02CFF0124002533
:104748004FF4807602274046694600968DF804703B
:104758008DF805408DF806508DF807400BF072FB78
:104768004046082122460BF0EDFB244BDFF89880E9
:104778001A6844F2A243B2FBF3FA0AF1FF3A204660
:1047880021461FFA8AFA0BF035FFC8F804A04846FC
:104798004146A8F80050A8F80250A8F8085088F830
:1047A8000A500CF0C3FA7023A8F80C300423A8F8B8
:1047B80010300AF1FF3A6323642203FB0AF3B3FBC8
:1047C800F2F39BB2C8F8143008F10C014846A8F877
:1047D8000E40A8F81870A8F81A50A8F81C60A8F895
:1047E8001E500CF0C1FB484621460CF034FB4846ED
:1047F80021460CF03AFEBDE8FC8700BFD00100203E
:104808000000024000000140E40C002083B50E4681
:104818000746154910201C4615460AF021FB1020B2
:1048280012490AF01DFB102011490AF019FB10204B
:104838000E490AF015FB002310200E4901930AF0D7
:104848000FFB334610200C493A460AF009FB1020AA
:104858000A492A460AF004FB1020094922460AF0B0
:10486800FFFA019B0133E7E7B3A60508B8A60508D8
:10487800D8A60508E8A60508F8A605080DA705089E
:104888001EA7050808B5164B1A6A01321A621A6A79
:10489800012A1A4603D0134840F21D210FE058623E
:1048A800194602E04B6A013B4B62506A0C4B0028E8
:1048B800F8D11A6A012A06D00A484FF40A710A4A3E
:1048C8000A4BFFF7A3FF1A6A013A1A621B6A2BB157
:1048D8000448054A064B40F22A21F2E708BD00BF0A
:1048E800E40C00202FA70508D6A2040859A705083C
:1048F8006AA7050810B5084C0221002220460BF0D3
:1049080016FB44F6FF70FFF7BDFF20460221012287
:10491800BDE810400BF00BBB000402400C4B0D49E6
:104928001A6844F2A2436428B2FBF3F3D4BF20EA26
:10493800E0706420013B9BB24B60013B584364220A
:10494800B0FBF2F080B2486103480C310CF08FBA2A
:10495800D0010020E40C00200000014010B5134BEA
:1049680093F828202AB11248124A134B4FF4427187
:104978000EE0012283F8282066234FF0C042013B55
:10498800DBB2108033B90A480A4A0C4B40F21231A4
:10499800FFF73CFF1488A4B28442F0D1084B198079
:1049A800024B002283F8282010BD00BFE40C002031
:1049B8002FA70508E0A204087BA7050851A605084B
:1049C8000000026010B5FFF7AFFE6420FFF7A6FFF6
:1049D80021210720FFF7C2FF3220FFF753FF0121F3
:1049E8000020FFF7BBFF3220FFF74CFF23210720F1
:1049F800FFF7B4FF3220FFF745FF00211020FFF733
:104A0800ADFF41F28830FFF73DFF33210720FFF764
:104A1800A5FF3220FFF736FF112046F63001FFF7D9
:104A28009DFF3220FFF72EFF4FF4C0610220FFF7F1
:104A380095FF3220FFF726FF122046F6EB41FFF7DD
:104A48008DFF3220FFF71EFF03204AF6A401FFF76F
:104A580085FF3220FFF716FF00210C20FFF77EFFAD
:104A68003220FFF70FFF0D2040F60C01FFF776FF0D
:104A78003220FFF707FF0E204FF42C51FFF76EFF8F
:104A88003220FFF7FFFEB0211E20FFF767FF32201C
:104A9800FFF7F8FE012042F63F31FFF75FFF3220B3
:104AA800FFF7F0FE05200021FFF758FF3220FFF73F
:104AB800E9FE00210620FFF751FF3220FFF7E2FE52
:104AC80016204EF61C71FFF749FF3220FFF7DAFE79
:104AD800172040F20311FFF741FF3220FFF7D2FE03
:104AE80000210B20FFF73AFF3220FFF7CBFE002111
:104AF8000F20FFF733FF3220FFF7C4FE41200021CB
:104B0800FFF72CFF3220FFF7BDFE42200021FFF700
:104B180025FF3220FFF7B6FE00214820FFF71EFFD1
:104B280040F23F143220FFF7ADFE21464920FFF73F
:104B380015FF3220FFF7A6FE00214A20FFF70EFFDF
:104B48003220FFF79FFE00214B20FFF707FF32209E
:104B5800FFF798FE44204FF46F41FFF7FFFE322025
:104B6800FFF790FE00214520FFF7F8FE3220FFF7FF
:104B780089FE21464620FFF7F1FE3220FFF782FE2C
:104B8800302040F20771FFF7E9FE3220FFF77AFE86
:104B980031204FF40171FFF7E1FE3220FFF772FE7A
:104BA80032204FF40171FFF7D9FE40F2025432204F
:104BB800FFF768FE21463320FFF7D0FE3220FFF7CB
:104BC80061FE342040F20751FFF7C8FE3220FFF79C
:104BD80059FE35204FF40171FFF7C0FE3220FFF770
:104BE80051FE36204FF40171FFF7B8FE3220FFF76F
:104BF80049FE21463720FFF7B1FEA4F500743220A4
:104C0800FFF740FE21463A20FFF7A8FE3220FFF7C3
:104C180039FE2F2041F2BE21FFF7A0FE3220FFF718
:104C280031FE21463B20FFF799FE3220FFF72AFE8E
:104C380000212320FFF792FE3220FFF723FE0021F8
:104C48002420FFF78BFE3220FFF71CFE25204FF4AF
:104C58000041FFF783FE3220FFF714FE00214F20AA
:104C6800FFF77CFE3220FFF70DFE4E200021FFF7F4
:104C780075FE3220BDE8104004E608B5124B93F8E3
:104C880029202AB11148124A124B40F222310FE072
:104C9800012283F82920222166234FF0C042013BDC
:104CA800DBB2118033B90948094A0B4B40F23B315A
:104CB800FFF7ACFD108880B22228F0D1024B002209
:104CC80083F8292008BD00BFE40C00202FA70508A1
:104CD800EDA204087BA7050851A6050810B51E4BD0
:104CE800032826D8DFE800F0021A080E1C8841F2D3
:104CF800280246F628000AE01C8841F2080246F617
:104D0800080004E01C8841F2300246F6300049F2FF
:104D180041318C4214BF014611460BE0188846F613
:104D2800200249F24131884214BF11464FF48151A3
:104D380000E000211B8848F68912934205D049F209
:104D48002032934204D1032000E01120FFF706FE31
:104D5800BDE8104091E700BF86010020014B188094
:104D68000A208FE5000002604FF0C043188003F569
:104D780000331A881A88188880B270474FF0C043E9
:104D880022221A8003F5003382B01A8892B2ADF855
:104D980006201B889BB2ADF80630BDF8060080B22D
:104DA80002B07047072040F27311D7E507200021B1
:104DB800D4E582B0044BADF80600BDF8062092B2E7
:104DC8005A8502B0704700BFE40C002082B0044B43
:104DD800ADF80600BDF8062092B25A8002B07047BE
:104DE80086010020014B80B21880704700000260E5
:104DF8004FF0C04380B218807047024B80B21880D1
:104E0800704700BF000002604FF0C04380B21880B6
:104E18007047024B80B21880704700BF00000260E4
:104E280082B0044B0190019ADA62DA6A002AFCD156
:104E380002B07047E40C002070B54FF0C0452A243A
:104E48002C800A4C060AC0B226802080100AD2B2F2
:104E5800208022802B222A800A0A2280C9B21A0ABC
:104E6800DBB221802280238070BD00BF0000026079
:104E780010B50B4614460246FFF7DEFF4FF0C0435D
:104E88002C22A0B21A80BDE8104067E7114B1B889E
:104E980048F68912934210B504460BD049F22032E5
:104EA800934212D1C1F1EF01202089B2FFF756FDDC
:104EB800212006E0C1F1EF014E2089B2FFF74EFD37
:104EC8004F202146BDE8104048E502460B46BDE8A4
:104ED8001040B1E78601002008B5FFF7D7FF0F4B58
:104EE8001B78012B4FF0C0420D4B0FD12E211180A2
:104EF8001A881A881B8892B202F0FC0002F47842E1
:104F080042EAC000C3F3C423184308BD222111801C
:104F18001A881A88188880B208BD00BFEC190020CA
:104F28000000026070B5074D064601242146304650
:104F3800FFF7D2FF0134A4B2C82C25F8020FF5D12F
:104F480070BD00BF0638002010B5084B1B78012B38
:104F5800144602D1BDE810408AE7FFF797FFFFF734
:104F68008CFE2046BDE81040F8E600BFEC19002092
:104F780070B5074D064601242146013435F8022F45
:104F88003046A4B2FFF7E0FFC82CF5D170BD00BFD2
:104F98000638002070B505460E46FFF7C3FF01240A
:104FA8002146013428463246A4B2FFF7CDFFC82C6B
:104FB800F6D170BD2DE9F04104460D461646BDF800
:104FC8001880032B39D8DFE803F00B351927381977
:104FD80080B2294642460137FFF7B6FFBFB200E06C
:104FE8000027B742F3D1BDE8F081E01B80B2294623
:104FF80042460137FFF7A8FFBFB200E00027B742DB
:10500800F3D1BDE8F081E91B89B220464246013759
:10501800FFF79AFFBFB200E00027B742F3D1BDE81F
:10502800F081791989B2204642460137FFF78CFF93
:10503800BFB200E00027B742F3D1BDE8F08170B5F8
:10504800194B1A4A598E92F9004064180025A4B2E7
:105058008AB0AC4208BF0124C62C28BFC6241570EC
:105068000F264FF6FF721E865C865A8519202B463E
:10507800009221460A22FFF79DFF21463046FFF79E
:105088002BFF224603460A4902A811F0ABFC02AAEC
:1050980006A8084911F0A6FC3220D22106AA2B4600
:1050A80000F002FF0AB070BDE40C0020591A00207D
:1050B80090A7050898A705082DE9F341BDF82050E9
:1050C8000C4690461F461A46002306460095FFF7F1
:1050D80071FF611E414430463A46002389B200956B
:1050E800FFF768FF30462146424601230095013EFE
:1050F800FFF760FFBF19B8B2214642460123089561
:1051080002B0BDE8F04155E72DE9F0410D46C5F183
:10511800F008411E5E18C2EB0802C5F1EF039BB20E
:1051280092B2B6B29A422CBF904698469A4234BF81
:1051380011461946864234BF3746074640F23F13A8
:10514800864238BF06469E4228BF1E46174B1B881C
:1051580048F68912B8F1EF0F28BF4FF0EF089342D5
:10516800044610D049F2203293421AD15020FFF75A
:10517800F5FB51204146FFF7F1FB52203946FFF776
:10518800EDFB53200AE041EA082189B24420FFF7E9
:10519800E5FB45203946FFF7E1FB46203146FFF79E
:1051A800DDFB20462946BDE8F0416FE68601002078
:1051B80000200146F0224FF4A073A5E770B580B235
:1051C80002FB03F489B292B29BB2FFF79DFF002065
:1051D800FFF784FD0025064E04E0708D80B2FFF7CE
:1051E800BDFD0135A542F8DBBDE87040E0E700BF32
:1051F800E40C002070B54FF0C0452A242C80094CDF
:10520800060A26802080080A208021802B212980F8
:10521800110A218022801A0A228023802C232B80C5
:1052280070BD00BF0000026070B5114B1B78012BE8
:10523800044607D1002040F23F110246EF23FFF752
:10524800D9FF04E0FFF7B4FF0020FFF747FDF02582
:1052580009E0013E2046B6B2FFF780FD002EF8D1E6
:10526800013DADB215B14FF4A076F2E770BD00BFB5
:10527800EC1900202DE9F04F1C463E4B87B01B78F7
:10528800039183469DF8441010980591012B039BC8
:10529800049092461FFA8BF09AB208D1411E531E11
:1052A8000919534489B29BB2FFF7A4FF09E01FFA1A
:1052B8008AF51146A3B22A46FFF726FF0020FFF71A
:1052C8000DFD0027DDF80C803E4640F23F1CA1464C
:1052D80039E0BBF1000F2EDB65452CDC0398002874
:1052E80029DBB8F1EF0F26DC220702D1002CC8BF5A
:1052F800013621492140002903DA013961F00F0103
:105308000131059A0AB1C1F10F01049830F816204D
:1053180003FA01F10A4012B26AB118494A8D0293A0
:1053280092B2A8B21FFA88F1CDF804C0FFF70CFEBC
:10533800DDF804C0029B013401354C45C9DB013658
:10534800013708F10108574503DA5D4600240123B7
:10535800F3E7084B1B78012B08D1002040F23F11DE
:105368000246EF2307B0BDE8F04F43E707B0BDE8BA
:10537800F04F1DE7EC1900200F000080E40C00201E
:105388002DE9F74F1F463B4BDDF830801B7816465A
:105398009DF83420012B044601920D4680B28AB252
:1053A80008D1411E531EC9199B1989B29BB2FFF738
:1053B80021FF09E01FFA86FE1146BBB27246FFF7CD
:1053C800A3FE0020FFF78AFC4FF0000BDA463DE011
:1053D800002C30DB09EB040340F23F1293422ADC35
:1053E800002D28DB0BEB0503EF2B24DC19F00F0F46
:1053F80004D1B9F1000FC8BF0AF1010A1E4B09EA2E
:105408000303002B03DA013B63F00F030133019A16
:105418000AB1C3F10F03012202FA03F338F81A2084
:1054280013401BB213B1154B588D01E0144A508834
:1054380080B2FFF793FC09F1010901E04FF0000980
:10544800B945C5DB0AF1010A0BF1010BB345F5DBE0
:10545800084B1B78012B08D1002040F23F1102466F
:10546800EF2303B0BDE8F04FC4E603B0BDE8F04F4A
:105478009EE600BFEC1900200F000080E40C00201D
:10548800860100202DE9F0411C4F069C3F789DF8CD
:105498001C60012F02FB03F580B28FB209D1411EB7
:1054A800CB1899B27B1E9A1893B23A46FFF7A2FE20
:1054B80007E092B29BB23946FFF726FE0020FFF7BD
:1054C8000DFC002709E034F8020B1EB1030A43EA79
:1054D800002080B2FFF742FC0137AF42F3DB074BF5
:1054E8001B78012B07D1002040F23F110246EF2321
:1054F800BDE8F0417EE6BDE8F04159E6EC19002030
:105508002DE9F0431F2093B0FFF78EFE4FF478404B
:10551800FFF78AFE4FF6E0754FF4FC60FFF784FE54
:105528002846FFF781FE0020514CFFF77DFE002042
:105538004FF6FF79014664220346A4F82A90CDF875
:105548000090FFF737FD00200A2164220346CDF8BA
:105558000090FFF72FFD00200146642201234FF43D
:10556800784765850095FFF725FD7720EF21C8224C
:1055780000234FF4FC6667850097FFF71BFDBD21EC
:105588003222012340F23F1066850096FFF712FD94
:10559800A02032220023782167850097FFF70AFDB3
:1055A800A0207821322201234FF01F08668500963B
:1055B800FFF700FDA020782132220223A4F82A80D8
:1055C800CDF80080FFF7F6FCA020782132220323D3
:1055D80065850095FFF7EEFC264B2749A3F8028066
:1055E80002AD3C22284611F03BF9EB20C3210522ED
:1055F800302300950025A4F82A900195FFF7C0FEF6
:1056080032210A2096220B4667850097FFF754FD42
:1056180032213C2096220B4666850096FFF74CFD0A
:1056280032210B4696226E20A4F82A80CDF80080FD
:10563800FFF742FDFFF7BAFBFFF7B4FB3220FFF795
:105648006DF92846FFF76AF96420FFF767F90B4BF5
:1056580003F110028DE8240028465A681B68294681
:10566800FFF710FF1195119B01331193FBE700BF62
:10567800E40C00208601002002A30408C0C701082A
:105688002DE9F14FFFF750F84FF0C0456420FFF7C0
:1056980045F90127FFF72EF94FF028096D48FFF764
:1056A800F1F82F800520A5F8009003F0CBF9CF235F
:1056B8002B80694B002683221E801A8030221A8094
:1056C800ED222A804FF064080322A3F800801A8094
:1056D80012221A8081221A80E8222A8085221A80C2
:1056E80079221F801A80CB222A8039221A804FF013
:1056F800340C02242C21F72219801E80A3F800C044
:105708001C802A8020221A80EA222A80C0221E8039
:10571800C1211E802A8026221A8029801121198001
:10572800C5212980352119803E211980C72129806A
:10573800BE211980362129803A205521A3F80090EE
:1057480028801980B12129804FF0100BF2211E808A
:10575800A3F800B02980082119802A80E0221F8040
:105768004FF01F092A801A22A3F800904FF0180A58
:105778001A800F210A22A3F800A01A801980062196
:105788001980452119808721198032211980072124
:105798001A804FF0E10E19801C80052419801C80A6
:1057A8001E80A5F800E04FF0250E1E80A3F800E04B
:1057B8004FF0270EA3F800E01C80A3F800B04FF0CC
:1057C800090BA3F800B04FF0780B1880A3F800B0CD
:1057D8004FF04D0BA3F800B01C800D24A3F800A0D7
:1057E8001C8038241C8018802A20A3F80090EF24FD
:1057F80028802B201E801E801E801C8028803F2031
:105808001E801E801F801880B720A5F800C0288041
:105818001980B62129801A8082221A801122A3F8C1
:1058280000E040461E8029272A8003F00BF94046F5
:105838002F8003F007F90948FFF724F82C232F805D
:1058480030462B8040F23F113246234601B0BDE876
:10585800F04FCFE4400D03000000026040420F000B
:105868002DE9F041022098B0012100240AF092FEAF
:10587800012502268048169616A98DF85D408DF8F8
:105888005E408DF85F408DF85C500AF0DBFA182016
:1058980029460AF07FFE284629460AF093FE21464B
:1058A8000C2276480AF04EFB0C22744829460AF06E
:1058B80049FB04210C2271480AF044FB05210C2203
:1058C8006E480AF03FFB07210C226C480AF03AFBAD
:1058D80008210C2269480AF035FB09210C22674887
:1058E8000AF030FB0A2165480C220AF02BFB0B2139
:1058F80062480C220AF026FB0E210C225F480AF0AF
:1059080021FB0F210C225D480AF01CFB07210C2209
:105918005B480AF017FB08210C2259480AF012FBD1
:1059280009210C2256480AF00DFB0A210C22544882
:105938000AF008FB0B210C2251480AF003FB0C214A
:105948000A464F480AF0FEFA0D210C224C480AF08C
:10595800F9FA0E210C224A480AF0F4FA0C224848B7
:105968000F210AF0EFFA4CF6B3734448169316A9C0
:105978008DF85C608DF85E408DF85F408DF85D5065
:105988000AF060FA16A94FF680733D4816938DF811
:105998005C608DF85E408DF85F408DF85D500AF0D0
:1059A80051FA40F6B830FEF76DFFFEF7A3FF40F658
:1059B800B830FEF767FF0F2311934FF48053102779
:1059C8000DF13C08099368464FF400231094129493
:1059D80014941594009401940294039704940694E3
:1059E800079408940A9405940B940C93CDF834808A
:1059F8000F95139509F09FFF0523684611930F969D
:105A08001094129414941594CDF83880139509F0D5
:105A180092FF294620460AF00EF840F6B830FEF705
:105A280031FF2046FFF7A0F904461649164E3846BE
:105A3800224609F015FA41F289239C4248F6891852
:105A4800124F01D044450ED1FEF7BCFF00233B7036
:105A5800A6F8008010200E4948F6891241F28923E1
:105A680009F0FEF905E0FFF70BFE49F241333D70FE
:105A7800338018B0BDE8F08100040240000C0240F9
:105A8800001002409DA7050886010020EC1900209F
:105A9800B4A705084FF0C04336221A8003F5003337
:105AA800012814BF682048201880704770B5244B1F
:105AB80001228CB01A7000240AE0A9B21F223046D5
:105AC8000135FFF741FA642DF7D10134642C02D077
:105AD8000025A6B2F1E73220014602460346FFF749
:105AE800ABF94FF0C0432E221A8003F50033002093
:105AF8001A881C881D88A4B200F09CF8ADB2002357
:105B0800224600930F492B4603A810F06BFF002391
:105B18000A20C82103AA00F0C7F904F0FC0204F423
:105B2800784444EAC20242EAD522074903A810F0A1
:105B380059FF0A20DC2103AA002300F0B5F9FEE78B
:105B4800EC190020F3A705080BA805082DE9F04F6C
:105B580040F23F19484534BF04464C46EF2B34BF4A
:105B680098464FF0EF084A4538BF9146EF2934BFB1
:105B78000D46EF25C4EB090AC5EB080785B0BAF155
:105B8800000FB8BFCAF1000A002FB8BF7F424FF616
:105B9800FF734C452CBF1A4601221FFA8AFA454565
:105BA80038BF0123BFB202930FFA8AF63BB29E4276
:105BB800BDF838B0019202DDC6F34F0607E00226B1
:105BC80093FBF6F67642B6B201E01E4603E00FFA02
:105BD8008AF35B420393144A1378022B2046294622
:105BE8005A4602D1FDF7FDFC01E0FFF7ADF94C453F
:105BF80001D1454514D0039A33B2934205DD019A89
:105C0800F31BA4189BB2A4B200E0334636B23AB2F2
:105C18009642DADA029A5344AD189BB2ADB2D4E791
:105C280005B0BDE8F08F00BF242C00200048704765
:105C3800F419002082B0064BADF80600BDF8062026
:105C480092B21A80188880B202B0FFF7B2B800BFCB
:105C5800F0190020014B188880B27047F019002015
:105C680082B0064BADF80600BDF8062092B21A8045
:105C7800188880B202B0FFF7A9B800BFF219002057
:105C8800014B188880B27047F2190020FFF7CCBA90
:105C9800FFF73ABA10B5BDF808400294BDE81040C5
:105CA800FFF788B910B5BDF808400294BDE8104068
:105CB800FFF702BAFFF782BA2DE9F04F4FEA420820
:105CC80000253D4C85B082468B46C8F1030817462F
:105CD8002E461FFA87F909EB0B0C228805EB0A03FD
:105CE8001FFA8CFC9BB26146184692B2CDF804C0EC
:105CF8000293FFF729F9C9EB0B0292B20392029BB8
:105D080022880399184692B2FFF71EF9DDF804C0FD
:105D18002288C5EB0A039BB26146184692B20293E9
:105D2800FFF712F9029B22880399184692B2FFF7EF
:105D38000BF905EB0B0292B2039209EB0A032288D6
:105D480003999BB2184692B20293FFF7FDF8029BA3
:105D58002288C5EB0B0C1FFA8CFC1846614692B2E0
:105D6800CDF804C0C9EB0A09FFF7EEF822880399B9
:105D78001FFA89F992B24846FFF7E6F82288DDF85B
:105D880004C092B248466146FFF7DEF8B8F1000F4A
:105D980004DA08EB860808F1060805E0F31B08F1A9
:105DA8000A0808EB8308013F01360135BE42ADB24F
:105DB8008FD905B0BDE8F08FF019002008B9FEF7BB
:105DC800F5BF012801D1FEF7EDBF704770470020ED
:105DD8000146F0224FF4A073FFF796B9704708B553
:105DE80005280CD8DFE800F0121403050709094854
:105DF80008BD094808BD094808BD094808BD094843
:105E0800094A0A4B40F24111FEF700FD084808BD57
:105E1800084808BD74010020640100205C010020CE
:105E28005401002016A805083EA3040851A6050839
:105E38007C0100206C01002010B50446FFF7CFFF5D
:105E4800014B18601C7110BD8C010020014B1879A2
:105E5800704700BF8C01002008B5FFF7C0FF80889D
:105E680008BD08B5FFF7BBFFC08808BDF7B51F46DA
:105E78000B4B0C4E1D681446EA882B68203C544393
:105E8800A4B2AE1B03EB440418BF0126AB888DE80F
:105E9800500017B1FFF7EEF901E0FFF771FAFEBD08
:105EA8008C0100207C0100202DE9F0410F46984626
:105EB80015460446084E08E0204643463946FFF793
:105EC800D5FF33689B88E418A4B215F8012B002A83
:105ED800F2D1BDE8F08100BF8C01002010B5044666
:105EE80008462146BDE81040DEE7094B70B5044678
:105EF80018790E461546FFF7B4FFC6F1F001091AE6
:105F080089B220462A460023BDE87040CCE700BF8E
:105F18008C010020704700BF044B1A680AB9044A74
:105F28001A601A681018186010467047180D00207B
:105F3800A43C00204FF0FF30704708B50248034AE0
:105F4800034B3721FEF762FC35A8050854A3040863
:105F580051A605080120704710B504460A480221D9
:105F68000AF09EFD0028F9D0074821460AF061FD95
:105F7800054801210AF094FD0028F9D00248BDE83F
:105F880010400AF053BD00BF0038004010B5194852
:105F980002210AF085FD0028F9D0164800210AF0F0
:105FA80048FD144801210AF07BFD0028F9D011486A
:105FB8000AF03CFD0402A4B2002301E001339BB2C5
:105FC800002BFBD00B4802210AF06AFD0028F9D00B
:105FD800084800210AF02DFD064801210AF060FD5D
:105FE8000028F9D003480AF021FD2043C0F3CB0074
:105FF80010BD00BF003800402DE9F0478AB00AAF55
:106008000A2001210AF0C6FA4FF4604347F8143D0C
:10601800474EDFF824A1012400254FF0020830463E
:1060280039468DF81A508DF818808DF819808DF83A
:106038001B4009F007FF30460D21052209F082FFB9
:1060480030460E21052209F07DFF052230460F213A
:1060580009F078FF21464FF480400AF0BFFA504615
:106068000AF09AFB4FF48273ADF802304FF40073D4
:10607800ADF80A303823ADF80C305046072369468E
:10608800ADF81030ADF80050ADF80450ADF806503A
:10609800ADF80850ADF80E500AF0B0FB5046214656
:1060A8000AF047FCA9468DF81A5030464FF480553F
:1060B800394605958DF818408DF819808DF81B40E4
:1060C80009F0C0FE3046294609F02DFF4025394623
:1060D80018488DF818908DF819808DF81A908DF859
:1060E8001B40059509F0AEFE21464FF480400AF0AA
:1060F80081FA062103200AF00BFD0C2307A88DF86E
:10610800213007958DF820908DF8224009F08EFBFC
:1061180017238DF8243009A80F238DF825308DF822
:1061280026308DF8274002F0ABFE0AB0BDE8F087B4
:1061380000040240000C024000380040014B18786F
:10614800704700BF1C0D0020024B5A889B880280B4
:106158000B8070471C0D0020014B00221A707047FD
:106168001C0D0020F0B593B068460021482210F0BD
:10617800B9FB6D46002464484FF4805109F0D5FE00
:10618800002301E001339BB2002BFBD09020FFF7E6
:10619800E3FE002301E001339BB2002BFBD0FFF7A5
:1061A800F5FE4FF480510746574809F0BCFE00231E
:1061B80001E001339BB2002BFBD053484FF48051D0
:1061C80009F0B3FE002301E001339BB2002BFBD0A2
:1061D800D020FFF7C1FE002301E001339BB2002B62
:1061E800FBD0FFF7D3FE4FF480510646464809F02E
:1061F8009AFE45F8047B01342E6244484021E4B2FB
:1062080009F07FFE10B9092CB5D101E0092C78D12D
:106218009DE80C00D218029B03980699D218049B9B
:10622800C018059BC018079BCB180899032490FB3E
:10623800F4F092FBF4F25B1893FBF4F3151AC11A0D
:106248009C1A002DB8BF6D420029B8BF4942002CE6
:10625800B8BF6442502D03DD502909DD502C50DCB5
:106268008D4205DAAC424FF0020405DB111806E056
:106278008C424FF0020401DAD11800E0C1180A9BE1
:10628800099A0C980F9DD2180B9BD2180D9BC01819
:106298000E9BC018109BEB18119D91FBF4F1032481
:1062A80092FBF4F290FBF4F05B1993FBF4F3161AEB
:1062B800C41A9D1A002EB8BF7642002CB8BF64429B
:1062C800002DB8BF6D42502E89B203DD502C09DD78
:1062D800502D16DCA64205DAB5424FF0020405DB64
:1062E800131806E0A5424FF0020401DAD31800E0C3
:1062F800C318074A93FBF4F39BB2938001235180A0
:10630800137013B0F0BD00BF00040240000C02403F
:106318001C0D002000000000FFF710BFF7B5054670
:106328000C4601A80DF10601FFF70EFF1B4BBDF847
:106338000660BDF8040093E80600724301FB0022E2
:1063480099685218164992FBF1F207EE102AF8EEF6
:10635800C77A40F23F17FCEEE77A17EE902A92B21E
:10636800B2F5207F28BF3A462A801D69DA685B6942
:106378006E4302FB0060C01890FBF1F107EE101AA3
:10638800F8EEC77AFCEEE77A17EE903A9BB2B3F5CF
:10639800F07F28BFEF232380FEBD00BF240D00201F
:1063A80040420F00FFF7D8BE014B187E704700BF70
:1063B800240D0020FFF7C8BE042808B505D90748F2
:1063C800074A084B7D21FEF721FA054B03EB8000B5
:1063D800038B0B80438B138008BD00BF56A80508AC
:1063E8005AA3040874A8050808B5082001F082F922
:1063F80042F69643C31A584240EB030008BD10B555
:106408000A2001F09FF90C4C20600E2001F09AF947
:106418006060122001F096F9A060162001F092F950
:10642800E0601A2001F08EF920611E2001F08AF93F
:1064380001236061237610BD240D002010B5FFF7FD
:10644800DBFD01F035FA044601F03EFA0749034640
:106458002246202008F004FDFFF7C6FF28B101F00E
:1064680041FA10B9BDE81040C9E710BDB0A8050849
:1064780010B5104C0A20216801F04BF961680E2014
:1064880001F047F9A168122001F043F9E1681620EC
:1064980001F03FF921691A2001F03BF961691E20DA
:1064A80001F037F9082042F69641BDE8104001F0A6
:1064B80013B900BF240D00202DE9F04F0346A7B003
:1064C800B0F800C01C898688DF885D89CDF810C0C7
:1064D800B249B0F802C0B3F80C90B3F80E80CDF80A
:1064E80024C00FFA84FB30B201220FFA87FE0BEBAF
:1064F800000C0A7629B20FFA89FACDF888C001EBA8
:106508000E0C0FFA88F2CDF890C00AEB0B0CCDF800
:1065180030C002EB010CCDF858C0B3F810C05B8A4C
:10652800CDF800C00FFA8CFC06910CEB00010A9123
:1065380002930CEB0A011BB2239103EB0E010E919F
:1065480099182591049900FA81F058445044604400
:10655800DDF824C006990EFA8CFEDDF810C01FFA8B
:1065680080FB1CFB0CF08E4416FB0600964414FBC3
:106578000400009A19FB09009E4412FB02001FFA4E
:106588008EFA0BF097FBDDF824C0029ACDE91201D0
:106598001CFB0CF017FB070015FB050018FB080097
:1065A80012FB02000BF086FBDDF824C0029ACDE94D
:1065B800140104991CFB01F317FB063615FB04664E
:1065C800009B18FB096612FB03600BF073FBDDE907
:1065D8001423CDE90001DDE912010BF0E1FB0446CB
:1065E8000D46DDE9000102460B460BF0D9FB0246D9
:1065F8000B46204629460BF01FFACDE918015846EC
:106608000BF068FBCDE91001DDE91023DDE900019D
:106618000BF0C6FBCDE9060150460BF05BFB80464C
:1066280089464246DDE912014B460BF0B9FBDDE92C
:106638001023CDE91C01DDE914010BF0B1FB0022A8
:1066480006460F46564BDDE918010BF0A9FB4246FA
:1066580004460D464B46DDE906010BF0A1FB024658
:106668000B460BF0EBF902460B46204629460BF089
:10667800E5F9424604460D464B46DDE91C010BF0A0
:106688008FFB02460B46204629460BF0D5F9DDE97B
:10669800102304460D46304639460BF081FB02466E
:1066A8000B46204629460BF0C7F9DDF828C0CDE98E
:1066B80002014FEA8C10DDF830C000EB0C20DDF849
:1066C80010C0A0241CFB04000BF0F4FADDF838C05D
:1066D800CDE90A014FEA8C10DDF858C000EB0C2018
:1066E800DDF824C01CFB04000BF0E4FACDE90C0132
:1066F80050460BF0DFFADDE91023CDE91601DDE99C
:106708000C010BF04DFB4246CDE91E014B46DDE97D
:106718000A010BF045FB4246CDE920014B46DDE975
:1067280000010BF03DFB32463B460BF085F9CDE905
:106738000E0158460BF0BEFADDE91C23CDE91A011B
:10674800DDE906010BF078F9DDF88CC0C024CDE94D
:10675800060104FB0CF0DDF888C0302505FB0C00B1
:10676800DDF810C078261CFB06000BF0A3FADDF854
:1067780094C0824604FB0CF0DDF890C005FB0C00C9
:10678800DDF824C01CFB06008B460BF093FADDE90C
:10679800102306460F460BF003FB03E0240D0020F0
:1067A800000014404246CDE904014B465046594684
:1067B8000BF0F6FADDE9142380468946DDE90A0183
:1067C8000BF0EEFADDE9002304460D46DDE90C0185
:1067D8000BF0E6FA02460B46204629460BF02CF948
:1067E8000022A14B0BF0DCFADDE9202304460D461C
:1067F800DDE91E010BF020F902460B46DDE9160122
:106808000BF0CEFA02460B46204629460BF016F945
:10681800002204460D46954BDDE90E010BF0C0FA47
:1068280002460B46204629460BF008F9DDE902230B
:106838000BF0E0FB88A3D3E900230BF0B1FA0BF0CF
:1068480049FD8B490860DDE91223DDE90C010BF0F5
:10685800A7FADDE9002304460D46DDE90A010BF03D
:106868009FFA02460B46204629460BF0E5F800221F
:106878007D4B0BF095FADDE91E2304460D46DDE954
:1068880020010BF0D9F802460B46DDE91A010BF09E
:1068980087FA02460B46204629460BF0CFF800221D
:1068A80004460D46714BDDE906010BF079FA024604
:1068B8000B46204629460BF0C1F8DDE902230BF010
:1068C80099FB65A3D3E900230BF06AFA0BF002FDEC
:1068D800674A5060DDE90E23DDE90A010BF060FA32
:1068E800DDE9062304460D46DDE90C010BF058FAF4
:1068F80002460B46204629460BF0A0F80022044623
:106908000D465A4BDDE918010BF04AFA02460B46D0
:10691800204629460BF092F8DDE902230BF06AFBCA
:106928004DA3D3E900230BF03BFA0BF0D3FC504BFB
:1069380059469860DDE9142350460BF031FADDE939
:10694800002304460D46304639460BF029FA024624
:106958000B46204629460BF06FF80022424B0BF0FD
:106968001FFA424604460D464B46DDE904010BF08A
:1069780063F802460B46DDE916010BF011FA0246F0
:106988000B46204629460BF059F835A3D3E90023D6
:1069980004460D46DDE90E010BF002FA02460B46ED
:1069A800204629460BF04AF8DDE902230BF022FBCA
:1069B80029A3D3E900230BF0F3F90BF08BFCDFF8E4
:1069C800B0C0DDE91223CCF80C00394630460BF094
:1069D800E7F9DDE9002304460D46504659460BF019
:1069E800DFF902460B46204629460BF025F800221F
:1069F8001D4B0BF0D5F9DDE9042304460D4640464E
:106A080049460BF019F802460B46DDE91A010BF06E
:106A1800C7F902460B46204629460BF00FF810A38B
:106A2800D3E9002304460D46DDE906010BF0B8F969
:106A380002460B46204629460BF000F8DDE9022302
:106A48000BF0D8FA04A3D3E900230BF0A9F90BF053
:106A580041FC074908610DE00000000080842E41D8
:106A68000000000000C0824000001440000089407F
:106A7800240D0020DDE90E23504659460BF090F90D
:106A8800DDE9062304460D46304639460BF088F901
:106A980002460B46204629460AF0D0FF11A3D3E947
:106AA800002304460D46DDE918010BF079F902468A
:106AB8000B46204629460AF0C1FFDDE902230BF008
:106AC80099FA0AA3D3E900230BF06AF90BF002FC48
:106AD800034A506127B0BDE8F04FC9E4AFF3008026
:106AE800240D00200000000000C0824000000000CB
:106AF80080842E41AFF30080064A074B1A60074A8C
:106B0800074B1A60074B42F210721A60064B642258
:106B18001A60704740420F001826002080C3C90140
:106B2800302C00200C2C0020C8250020012810B58E
:106B380002D002283AD123E01D4B1E4C1B78012BB2
:106B48001D4B0ED11968C82000F0E3FD2168CC2048
:106B580000F0DFFD194BD020196800F0DAFDD420D1
:106B68001EE01968D82000F0D4FD2168DC2000F070
:106B7800D0FD124BE020196800F0CBFDE4200FE0B7
:106B88000D4BE820196800F0C4FD0A4BEC20196889
:106B980000F0BFFD094BF020196800F0BAFDF420A1
:106BA800074B1968BDE8104000F0B3BD10BD00BF29
:106BB800F40D0020302C0020182600200C2C00207A
:106BC800C825002010B5224B1B78012B02D0022BC0
:106BD8003DD128E01F4B204C1B78012B0FD1C8203A
:106BE80000F0B0FD2060CC2000F0ACFD1B4B18601D
:106BF800D02000F0A7FD1A4B1860D4200EE0D82052
:106C080000F0A0FD2060DC2000F09CFD134B186014
:106C1800E02000F097FD124B1860E42000F092FD90
:106C2800104B186010BDE82000F08CFD0A4B18606E
:106C3800EC2000F087FD094B1860F02000F082FD81
:106C4800074B1860F42000F07DFD064B186010BD5E
:106C5800B5010020F40D002018260020302C00205B
:106C68000C2C0020C825002008B504F0CFFD10B179
:106C7800BDE80840A6E7BDE808403DE7064B0749E0
:106C88005960C021002219721E211A70D9601A7425
:106C98005A611A76DA617047201A002040787D011F
:106CA80010B50321FF22C02001F0D2FB1F4C102198
:106CB80080222060C02001F0CBFB112180222060BF
:106CC800C02001F0C5FB122180222060C02001F005
:106CD800BFFB132180222060C02001F0B9FB1421E2
:106CE80080222060C02001F0B3FB152180222060A3
:106CF800C02001F0ADFB802220601621C02001F0E9
:106D0800A7FB2060C0201721802201F0A1FB802270
:106D18002060B721C02001F09BFB054B00221A74AC
:106D28005A611A76DA6101221A7010BDF025002026
:106D3800201A002038B5C0200321FF2201F088FB6B
:106D48000B4D00242B19615D5A78C020023401F0E4
:106D58007FFBC82CF6D1B121AC22C02001F078FB12
:106D6800C0200321002201F073FB002038BD00BFC2
:106D780086A304082DE9F34706460F4692461D46AA
:106D88001AB90C1FE401914635E005EE902A06EE8B
:106D9800903AB8EE657AF8EE667AFC01C7EE277A83
:106DA800A4F500749FED5C7A67EE877A17EE900A77
:106DB8000AF0A2FF41EC100B0DF0B2F859EC108B61
:106DC800494640460BF0AEFA24184FEACA100AF0BA
:106DD80071FFCDE9000128460AF06CFF4B46424698
:106DE8000AF0DEFF02460B46DDE900010AF024FE48
:106DF8000BF098FA8146002E14BF4FF022084FF08E
:106E08001A08C5F307224146C02001F021FB08F10A
:106E18000101EAB2C02001F01BFBC4F3014208F1F2
:106E28000201C02001F014FBC4F3072208F103019A
:106E3800C02001F00DFBE2B208F10401C02001F00E
:106E480007FBC9F3034305F4702243EA123208F141
:106E58000501C02001F0FCFA08F10601C9F3072278
:106E6800C02001F0F5FA08F107015FFA89F2C020A5
:106E780001F0EEFAC020B121A02201F0E9FA07EEF4
:106E8800107A264CF8EEC77A0EBBD4ED015A06EEFE
:106E980090AAB8EE657A05EE905AB8EE666AF8EEF2
:106EA800656A0123C6EE266A237477EEA67A67EE32
:106EB800277A17EE900A0AF01FFF41EC100B0DF02D
:106EC8002FF851EC100B0BF02DFA606120E005EE65
:106ED80090AAD4ED016AB8EE656A05EE905AB8EE4C
:106EE800667AF8EE656A0123C6EE266A237677EE9F
:106EF800A67A67EE277A17EE900A0AF0FDFE41ECB3
:106F0800100B0DF00DF851EC100B0BF00BFAE061C3
:106F18000020BDE8FC8700BF00000043201A0020C5
:106F28000022012326E7012838B50D4604D002289F
:106F38000CBF3C242C2400E034242146C02001F05E
:106F480001FB05F0070200F00F0040EA021221469B
:106F5800C020BDE8384001F07BBA2DE9F3470A9C10
:106F68001D4607468A461646524B01E06D086408DE
:106F78009C42FBD82DB906F10076043EF601A946DD
:106F880034E006EE905AB8EE667A06EE904AF8EECD
:106F9800667AF601C7EE277AA6F500769FED467A5F
:106FA80067EE877A17EE900A0AF0A6FE41EC100BFE
:106FB8000CF0B6FF59EC108B494640460BF0B2F97D
:106FC8003618E8010AF076FECDE9000120460AF0FD
:106FD80071FE4B4642460AF0E3FE02460B46DDE9E7
:106FE80000010AF029FD0BF09DF98146022F9BBF95
:106FF800324BDB194FF0000893F8C880C4F307221E
:107008004146C02001F024FA08F10101E2B2C9B2F8
:10701800C02001F01DFA08F10201C9B2C6F301420D
:10702800C02001F015FA08F10301C9B2C6F307221E
:10703800C02001F00DFA08F10401C9B2F2B2C02073
:1070480001F006FA04F47024C9F3034308F10501BA
:1070580043EA1432C9B2C02001F0FAF908F1060176
:10706800C9B2C9F30722C02008F1070801F0F0F9F6
:107078005FFA89F25FFA88F1C02001F0E9F9BAF104
:10708800010F0CBF2F220F220DB942F04002012F31
:1070980006D002D3022F0AD105E0C020102104E057
:1070A800C020112101E0C020122101F0D1F90020F7
:1070B800BDE8FC87FFFF0F000000004386A304081B
:1070C80007B5012300930023FFF747FF0EBD0028F3
:1070D8000CBFFF22002208B5C020032101F0B8F937
:1070E800002008BD08B5C020B121AC2201F0B0F9DC
:1070F800002008BD08B50420012109F04BFA4FF41F
:1071080080700121BDE8084009F074BA07B5022370
:10711800009303238DF804300348002369468DF853
:10712800073008F08FFE0EBD0008024030B5124D42
:107138008BB0002406A8069407940894099408F0D4
:107148004FF800948DF804408DF80540029403949C
:1071580004942846012469468DF8144008F011F873
:1071680028460B212246062308F086F828462146A1
:1071780008F050F80BB030BD0020014010B50021D8
:1071880004460122302001F063F9C0B9012001F062
:1071980059FC002CB8BF4034E4B2102122463020FC
:1071A80001F056F9012001F04DFC30201121224652
:1071B80001F04EF90120BDE8104001F043BC10BDBC
:1071C80010B5002104460122302001F041F9C0B970
:1071D800012001F037FC002CB8BF4034E4B2122182
:1071E8002246302001F034F9012001F02BFC302038
:1071F8001321224601F02CF90120BDE8104001F0CE
:1072080021BC10BD38B5012205460C4630200021AE
:1072180001F01EF9F0B9012001F014FC25EAE5722D
:107228005F2AA8BF5F223B21D2B2302001F010F9BB
:10723800012001F007FC24EAE4725F2AA8BF5F225C
:10724800D2B230203C2101F003F90120BDE83840DA
:1072580001F0F8BB38BD302810B504460ADC10F13F
:107268007F0F02DB002802DB05E06FF07E0404F5E7
:10727800807400E03024002130200A4601F0E8F84C
:10728800A8B90120E4B201F0DDFB412122463020FB
:1072980001F0DEF8012001F0D5FB30204221224622
:1072A80001F0D6F80120BDE8104001F0CBBB10BDBD
:1072B800282810B5044609DC10F1180F02DB002855
:1072C80002DB04E06FF017047F3400E0282400217B
:1072D80030200A4601F0BCF8A8B90120E4B201F058
:1072E800B1FB53212246302001F0B2F8012001F011
:1072F800A9FB30205421224601F0AAF80120BDE85C
:10730800104001F09FBB10BD08B5302000210122BC
:1073180001F09EF860B9012001F094FB3020332180
:10732800402201F095F80120BDE8084001F08ABB31
:1073380008BD10B530200021012201F089F804466B
:1073480060B9012001F07EFB30203321224601F094
:107358007FF80120BDE8104001F074BB10BD10B5E6
:1073680030200021012201F073F80446A0B9012061
:1073780001F068FB34212246302001F069F8012031
:1073880001F060FB30203721224601F061F801202E
:10739800BDE8104001F056BB10BD4020EEE640208D
:1073A8000EE708B500210122302001F051F8012034
:1073B80001F048FB30203421024601F049F8012051
:1073C80001F040FB30203721024601F041F801204E
:1073D800BDE8084001F036BB08B500210122302085
:1073E80001F036F8012001F02DFB302034210C2269
:1073F80001F02EF80120BDE8084001F023BB000091
:107408002DE9F04F984B994A1968994B002914BFF8
:1074180091469946974B2DED048BC3F80090964BF7
:107428000025002287B01A80AA46AB46A8465AE033
:10743800A2004046CDF804C002920AF05DFC07465F
:10744800584601F100460AF057FC02460B463846FA
:1074580031460AF0F1FA39F9243007EE103AF8EE1D
:10746800C77A064617EE900A0F460AF045FC024610
:107478000B46304639460AF0E1FA0AF073FF074630
:1074880050460AF039FC0446284601F100460AF045
:1074980033FCCDE90401DDE90423204631460AF036
:1074A800CBFA029A09EB02030446B3F9023007EE5D
:1074B800103AF8EEC77A0D4617EE900A0AF01CFC4F
:1074C80002460B46204629460AF0B8FA0AF04AFF57
:1074D800DDF804C0684A0CF1010CC3465546A2F811
:1074E80000C08246B846644BB3F800C00FFA8CF46B
:1074F800B32C9DDD58460AF0FFFBCDE9020140465A
:107508000AF0FAFB002206460F465C4BDDE9020151
:107518000AF046FC02460B46304639460AF08EFA17
:107528000022574B0AF066FD0AF01CFF4CA3D3E972
:10753800002309EE900ADDE902010AF031FC00227D
:107548004F4B0AF057FD0AF00DFF09EE100A2846C6
:107558000AF0D2FB044650460D460AF0CDFB002245
:1075680006460F4620462946444B0AF019FC0246B7
:107578000B46304639460AF061FA0022404B0AF0C1
:1075880039FD0AF0EFFE36A3D3E9002308EE900A8E
:10759800294620460AF004FC0022394B0AF02AFD4D
:1075A8000AF0E0FE08EE100A69EE287A58EE297A09
:1075B80017EE900A0AF0A0FB68EE097A48EEA97A5D
:1075C800044617EE900A0D460AF096FB45EC104B60
:1075D80041EC110B0CF0A8FD51EC100B0AF0C2FEA7
:1075E80028EE088A08EEA88A07EE100A254B264CD2
:1075F800F1EE477AC3ED007A18EE100A0AF07CFB28
:1076080041EC100B0CF09EFE29EE099A51EC100B80
:1076180009EEA99A0AF0A6FE206019EE100A0AF0EF
:107628006BFB41EC100B0CF08DFE51EC100B0AF0CB
:1076380099FED4ED007A07EE100A87EE877A134B8D
:107648001860134BFDEEE77A83ED007A114BC3ED1A
:10765800007A07B0BDEC048BBDE8F08FAFF3008073
:10766800912B50E67AB6EB3F481A0020CA22002038
:107678002A1D0020441A0020501A00200000E03F74
:1076880000005940342C00204C2C0020402C0020B5
:107698003C2C00204C1A002010B5084C204608F05D
:1076A8001EF8074B1860FFF7ABFE064B0649012290
:1076B80020461A80BDE8104008F092B810600240D9
:1076C800481A0020400D002020800010014B186847
:1076D800704700BF4C1A002038B505460C460135E6
:1076E800C1F3072101F0BCF9A8B2E1B201F0B8F981
:1076F80000B238BD38B5044600F0ECFF0134054649
:10770800A0B200F0E7FFEDB2C0B240EA052000B237
:1077180038BD37B50B0E8DF804300B0C8DF80530DD
:107728000B0A8DF806308DF80710002400E0284673
:1077380001AB451CE15C013401F092F9042CADB2B7
:10774800F5D13EBD37B5002400E02846451C00F0C1
:10775800C1FF01ABADB2E0540134042CF5D19DF862
:1077680005009DF80430000440EA03609DF80730E6
:1077780018439DF8063040EA03203EBD37B5002384
:107788000193002400E02846451C00F0A3FF01AB4C
:10779800ADB2E0540134042CF5D19DED010A3EBD93
:1077A8007047000038B50446642001F04BF925788D
:1077B8006068AD00EDB2257008F0A9FB237A40FAA5
:1077C80003F000F003000543104B257005F00F058A
:1077D8005A5D6378D218D2B2D3B20132D2B2022A39
:1077E800637001D80022A2705BB2012B03DD012374
:1077F800A3700023637094F90130013303DAFF2387
:10780800A3700023637094F9020038BD52A40408E1
:10781800F7B504200121234F08F0BCFE02AD012179
:107828004FF48040012408F0E5FE00264FF4B073C1
:107838003846694645F8083D8DF804608DF80740DC
:1078480008F000FB1020214608F0A4FE78236946C2
:10785800154800938DF804608DF8074008F0F2FA97
:107868000420214608F096FE21464FF4804008F097
:10787800C1FE1C233846694600938DF804608DF8D4
:10788800074008F0DFFA0220214608F083FEB02303
:1078980006488DF8046069468DF80740009308F0A3
:1078A800D1FAFEBD00080240001002400004024068
:1078B800802108B5034808F024FBD0F1010038BF47
:1078C800002008BD0004024008B54FF48071044848
:1078D80008F017FBD0F1010038BF002008BD00BF39
:1078E8000008024008B5FFF7E3FF08B1FFF7ECFF17
:1078F800C0B208BD70B500283AD01E4B1A7880185F
:107908001D4AC0B292F90020187040B282421B4A48
:1079180002DD11780139197093F9001092F90020ED
:1079280091FBF2F402FB14141549E4B21C700A88A6
:10793800144B1A80144B154A18881080144A92F96F
:10794800000064B2013094FBF0F200FB1240114CCD
:107958002688114C258800FB065008800F490888A6
:107968000F49098802FB00121A800E4B01221A7077
:1079780070BD00BFDE39002009360020E535002043
:10798800143A00202A360020DC390020DC37002099
:10799800163A002038370020783A0020A43A002010
:1079A800BA370020E4350020F0B5264A264C0023DB
:1079B8001370264A25681678254A12680FE0D45CA9
:1079C8002F197F7817F0040F07D0302C02D120230D
:1079D800135431E01B4A137003E00133DBB29E42BB
:1079E800EDDA184B1B788342194B16D9A9B11A68DE
:1079F800164C3121115430210BE01A681518125C0D
:107A08002E2A19D0303AD2B2092A88BF29700130FB
:107A1800C0B222788242F0DA0EE01B681A5C79B1B3
:107A28002E2A0DD05118C9B2392903D82F2998BF49
:107A3800302100E039211954BDE8F040FCF7BEBC04
:107A4800F0BD00BF440D002024030020983B002017
:107A5800003A002010B5642000F0F4FF8C48FFF7CE
:107A6800A1FE8C4B1B7804460C2B00F2E780DFE864
:107A780013F00D000D00E5007400740037008A0053
:107A8800E5008A008D00A700E500CE00FFF71CFF87
:107A980018B10120F9F76CFED0E07F4B18887F4BB6
:107AA8001B88C01A7E4B1B8890FBF3F07D4B1A880D
:107AB8007D4B1B88D31A7D4A128893FBF2F3DBB205
:107AC800C0B2032B00F29F80DFE803F0020406082F
:107AD800774A3FE0774A3DE0774A3BE0774A39E02A
:107AE800FFF7F2FED8B100210A22754810F0CAF853
:107AF800744B002118600A22734810F0C3F8734BC6
:107B080018600420FEF798F996200521704A002392
:107B1800FEF7CAF90020FEF78FF906F011FF5E4B59
:107B280018885E4B1B88C01A5D4B1B8890FBF3F0CE
:107B38005C4B1A885C4B1B88D31A5C4A128893FBEF
:107B4800F2F3DBB2C0B213B1012B5CD101E05C4AA5
:107B580000E05D4A5F4B1A6055E000286ED05E4B2E
:107B68001A7806DD0132D2B20F2A1A7008D910220B
:107B780005E0013AD2B2102A1A7001D900221A700F
:107B8800F9F7B0FF5AE0554B187057E0FFF79CFE25
:107B9800A0B1002152480FF0C1FF524B042083EDE1
:107BA800000AFEF749F9B42005214F4A0023FEF7E1
:107BB8007BF9FAF79DFB0020FEF73EF9484A16E0EC
:107BC800FFF782FE90B1002148480FF0A7FF484B0D
:107BD800042083ED000AFEF72FF996200521424A7A
:107BE8000023FEF761F90020FEF726F93F4A394BDA
:107BF8001A60294B1888294B1B88C01A284B1B88E8
:107C080090FBF3F0C0B22146FFF7CEFE16E0FFF777
:107C18005BFE08B107F06CF8364B1A68A41814F527
:107C2800967FB8BF344A1C60B8BF1A601B68B3F5AA
:107C3800967F03DD2F4B4FF496721A602F48FFF79B
:107C4800B1FD144B1B78013B0A2B60D8DFE803F029
:107C5800065F5F5F5C15155F11111500FFF74AFE9F
:107C6800FFF726FE002852D00220BDE81040F9F7A1
:107C78007FBD234B1B78022B46D10028214B01D115
:107C8800187010BD01DD012200E0FF221A7010BD3E
:107C980094010020A4250020143A0020783A0020FE
:107CA80038370020DC390020BA370020A43A0020F9
:107CB800E025002004260020162C0020CC250020DA
:107CC800803A0020B0010020F0390020AC010020EB
:107CD800EBA80508003A0020162600200C3A0020E0
:107CE800FC3500200C030020FBA8050820360020E6
:107CF80008030020103A0020D4FEFFFFA001002056
:107D080004380020591A0020BDE81040F2E510BDE3
:107D180010B58CB01E490F2268460EF0A1FD1D4912
:107D28000F2204A80EF09CFD1B490F2208A80EF094
:107D380097FD00210822302000F08AFB012000F086
:107D480081FE002404AB1DF80420E15C302000F023
:107D58007FFB0134012000F075FE0F2CF2D10021C9
:107D68000922302000F074FB012000F06BFE002493
:107D780008AB1DF80420E15C302000F069FB0134F9
:107D8800012000F05FFE0F2CF2D10CB010BD00BF37
:107D980064A4040873A4040882A4040810B58CB071
:107DA8001E490F2268460EF05BFD1D490F2204A8EC
:107DB8000EF056FD1B490F2208A80EF051FD0021B8
:107DC8000822302000F044FB012000F03BFE002494
:107DD80004AB1DF80420E15C302000F039FB0134CD
:107DE800012000F02FFE0F2CF2D1002109223020B3
:107DF80000F02EFB012000F025FE002408AB1DF842
:107E08000420E15C302000F023FB0134012000F065
:107E180019FE0F2CF2D10CB010BD00BF91A40408BC
:107E2800A0A40408AFA4040810B58CB01E490F2202
:107E380068460EF015FD1D490F2204A80EF010FD2E
:107E48001B490F2208A80EF00BFD00210822302044
:107E580000F0FEFA012000F0F5FD002404AB1DF847
:107E68000420E15C302000F0F3FA0134012000F036
:107E7800E9FD0F2CF2D100210922302000F0E8FAA8
:107E8800012000F0DFFD002408AB1DF80420E15CB0
:107E9800302000F0DDFA0134012000F0D3FD0F2C72
:107EA800F2D10CB010BD00BFBEA40408CDA40408D4
:107EB800DCA4040807B50220012108F06BFB0123AC
:107EC80000938DF8043002238DF805300448002310
:107ED80069468DF806308DF8073007F0B3FF0EBD00
:107EE8000004024010B5084C01210022204608F089
:107EF8001EF840F2FF4000F0A5FD012120460A4689
:107F0800BDE8104008F013B80004024008B5FFF7B8
:107F1800E9FF00210A46302000F09AFA012000F01B
:107F280091FD01210A46302000F092FA012000F06C
:107F380089FD00210122302000F08AFA012000F09A
:107F480081FD01210822302000F082FA012000F092
:107F580079FD02210122302000F07AFA012000F098
:107F680071FD00210A46302000F072FA012000F06D
:107F780069FD1B21CD22302000F06AFA012000F0B3
:107F880061FD04210322302000F062FA012000F094
:107F980059FD06210922302000F05AFA012000F08C
:107FA80051FD07210822302000F052FA012000F08C
:107FB80049FD08217022302000F04AFA012000F023
:107FC80041FD1E213020B02200F042FA012000F0CD
:107FD80039FD05219122302000F03AFA012000F005
:107FE80031FD0D210322302000F032FA012000F08B
:107FF80029FD0E210022302000F02AFA012000F08D
:1080080021FD14218022302000F022FA012000F006
:1080180019FD0B218822302000F01AFA012000F007
:1080280011FD0C218222302000F012FA012000F00C
:1080380009FD12218822302000F00AFA012000F000
:1080480001FD13218C22302000F002FA012000F0FB
:10805800F9FC00210A46302000F0FAF9012000F06E
:10806800F1FC3D210222302000F0F2F9012000F05D
:10807800E9FCFFF74DFEFFF791FEFFF7D5FE302034
:108088000021012200F0E4F9012000F0DBFC3D2191
:108098006422302000F0DCF9012000F0D3FC032139
:1080A8000022302000F0D4F9012000F0CBFC04219C
:1080B8000022302000F0CCF9012000F0C3FC0021A0
:1080C8000122302000F0C4F9012000F0BBFC0C2193
:1080D8000822302000F0BCF9012000F0B3FC0D218B
:1080E8000822302000F0B4F9012000F0ABFC0E218A
:1080F8000822302000F0ACF9012000F0A3FC0F2189
:108108000822302000F0A4F9012000F09BFC002197
:108118000A46302000F09CF9012000F093FC02226E
:108128004021302000F094F9012000F08BFC302031
:108138004121002200F08CF9012000F083FC3F214E
:10814800D422302000F084F9012000F07BFC0021CB
:108158000122302000F07CF9012000F073FC10218E
:108168000F22302000F074F9012000F06BFC11217F
:108178000F22302000F06CF9012000F063FC12217E
:108188000022302000F064F9012000F05BFC13218C
:108198000022302000F05CF9012000F053FC092196
:1081A8003C22302000F054F9012000F04BFC002163
:1081B8000122302000F04CF9012000F043FC30206F
:1081C8003421024600F044F9012000F03BFC302045
:1081D8003721024600F03CF9012000F033FC36213B
:1081E8000322302000F034F9012000F02BFC392163
:1081F8000322302000F02CF9012000F023FC3B2161
:108208003C22302000F024F9012000F01BFC3C2126
:108218000A46302000F01CF9012000F013FC002170
:108228000A46302000F014F9012000F00BFC51211F
:10823800C022302000F00CF9012000F003FC52218C
:108248003020002200F004F90120BDE8084000F0C9
:10825800F9BB00BF2DE9F04F454E464D93B00121C3
:108268004FF4001008F096F9304607F039F94FF04E
:10827800C0630293404B0393404B002404934FF494
:10828800B4794FF400334FF480684FF400674FF42B
:10829800005A4FF4807B304602A90C93019309974A
:1082A800CDF8189005940794CDF82080CDF828A033
:1082B800CDF82CB00D9407F09FF92246304630498E
:1082C80007F0F5F93046012107F0FBF901210A46CC
:1082D8004FF0402008F0CCFB284607F001F9294A66
:1082E800019B0392284A0C9304922846402202A933
:1082F800059209970294CDF818900794CDF820803C
:10830800CDF828A0CDF82CB00D9407F075F92246C9
:1083180028461E4907F0CBF92846012107F0D1F974
:1083280042F2107701220221194808F0A1FB3846D1
:1083380000F088FB3046012107F099F90121284611
:1083480007F095F9384600F07DFB0B238DF8443093
:1083580011A801238DF845408DF846408DF8473027
:1083680000F08EFD384600F06DFB13B0BDE8F08FCD
:1083780010600240886002400C400040CA22002081
:108388002A1D00200C3C0040FA1F00205A1A002029
:10839800003C004002481021012207F0DFB900BF6D
:1083A8001060024013B50220012108F0F3F84FF4E1
:1083B80010730E4C009302238DF804308DF80530AD
:1083C80001238DF806302046002369468DF80730D2
:1083D80007F038FD20460621042207F0B3FD2046A9
:1083E8000921042207F0AEFD1CBD00BF00040240B5
:1083F80030B5154D85B001214FF4001008F0EEF8A6
:10840800284607F0B5FD0023ADF804304BF6FF739E
:10841800ADF806303323ADF808304FF48063ADF87B
:108428000A304FF48043ADF80C3004AC074B2846B3
:10843800012144F8103D07F03DFE2846694607F043
:10844800C5FD05B030BD00BF00540040801A0600CD
:1084580073B54FF4961306460D461446019304E08F
:10846800019B5A1E0192002B57D031484FF400311E
:1084780007F038FF0028F3D12D48012107F026FE28
:108488004FF48053019304E0019B5A1E0192002B84
:1084980045D02748274907F010FF0028F4D0244882
:1084A8003146002207F02AFE4FF48053019304E07E
:1084B800019B5A1E0192002B33D01D481E4907F01C
:1084C800FCFE0028F4D01A48294607F09AFE4FF41B
:1084D8008053019303E0019B5A1E01921BB3144879
:1084E800164907F0EAFE0028F5D01148214607F0A2
:1084F80088FE4FF49613019303E0019B5A1E0192E4
:108508009BB10B480E4907F0EDFE0028F5D008484E
:10851800012107F0E7FD002008E0012006E0022025
:1085280004E0032002E0042000E005207CBD00BF39
:10853800005400400100030082000700800007008B
:108548000400001037B54FF4961304460D46019306
:1085580005E0019B5A1E0192002B00F09B805648B3
:108568004FF4003107F0BEFE0028F2D15248012135
:1085780007F0ACFD4FF48053019305E0019B5A1EB0
:108588000192002B00F088804B484C4907F095FE7B
:108598000028F3D048482146002207F0AFFD4FF4E9
:1085A8008053019304E0019B5A1E0192002B75D061
:1085B8004148434907F081FE0028F4D03E48294647
:1085C80007F01FFE4FF48053019304E0019B5A1EED
:1085D8000192002B64D038483A4907F083FE0028FE
:1085E800F4D03548012107F071FD4FF48053019311
:1085F80004E0019B5A1E0192002B53D02E482F49AC
:1086080007F05BFE0028F4D02B482146012207F032
:1086180075FD4FF48053019304E0019B5A1E0192AB
:10862800002B41D0244C2849204607F05BFE002847
:10863800F3D02046002107F069FD20460121238B55
:1086480007F050FD4FF48053019304E0019B5A1E3C
:108658000192002B2AD018481C4907F043FE002835
:10866800F4D0154807F0CFFD4FF480530193124A18
:1086780003E0019B591E0191D3B113889B05F8D4DF
:10868800012104460C4807F041FD0B48104907F04A
:1086980043FE0EE001240CE002240AE0032408E073
:1086A800042406E0052404E0062402E0072400E090
:1086B800082420463EBD00BF0054004001000300CE
:1086C80082000700040000100200001040000010A3
:1086D8000004001013B54FF496130446019305E007
:1086E800019B5A1E0192002B00F0AF8060484FF4A6
:1086F800003107F0F7FD0028F2D15D48012107F0AD
:10870800E5FC4FF48053019305E0019B5A1E01924A
:10871800002B00F09C805648564907F0CEFD0028F3
:10872800F3D05348A021002207F0E8FC4FF480530F
:10873800019305E0019B5A1E0192002B00F08980ED
:108748004B484D4907F0B9FD0028F3D0210A4848A5
:1087580007F057FD4FF48053019304E0019B5A1E24
:108768000192002B77D04248444907F0BBFD00280E
:10877800F4D0E1B23E4807F044FD4FF48053019332
:1087880004E0019B5A1E0192002B66D038483B49F1
:1087980007F0A8FD0028F4D03548012107F096FC21
:1087A8004FF48053019304E0019B5A1E0192002B61
:1087B80055D02F482F4907F080FD0028F4D02C48C9
:1087C800A121012207F09AFC4FF48053019304E0A1
:1087D800019B5A1E0192002B43D0254C2849204664
:1087E80007F080FD0028F3D02046002107F08EFC1A
:1087F80020460121238B07F075FC4FF48053019329
:1088080004E0019B5A1E0192002B2CD018481D49E8
:1088180007F068FD0028F4D0154807F0F4FC4FF481
:1088280080530193124A03E0019B591E0191E3B161
:1088380013889905F8D4012104460D4807F066FC11
:108848000B48114907F068FD10E001240EE00224EE
:108858000CE003240AE0042408E0052406E00624CA
:1088680004E0072402E0082400E0092420461CBD97
:1088780000540040010003008200070004000010BB
:1088880002000010400000100004001013B54FF45F
:1088980096130446019305E0019B5A1E0192002B92
:1088A80000F0AF8060484FF4003107F01BFD00284E
:1088B800F2D15D48012107F009FC4FF48053019380
:1088C80005E0019B5A1E0192002B00F09C8056483F
:1088D800564907F0F2FC0028F3D05348A0210022A3
:1088E80007F00CFC4FF48053019305E0019B5A1EDE
:1088F8000192002B00F089804B484D4907F0DDFCC0
:108908000028F3D0210A484807F07BFC4FF4805335
:10891800019304E0019B5A1E0192002B77D0424834
:10892800444907F0DFFC0028F4D0E1B23E4807F0E4
:1089380068FC4FF48053019304E0019B5A1E019296
:10894800002B66D038483B4907F0CCFC0028F4D00F
:108958003548012107F0BAFB4FF48053019304E036
:10896800019B5A1E0192002B55D02F482F4907F022
:10897800A4FC0028F4D02C48A121012207F0BEFB5A
:108988004FF48053019304E0019B5A1E0192002B7F
:1089980043D0254C2849204607F0A4FC0028F3D0F2
:1089A8002046002107F0B2FB20460121238B07F067
:1089B80099FB4FF48053019304E0019B5A1E0192E6
:1089C800002B2CD018481D4907F08CFC0028F4D047
:1089D800154807F018FC4FF480530193124A03E03E
:1089E800019B591E0191E3B113889C05F8D401211C
:1089F80004460D4807F08AFB0B48114907F08CFC28
:108A080010E001240EE002240CE003240AE0042410
:108A180008E0052406E0062404E0072402E0082410
:108A280000E0092420461CBD00540040010003005A
:108A3800820007000400001002000010400000102F
:108A48000004001082B0002304E0019B013301936D
:108A5800009B01330093009B8342F6D302B070471A
:108A680037B54FF4805304460D46019304E0019B4B
:108A78005A1E0192002B6DD03C484FF4003107F08C
:108A880031FC0028F3D13948012107F01FFB4FF4CE
:108A98008053019304E0019B5A1E0192002B5BD086
:108AA8003248334907F009FC0028F4D02F48A021A8
:108AB800002207F023FB4FF48053019304E0019B4D
:108AC8005A1E0192002B49D028482A4907F0F5FB85
:108AD8000028F4D0210A254807F093FB4FF480536F
:108AE800019304E0019B5A1E0192002B38D01F48C5
:108AF800214907F0E2FB0028F4D0E1B21B4807F057
:108B080080FB4FF48053019303E0019B5A1E0192AE
:108B180043B31648184907F0D0FB0028F5D013488E
:108B2800294607F06EFB4FF49613019303E0019B6F
:108B38005A1E0192C3B10D48104907F0D3FB002813
:108B4800F5D00A48012107F0CDFA0D48FFF77AFF62
:108B580000200AE0012008E0022006E0032004E0EB
:108B6800042002E0052000E006203EBD005400403D
:108B780001000300820007008000070004000010C5
:108B8800A0860100F7B54FF4805304460D461646FB
:108B9800019304E0019B5A1E0192002B74D04048B7
:108BA8004FF4003107F09EFB0028F3D13C48012127
:108BB80007F08CFA4FF48053019304E0019B5A1E8E
:108BC8000192002B62D03648364907F076FB002820
:108BD800F4D03348A021002207F090FA4FF48053D4
:108BE800019304E0019B5A1E0192002B50D02C489F
:108BF8002D4907F062FB0028F4D0210A284807F025
:108C080000FB4FF48053019304E0019B5A1E01922C
:108C1800002B3FD02248254907F04FFB0028F4D00D
:108C2800E1B21F4807F0EDFA4FF48053019304E0D6
:108C3800019B5A1E0192002B2ED019481B4907F0A0
:108C48003CFB0028F4D000244FF4961710E0295D6F
:108C5800134807F0D6FA019703E0019B5A1E0192C8
:108C6800E3B10F48124907F03DFB0028F5D0013465
:108C7800E3B2B342EBD30A48012107F033FA0D48B7
:108C8800FFF7E0FE00200AE0012008E0022006E0ED
:108C9800032004E0042002E0052000E00620FEBDD9
:108CA8000054004001000300820007008000070014
:108CB80004000010A086010013B50520012107F06B
:108CC80069FC184C4FF4E053009302238DF80430EC
:108CD8008DF805302046002369468DF806308DF85A
:108CE800073007F0AFF820460A21062207F02AF9D4
:108CF80020460C21062207F025F9062220460B21E2
:108D0800A4F5006407F01EF94FF4004320466946B5
:108D1800009307F097F820460F21062207F012F972
:108D28001CBD00BF000802401FB50446FFF7C2F88B
:108D3800FFF75EFBFFF7EAF8FFF7BEFF01214FF4EC
:108D4800004007F04BFC02940F4C1023ADF80230A2
:108D5800204600236946ADF80430ADF80C30ADF874
:108D68000030ADF8063007F068FD69464FF0402046
:108D780007F037FE2046012107F0E7FD4FF04020BD
:108D8800012107F0E2FD1FBD003C004082B0002336
:108D980004E0019B01330193009B01330093009B86
:108DA8008342F6D302B0704707B50420012107F0CB
:108DB800F1FB01214FF4804007F01CFC4FF40073D5
:108DC800009300238DF804300348012369468DF889
:108DD800073007F037F80EBD000802400D4B07B505
:108DE8001A680D484FF47A73B2FBF3F20B4B013A51
:108DF8005A600B4AF02182F8231000229A60072259
:108E08001A60084B084A00930121084B01F0ECFF57
:108E18000EBD00BFD00100201C26002010E000E09D
:108E280000ED00E0EC020020D00200203802002013
:108E3800054B1A6812B11A68013A1A60034B1A688E
:108E480001321A60704700BFDC250020F42500209D
:108E580082B0044B0190019A1A601A68002AFCD16A
:108E680002B07047DC250020704700BF40F0BE60AC
:108E7800024B40F42020D860704700BF00ED00E0AE
:108E8800C37810B503B3164B4278DB688478DB43AC
:108E9800C3F30223C3F10401C9B202FA01F10F229C
:108EA80042FA03F2C9B222400A430E4B017812017A
:108EB800CB18D2B283F8002303780122590903F0B2
:108EC8001F0302FA03F307E003780122590903F0AC
:108ED8001F0302FA03F32031024A42F8213010BD81
:108EE80000ED00E000E100E021F0604121F07F01A9
:108EF800014B08439860704700ED00E0044B1A6985
:108F080009B1104301E022EA00001861704700BF70
:108F180000ED00E0044B1A6804280CBF42F004027C
:108F280022F004021A60704710E000E0014B93ED54
:108F3800000A70473C2C0020014B93ED000A704753
:108F4800342C0020014B93ED000A7047482C002078
:108F5800014B93ED000A7047382C0020014B93ED2C
:108F6800000A70474C2C0020014B93ED000A704713
:108F7800402C00200000000010B5FDF791FE0020F5
:108F8800012324210246FDF7F5FE114B1C78002031
:108F9800012C05D10146FDF7C6FF2046002104E05B
:108FA8000721FDF7C0FF01200721FDF7BCFF632261
:108FB8001221C020FFF74CFA02200121FDF7B3FF70
:108FC800FEF790F80120BDE81040FEF780B800BF1A
:108FD800F40D00200D4B1B78062B05D10C4B0D4AC8
:108FE800196812688A181A600B4B1B78012B084BFA
:108FF800196805D1094A914207DD01321A607047A4
:10900800074A914201DD01321A607047A425002009
:10901800102C00209C250020F40D00207FD1F008A2
:10902800FF27ED080E4B1B78062B05D10D4B0E4A7A
:10903800196812688A1A1A600C4B1B78012B094BA5
:1090480005D10B4A1968914208DC1A6070471A6802
:10905800B2F57A2FDCBF4FF47A221A60704700BF4E
:10906800A4250020102C00209C250020F40D0020B1
:1090780020A107002DE9F04F694B6A4C1B688DB0A1
:1090880019220A9068485343B0FBF1F01C190D46A9
:1090980008F010FE41EC100B0AF042FF51EC100BE7
:1090A80009F040F910F0010F804618BF00F1FF38B1
:1090B80005FB08F008F0FEFD064620460F4608F0BE
:1090C800F9FD02460B463046394608F093FF044640
:1090D8000D4645EC104B0AF023FF57EC106B204669
:1090E80032463B46294608F0A7FCCDE9020139463D
:1090F800304609F017F946A3D3E900230B90DDE9C0
:10910800020109F0C9F8002858D1012000264FF0C3
:109118001509314607464FF0000A4FF0000B03E0EF
:1091280030463946069E049FA7FB0A23541807FBBE
:109138000B333E4A43F100050023A242AB41CDE97F
:1091480004453ED3A6FB0A23141806FB0B33374805
:1091580043F100050021A042A941CDE9064530D3DD
:10916800DDE902012CA3D3E90023049C069D09F044
:1091780093F840BBDDE9022300202D4908F03AFFAF
:1091880082468B464BEC10AB0AF0CAFE5046594655
:1091980053EC102B8DED080B08F04EFCCDE90201C5
:1091A800DDE9080109F08CFB09F1FF395FFA89F95B
:1091B80082468B46B9F1000FB2D104E001250024A4
:1091C80001E035463C460B9A0A9BD1B25BB918467A
:1091D80022462B46FDF7CEFD0A980123009301464F
:1091E8004246034609E022462B460120FDF7C2FD10
:1091F80001200090014642460023FDF7AEFEFDF730
:1092080071FF01200DB0BDE8F04FFDF760BF00BF52
:10921800956479E17FFDA53DBBBDD7D9DF7CDB3DFA
:10922800103A002040787D0100E9A435FFFF0F00C7
:109238000000F03F224A234B1278012A10B518602B
:1092480009D1214A904201DD01321A601F4A1B6888
:1092580093420DDC0AE01E4A904201DD01321A6099
:109268001B68B3F57A2F03DC4FF47A22154B1A608A
:10927800144B184A1968184B184C1B68CB189342A2
:10928800236018DC0020FFF7F5FE01202168FFF7B6
:10929800F1FE0B4B1C780020012C05D10146FDF78F
:1092A80042FE2046002104E00721FDF73CFE012094
:1092B8000721FDF738FE034B1A68094B1A6010BDE9
:1092C800F40D0020102C00207FD1F00820A1070009
:1092D800FF27ED0880D1F008282C00202C2C002036
:1092E800F8350020014B1868A4E700BF10260020BD
:1092F8007047FEE7FEE7FEE7FEE7704770477047F6
:1093080002F022B910B5094CA37A4BB1084B1A6880
:1093180022F006021A6000F013F8204600F041FE21
:109328004FF48020BDE8104006F0E8BA1C26002063
:1093380010ED00E0014801F003B800BF1C26002032
:10934800364BD3F8882042F47002C3F88820344B97
:109358001A6842F001021A6000229A60196821F026
:10936800847121F4803119602E495960196882B0DE
:1093780021F480211960DA60009201921A6842F49F
:1093880080321A601A6802F400320192009A01329F
:109398000092019A1AB9009AB2F5A06FF2D1204B47
:1093A8001B6813F4003318BF01230193019B012BA1
:1093B8002ED11B4B1A6C42F080521A641A4A11685B
:1093C80041F4804111609A689A609A6842F40042B8
:1093D8009A609A6842F4A0529A60144A5A601A68CD
:1093E80042F080721A6019680D4A8901FBD5104B4A
:1093F80040F205611960936823F003039360936852
:1094080043F002039360936803F00C03082BFAD12E
:10941800024B4FF000629A6002B0704700ED00E026
:109428000038024010300024007000400854400703
:10943800003C0240184B194A996801F00C010429B4
:1094480003D0082903D0164B19E0164B17E05968CA
:109458005A6811F4800F596814BF124B104B02F070
:109468003F02B3FBF2F30C4A5268C2F30142C1F364
:109478008811013252004B43B3FBF2F3074A1360E1
:10948800054B9A68054BC2F303129A1819681279AA
:1094980021FA02F21A60704700380240D001002019
:1094A8000024F40000127A0037B51C23012400259B
:1094B80001A88DF804308DF805508DF806408DF818
:1094C8000740FFF7DDFC2046214607F087F80A49E8
:1094D80040F2E1434B6040F24F130B800D814D8009
:1094E8004FF0804007F022FC4FF080402146224692
:1094F80007F0E1FF3EBD00BF502C002008B54FF03B
:109508008040012107F0ECFF60B101214FF080405D
:1095180007F0F1FFFEF79EFA034B044A11781A7818
:109528008A181A7008BD00BFC32500200C3A002015
:1095380008B5402006F0D4F930B1FCF713FE4020FE
:10954800BDE8084006F0DAB908BD0000014608B5D4
:10955800044808F08FF90348402108F038FA002839
:10956800F9D008BD00440040F0B589B04FF4E133AC
:109578000120019300232B4CADF808301E4601460C
:10958800ADF80A30ADF80C30ADF810300C23ADF85A
:109598000E3006F0FFFF4FF40030012107F01EF8EF
:1095A80020680221072206F0CDFC0722606803210B
:1095B80006F0C8FC0125022704232068059305A9A5
:1095C8008DF81A608DF81B508DF818708DF8197089
:1095D80006F038FC08236068059305A98DF8187013
:1095E80006F030FCA06801A908F09AF82A4640F273
:1095F80025510D4808F0D2F9262307A88DF81C300C
:109608008DF81D608DF81E608DF81F50FFF738FC2F
:10961800A068294608F001F9044A054B1A6009B008
:10962800F0BD00BFE401002000440040559500084B
:109638009C3B0020024B9868002108F0EEB800BF60
:10964800E401002010B5094C40F22551204608F0ED
:10965800C8F950B1A288D2B2112A02D1044B012113
:109668001970044B19884A401A8010BD0044004004
:10967800550D0020600D00207047704773B501201C
:10968800014606F087FF264C4FF4D8530093022377
:1096980003268DF804302046002369468DF80630ED
:1096A8008DF807308DF8056006F0CCFB20460821C0
:1096B8000A2206F047FC204609210A2206F042FC4D
:1096C80020460B210A2206F03DFC0A2220460C21E6
:1096D80006F038FC01254FF4806320466946009364
:1096E8008DF806508DF807508DF8056006F0AAFB36
:1096F8000A210A46204606F025FC29464FF48040F8
:1097080006F078FF8020294606F050FF4FF0805081
:10971800294606F09FFF284606F0F0F87CBD00BFFA
:109728000000024007B54FF4C060FFF79FFB4323DA
:109738008DF804300322012301A88DF805308DF837
:1097480006208DF80730FFF79BFB0EBD78235843A2
:109758000723B0FBF3F0002301338342FCD97047A1
:109768004FF47A735843F1E737B50023104C01934F
:1097780005460320FFF7EAFFEB681A69013C0192EE
:1097880013D0019A002AF4DA019A42F001020192F8
:10979800019A1A61064A1969013A019102D00199A0
:1097A800C907F8D40320FFF7D1FF00203EBD00BF52
:1097B800410D030010B5C47874B900EB820003337F
:1097C8009B10D0F8D000224603E051F8044C013237
:1097D800046004319A42F8D1002010BD033230B53C
:1097E8009210D0F8D0400B46002003E025680130E5
:1097F80043F8045C04339042F8D101EB800030BD9B
:109808000122F0B50023827040220129C3708280B2
:109818000CD108230370042343704FF4A073C38052
:1098280002230372C1724FF0A04309E041B90C232F
:109838000370062343704FF4A063C3801F4BC172AB
:1098480003F500620261C3604678044601461A4681
:10985800002508E002F5106C02F530620A65C1F8CF
:1098680014C001353A460431B54202F12007F1D35C
:1098780003F58062426103F58862C0F8CC2006785F
:1098880003F5A0650146002203E0C1F88C500132BF
:1098980020350431B242F8D31946002202E0C4F858
:1098A800CC1001320434B24201F58051F7D303F5EC
:1098B8006063C0F80C310020F0BD00BF0000044018
:1098C80038B5037AC2680025012B044625D1936B6D
:1098D800417A65F3104309B143F480139363D36865
:1098E80023F4800323F0500343F010036FF3C30302
:1098F8006FF3C7136FF351436FF3D343D36020461D
:10990800FFF732FFE378012B3ED1052363F34405CB
:10991800E36845F020059D6036E0D36843F04003D6
:10992800D360FFF721FF237A627A032B14BF4FF429
:1099380034134FF43C130AB143F48013E268142043
:109948009363FFF70DFFE268217AD368032908BF04
:1099580043F48033D360237A032B15D1156B01238D
:1099680063F39B656FF3D7552D2345F0805563F35B
:1099780016451563C820FFF7F3FEE36845F40005B4
:109988001D63C820FFF7ECFEE378012B07D1E368DD
:109998009D68052262F3440545F020059D6000207E
:1099A80038BDC3689A6842F001029A600020704787
:1099B800C3689A6822F001029A600020704707B5D0
:1099C80000230193019B43F020030193019B61F362
:1099D8008A130193019BC2681361064B1169013B0D
:1099E800019102D001998806F8D40320FFF7AEFE52
:1099F80000200EBD410D030007B500230193019B14
:109A080043F010030193019BC2681361064B11696F
:109A1800013B019102D00199C906F8D40320FFF750
:109A280095FE00200EBD00BF410D030008B5C268B9
:109A3800D36801296FF35D736FF39E7302D143F00E
:109A4800005302E009B943F080433220D360FFF7A6
:109A580087FE002008BDC368586900F00100704700
:109A6800C3685B6913F0010F14BF00200120704721
:109A7800C368586900F001007047C3685A6998695B
:109A880010407047C3685868704703691A6861F3E3
:109A980001021A607047C268002393614FF0FF33D8
:109AA8005361536053610B4B9361C3789169002BE9
:109AB80014BF4FF400634FF4016343F4701343F48D
:109AC800405343F0080321EA03010B43936100204C
:109AD800704700BF00080080F8B5D0F80C310022AC
:109AE8001A60036915461A6865F3CC221A60C37AAE
:109AF800012B04461BD10321FFF7C7FFE368802130
:109B08004FF4800261F30F0259629A62C02262F335
:109B18000F0561F31F454FF4A072C3F8045162F3B7
:109B28000F056FF31F45C3F80851C3F80C511021F6
:109B38002046FFF744FF2046FFF75EFF2269002317
:109B48004FF0FF311361204653611E469161FF2596
:109B5800D361214610E082691768C7F3076707F0E9
:109B68008007FFB2002F14BF4FF0904700271760FF
:109B7800013316610430956062789342EBD3002379
:109B88001D46FF2010E04A6D1668C6F3076606F00A
:109B98008006F6B2002E14BF4FF0904600261660DD
:109BA800013315610431906062789342EBD32369E5
:109BB8001A6942F480721A61E278012A04D1054ACE
:109BC800402161F359421A632046FFF764FF0020E1
:109BD800F8BD00BF0301010003699B68C3F341039B
:109BE800013B022B9ABF024AD05C0320704700BF9A
:109BF80020A5040810B5036981699C680A68C4F344
:109C08004100022802D06FF30A0202E0032060F349
:109C18000A020A605A6842F480725A60002010BD35
:109C280030B54D780B780022012D00EB830405D167
:109C380005FA03F3A46963F30F0205E0012505FAA9
:109C480003F3646D63F31F422368C3F3072505F02C
:109C58008005EDB26DB98D6865F30A03CD78C988C2
:109C680065F3934361F3995343F0805343F40043FE
:109C780023600369D9690A43DA61002030BD30B531
:109C88004D780B780024012D224600EB830105D185
:109C980005FA03F3896963F30F0205E0012505FA64
:109CA80003F3496D63F31F4203696FF3CF340C600C
:109CB800D96921EA0202DA61002030BDF8B54F788F
:109CC8000B78012F00EB830349D19E694C693568F5
:109CD80033692A4664F3120314B967F3DC430BE0D3
:109CE8008F68E419013CB4FBF7F7CC7867F3DC43E1
:109CF800012C08BF64F35E733361C378012B06D16E
:109D08000B780C6900EB83039B695C610CE0CB78F2
:109D1800012B09D04B693BB103690C785E6B0127B5
:109D280007FA04F434435C63CB78012B07D1036949
:109D38009B68DB0554BF45F0005245F080520B7814
:109D480000EB830342F004429B691A60CB78012B35
:109D580038D10A788B8AC968FFF72CFD32E05E6D2E
:109D68004F6935688C6833692A462FB964F3120342
:109D7800012464F3DC430AE03F19013FB7FBF4F721
:109D8800BF05BF0D67F3DC437C4364F31203336103
:109D9800C378012B05D10B780C6900EB83035B6D4D
:109DA8005C61CB78012B06D14B7913B145F0005299
:109DB80001E045F080520B7800EB830042F004424A
:109DC800436D1A600020F8BD73B54D78012D3DD163
:109DD80083694A691E681C690094E4B242B962F357
:109DE80006048DF800409DF8024065F3C4040EE0B7
:109DF8008D68AA4286BF4D6165F3060462F30604C6
:109E08008DF800409DF80240012262F3C4048DF8E9
:109E18000240009A1A61C278012A05D10A780C69B1
:109E280000EB82029269546146F004421A60C378DA
:109E3800002B34D14B69002B31D003690A78586B59
:109E4800012101FA02F202435A6328E00B784E69B5
:109E58008C6800EB83035B6D1A681D690095EDB291
:109E680006B14C6164F306059DF802408DF8005078
:109E7800012565F3C4048DF80240009C1C61C37879
:109E8800012B05D10B780C6900EB83035B6D5C61DA
:109E98000B7800EB830042F00442436D1A60002007
:109EA8007CBD4B78012B0B7800EB83000AD18269CB
:109EB8001368C3F3076101F08001C9B221B143F00F
:109EC800804301E0426D136843F4001313600020DF
:109ED80070474B78012B0B78C97800EB83000CBFD7
:109EE8008269426D02391368C9B26FF3555301296B
:109EF80098BF43F0805313600020704703699A6944
:109F0800D8691040000C704700EB810102694B6D65
:109F18009B6850691840704703699869DB69184065
:109F280080B2704782B000230093C0238DF80330BD
:109F38000122002362F3C4038DF8023018238DF840
:109F48000030009A436D1A61C278012A06D100F5E3
:109F5800B96058611A684FF080221A6002B07047E1
:109F6800D0F8143110B50446D3B103699A68D20702
:109F780016D5827A42B1D0F80C21D0F80C116FF3C3
:109F880041026FF300020A605A6842F001025A6007
:109F98000520FFF7E5FB23695A6822F001025A60A1
:109FA80010BD837A63B103699B68D90708D5D0F8D7
:109FB8000C31D0F80C216FF341036FF300031360E9
:109FC8007047012310B5002280F812310446034679
:109FD800FF2104E058698160186D01328160607862
:109FE80004338242F6D3236900221A615A61DA6186
:109FF8004FF0FF329A612046FFF7FEFC2046102101
:10A00800BDE81040DBE44B78012B0B7800EB8300B4
:10A018000FD183691868C0F3074000F02003DBB252
:10A02800CBB900F00200C0B200280CBF30202020BD
:10A038007047436D1868C0F3074000F02003DBB297
:10A048005BB900F00200C0B200280CBF4FF44050CA
:10A058004FF400507047102070474FF480507047FD
:10A068004B78012B0B7810B500EB83030AD19C6960
:10A07800102A236802D1BDE8104012E7202A0CD02C
:10A08800302A0FE05C6DB2F5805F236802D143F49B
:10A0980000131BE0B2F5005F02D143F0006315E046
:10A0A800B2F5405F0FD1C3F3074202F02002D2B2EB
:10A0B80022B100234B71BDE810400AE743F08063EA
:10A0C80043F0802302E00AB962F3CF33236010BD66
:10A0D800F8B50446FFF794FB0122002384F8122107
:10A0E80084F8133128271646194640250CE007FB4B
:10A0F80003F000F58C7022182354D3805670D17069
:10A108009560D1605161013362789342EFD30023A7
:10A118002826194640250CE006FB03F000F55C7084
:10A1280022182354D3805170D1709560D160516149
:10A13800013362789342EFD32046FFF739FC20467B
:10A14800FFF7BEFB00212046FFF770FC2046FFF713
:10A15800C3FC2046BDE8F840FFF723BC70B5CDB27C
:10A168000C464FF0280601F07F0106FB010115F0AF
:10A17800800F14BF01F58C7101F55C7104F07F0448
:10A18800ED090C704D708A60CB7005B1CC80022B44
:10A1980001D100230B71FFF743FD002070BD10B5FE
:10A1A800CAB201F07F034FF0280404FB030312F046
:10A1B800800F14BF03F58C7303F55C7301F07F0106
:10A1C800D20919705A701946FFF759FD002010BDC1
:10A1D80038B501F07F0528246C4304F55C74011937
:10A1E8004B6100238B614B70EBB20355CA60C47896
:10A1F800012C08BF0A6113B9FFF7E6FD01E0FFF77C
:10A208005DFD002038BD70B501F07F042825654349
:10A2180005F58C7541190126E4B2CA600A6100226D
:10A228004E7044558A614B6114B9FFF7CDFD01E0CA
:10A23800FFF744FD002070BDCAB212F0800F10B5C0
:10A248004FF0280306D001F07F0403FB040303F555
:10A258008C7303E003FB010303F55C73D20901244B
:10A2680001F07F0119709C705A701946FFF719FEAA
:10A27800002010BDCAB212F0800F10B54FF02803AD
:10A2880006D001F07F0403FB040303F58C7303E09D
:10A2980003FB010303F55C730024D20901F07F017D
:10A2A80019709C705A701946FFF713FE204610BDAE
:10A2B80008B50B0604D501F07F01FFF780FB01E02C
:10A2C800FFF79AFB002008BD0369002261F30A1218
:10A2D80019680A431A60704703695A6803206FF3C4
:10A2E80041025A60FFF73CBA03695A68032042F0FA
:10A2F80002025A60FFF734BA11F0800F4FF02803BA
:10A3080006D001F07F0103FB010101F58C7103E028
:10A3180003FB010101F55C71FFF775BE11F0800FB9
:10A328004FF0280306D001F07F0103FB010101F57E
:10A338008C7103E003FB010101F55C71FFF790BE2E
:10A348002DE9F74F0446FFF78BFB002800F03F820A
:10A358002046FFF792FB0546002800F03882C0F33C
:10A36800074000F00800C0B2002861D02046FFF77F
:10A37800C5FDA146824627464FF00008DFF86CB3BA
:10A388002E4650E01AF0010F46D05FFA88F21146C7
:10A3980020460092FFF7B8FD10F0010F0546009A1D
:10A3A80020D07B6D01259D60E178A94207D11B690A
:10A3B800D9F87813C3F31203CB1AC9F88833DBF83A
:10A3C800003020461B6811469847E378012B09D1D5
:10A3D800B8F1000F06D194F81131052B02D12046AF
:10A3E800FFF7A0FD05F00203DBB213B17B6D022578
:10A3F8009D6005F00403DBB213B17B6D04259D60FD
:10A4080005F00805EDB23DB1DBF8003020469B6849
:10A4180098477B6D0820986008F101084FEA5A0AAE
:10A42800043709F12809BAF1000FABD135460120EC
:10A43800C5F3074303F00403DBB2002B00F0AF8041
:10A448002046FFF769FD264683464FF00008019530
:10A458009FE01BF0010F00F0978023695FFA88F9ED
:10A4680019695D6B04EB890225FA09F59269ED011A
:10A478009268EDB20D431540EA071CD55A6B0120CE
:10A4880000FA08F122EA01025A63B369974A986010
:10A49800136805465B68204649469847E378AB420F
:10A4A80009D1B8F1000F06D194F81131042B02D16B
:10A4B8002046FFF737FD05F00403DBB213B1B3699B
:10A4C80004259D6005F00803DBB213B1B3690825C4
:10A4D8009D6005F01003DBB213B1B36910259D60D0
:10A4E80005F02003DBB213B1B36920259D6005F0A8
:10A4F8004003DBB213B1B36940259D6005F0020348
:10A50800DBB213B1B36902259D6025F07F0515F014
:10A51800FF0F39D0282505FB084505F58C75C2467F
:10A52800AB696A69C3EB020CAB689C4528BF9C46C3
:10A538000CF1030CB3694FEA9C0C9B696746A04673
:10A5480014E0AA68E9681C1B944228BF1446A3B209
:10A5580040464A46FFF72EF9EB681B19EB60AB69DA
:10A56800E71C1C19AC61B3699B69BF089BB2BB426D
:10A5780005D9AC696B699C4201D2002BE1D1B36962
:10A58800802544469D60D04608F101084FEA5B0BE0
:10A598000436BBF1000F7FF45CAF019D012005F08C
:10A5A8000203DBB213B1E36802225A61C5F3076301
:10A5B80003F08003DBB2CBB1A37A43B1D4F80C31FA
:10A5C800D4F80C216FF341036FF300031360236980
:10A5D8005A6822F001025A60444B1B6820469B6966
:10A5E8009847E3684FF000425A610120C5F30723FA
:10A5F80003F00803DBB2F3B13C4B1B6820465B69F0
:10A6080098472369E2689B684FF400615161A27A18
:10A6180082B1DB070ED5D4F80C311A6842F001027A
:10A628001A601A6842F003021A60314B1A6942F044
:10A6380006021A61012005F00803DBB243B12B4B77
:10A648001B682046DB689847E36808225A610120A6
:10A6580005F01003DBB2002B33D0E3689A6922F0CF
:10A6680010029A611F6A282607F00F0306FB0346AB
:10A67800C7F34343022B06F55C7602D0062B1AD1AA
:10A688000EE047F6F0733B40ABB1C7F30A1720461C
:10A69800F1683A46FFF7A2F8F368DB19F36007E0C0
:10A6A80004F5B96120460822FFF798F8C7F30A179E
:10A6B800B369DF19B761E3689A6942F010029A61D9
:10A6C8000120C5F3072303F01003DBB2002B39D0B8
:10A6D80023695A68002622F001025A603146204652
:10A6E800FFF76DF923463246FF2108E0800200207B
:10A6F80000ED00E058698160186D01328160607872
:10A7080004338242F6D3236901274FF0FF3267F3FF
:10A718000F069A6167F31F460F22DE615A612F22E6
:10A728001A611A686FF30A121A602046FFF7FAFBDB
:10A73800E3684FF480525A61264B1B6820461B6918
:10A7480098473846C5F3072303F02003DBB2EBB183
:10A758002046FFF74FFAE3682046DE68FFF73CFA29
:10A76800032806D10023A3704FF40073A3800923A4
:10A7780004E00123A3704023A380052363F38D26FF
:10A78800E3684FF40052DE6001205A61C5F30743C5
:10A7980003F01003DBB24BB10E4B1B682046DB699C
:10A7A8009847E3684FF480125A610120C5F30745C2
:10A7B80005F02005EDB255B1064B1B6820461B6A13
:10A7C8009847E3684FF400125A610120FFE7BDE89B
:10A7D800FE8F00BF8002002043230B800048704793
:10A7E800F001002038B51F4B1A68511C052A196062
:10A7F80035D11979002201291A6030D09968B1F54C
:10A80800006F08BF9A60174B9968DC68A1421A4626
:10A8180002D100221A7122E086BFC1F500631361DC
:10A82800C1EB0404D0F8EC3598BF14611569B3F88E
:10A8380039300C4C9D428AB204D95918ED1AA160DE
:10A84800256104E06918A1600021ABB221610549C6
:10A8580001240C7104498A188121FFF7D4FC0020D7
:10A8680038BD00BF640D0020EF2C002038B5282328
:10A878000A4D03FB01010A4BB1F888131B69044612
:10A8880028469847D4F8EC352046B3F840300121E3
:10A898002A46FFF79DFC002038BD00BFA72C0020EA
:10A8A8006C02002070B50B7813F0600506460C4664
:10A8B80025D0202D1FD1CD88B5B113F0800F487851
:10A8C80008D0214B21499B682A469847E2881F49AE
:10A8D800304625E01E4B1D4958641E4B30465D61CD
:10A8E8002A4600F022FB1DE0174B48789B68294652
:10A8F8002A46984725E000F077FB022521E04B78AF
:10A908000A2B11D00B2B14D0062B1AD14B881B0AFB
:10A91800212B03D1CA883A2A28BF3A220E49304649
:10A9280000F0EAFA00250CE00C49012200F0E4FAF4
:10A9380007E08B781BB9074A1D46936101E000F0D8
:10A9480053FB284670BD00BF6C020020E72C002096
:10A95800F0010020640D0020020200207C0D002080
:10A9680010B581210446FFF71AFC01212046FFF7A4
:10A9780016FC82212046FFF712FC024B5B689847C1
:10A98800002010BD6C02002038B5D0F8EC35044624
:10A99800B3F8392081210223FFF7E0FBD4F8EC3526
:10A9A8000121B3F8402020460223FFF7D7FB82217C
:10A9B800082203232046FFF7D1FB094B022200257A
:10A9C8001A715D71074B1B689847D4F8EC35064A35
:10A9D800B3F8403020460121FFF7FAFB284638BD7E
:10A9E800B00200206C020020A72C002010B5074CF4
:10A9F800606CFF2807D0064B064A9B6806495269D7
:10AA08009847FF236364002010BD00BFF0010020B9
:10AA18006C020020640D0020E72C002038B5104996
:10AA28000B79012B19D10C690CB90C7115E0D0F810
:10AA3800EC358D68B3F839309C42AAB203D95D1958
:10AA48008D60E41A03E0A3B22C198C6000240C6119
:10AA5800044952188121FFF7D6FB002038BD00BFFA
:10AA6800640D0020EF2C0020002070470020704764
:10AA78000023F0B5084A094E1D4609E01468C75C72
:10AA8800375501340133B4F5006F146008BF156001
:10AA98008B42F3D10020F0BD700D0020EF2C002078
:10AAA800104B114AD3F800C000232DE9F0410F4F95
:10AAB80016461D460DE0146810F8038007F8048058
:10AAC8000134802C08BF2C4614603468644505D0D6
:10AAD80001338B42EFD10020BDE8F0810220BDE8B0
:10AAE800F08100BF7035002084350020F03400204C
:10AAF80021280FD1084B1A680A701A68120A4A707E
:10AB08005A888A70DA78CA701A790A715A794A7139
:10AB18009B798B71002070476402002007B502AB57
:10AB2800012103F8010D1846FFF7A2FF0EBD002111
:10AB380000E00131435C002BFBD199E798E70B4B10
:10AB48000B491A68096891420BD00A498A5C02705D
:10AB58001A680132802A1A6005D100221A60012081
:10AB68007047002070470120704700BF70350020F3
:10AB780084350020F0340020204B1A68204B1B68D5
:10AB88009A42F0B509D135E00133802B08BF002384
:10AB98009A4203D11A4B1A602CE01A4CE15C002946
:10ABA800F2D00A29F0D00D29EED0154C1549134DD5
:10ABB80023600E460023CF182268BA5CC25422686C
:10ABC80001339F18802F08BF53422F689A18974265
:10ABD80010D0B25C1AB10A2A01D00D2AEBD100229A
:10ABE800C254074A116859187F29116003D980395E
:10ABF800116000E000231846F0BD00BF8435002036
:10AC080070350020F0340020704700BFD0F8E435DC
:10AC180010B51B6904469847032384F812310020B5
:10AC280010BD08B5042380F81231D0F8E435DB688C
:10AC38009847002008BD08B5D0F8E035DB6903B1B6
:10AC48009847002008BD08B5D0F8E0351B6A98473A
:10AC5800002008BD08B5D0F8E0355B6A98470020A9
:10AC680008BD002110B5402204460B46FFF776FACE
:10AC78008021402200232046FFF770FA012384F840
:10AC88001231D4F8E435A0785B689847002010BDED
:10AC980013B56946044600F085F99DF8001001F0E7
:10ACA8001F03012B07D0022B0AD073B9204669462F
:10ACB80000F026FA0FE02046694600F007FA0AE09D
:10ACC8002046694600F0A2F905E021F07F01C9B2EB
:10ACD8002046FFF7B1FA00201CBD38B5044600290C
:10ACE8003DD190F81131022B42D1D0F83421D0F85F
:10ACF80020319A4211D9C178D21A0129C0F83421D9
:10AD080004D1D0F82411CB18C0F8243192B22046CF
:10AD1800D4F8241100F000F92AE0D0F83821B2FB69
:10AD2800F3F503FB152565B99A420AD3D0F83C31EF
:10AD38009A4206D229462A4600F0EEF8C4F83C5159
:10AD480016E0D4F8E035DB682BB194F81221032A19
:10AD580001D120469847204600F00FF908E0D0F8C6
:10AD6800E0355B6923B190F81221032A00D1984796
:10AD7800002038BD10B5044659BB90F81131032B9B
:10AD880030D1D0F88C23D0F878339A4214D9C178CE
:10AD9800D21A0129C0F88C2304D1D0F87C13C91821
:10ADA800C0F87C139A4228BF1A4692B22046D4F8BB
:10ADB8007C1300F0CAF815E0D0F8E0351B6923B120
:10ADC80090F81221032A00D19847204600F0C6F8CF
:10ADD80008E0D0F8E0359B6923B190F81221032AE6
:10ADE80000D19847002010BD2DE9F041069F044688
:10ADF800164698460D46FEF741FC20462946C4F8FB
:10AE0800E085C4F8E475C4F8E865FFF761F9D4F89B
:10AE1800E4351B6898472046BDE8F041FEF782BC40
:10AE280000207047D0F8E03510B504461B689847F5
:10AE3800D4F8E4359B689847002010BD08B5D0F8D1
:10AE4800E0355B689847002008BD000012230B809E
:10AE580000487047B002002004230B800048704768
:10AE6800C202002010B5044C04480A46214600F0EE
:10AE780075FA204610BD00BF88350020BFA9050817
:10AE88000A4608B50248034900F068FA014808BDB7
:10AE9800D2A90508883500200A4608B502480349A2
:10AEA80000F05CFA014808BDE0A9050888350020D3
:10AEB80008B50A4608B9044800E00448044900F007
:10AEC8004DFA034808BD00BFEBA90508F8A9050815
:10AED8008835002008B50A4608B9044800E0044847
:10AEE800044900F03BFA034808BD00BF05AA05085D
:10AEF80026AA05088835002010B513460C46C0F868
:10AF08003821C0F83421022280F81121002122467C
:10AF1800FFF779F9002010BD10B50C461346002143
:10AF28002246FFF770F9002010BD10B513460C46F5
:10AF3800C0F89023C0F88C23032280F81121002147
:10AF48002246FFF745F9002010BD10B50C46134600
:10AF580000212246FFF73CF9002010BD0021042300
:10AF680010B50A46044680F811310B46FFF74BF935
:10AF78002046FEF7D7FF002010BD0021052310B59D
:10AF88000A46044680F811310B46FFF721F920469E
:10AF9800FEF7C8FF002010BD282303FB0100B0F80E
:10AFA8008803704790F8C8350B7090F8C9354B7016
:10AFB80090F8CB2590F8CA3503EB02234B8090F824
:10AFC800CD2590F8CC3503EB02238B8090F8CF2564
:10AFD80090F8CE3503EB02239BB2CB80C0F83C310E
:10AFE800012380F81131704710B591F90030002B1A
:10AFF800044601DBCB880BB9802100E00021FFF774
:10B008001BF92046BDE81040FEF78CBF38B50D4649
:10B0180004466B780979012B10D027D3032B51D123
:10B0280090F81231022B28D0032B47D16B889BB99B
:10B0380091B1802910D0FFF7FFF80DE090F8123198
:10B04800022B1AD0032B39D16B88002B3AD149B186
:10B05800802907D0FFF70EF9D4F8E03520469B6821
:10B06800294698472046FFF779FF2BE090F81231E0
:10B07800022B02D0032B21D106E019B3802921D05D
:10B088002046FFF7D9F81DE011F0800F4FF0280394
:10B0980006D001F07F0103FB010393F81A2103E0B6
:10B0A80003FB010191F87223074B02B101221A60D8
:10B0B800204605490222FFF71FFF03E020462946E4
:10B0C800FFF792FF002038BD800D002038B590F8BA
:10B0D8001231032B04460D460CD10B79012B09D8EC
:10B0E800D0F8E0359B689847EB883BB92046FFF7D6
:10B0F80035FF03E020462946FFF776FF002038BDDC
:10B1080073B54B7804460D46092B00F21C81DFE825
:10B1180013F0D10008011A01E4001A0172000A00B4
:10B128001A01C00092004B881A0A013A062A00F256
:10B138000A81DFE812F007001A0027000801080159
:10B1480008010801D4F8E835A0781B680DF106015C
:10B158009847EB88402B014603D094F81231012B15
:10B168003AD10823ADF8063036E0D4F8E035A078B7
:10B178009B6A0DF106019847022343700146C4F803
:10B18800EC0529E0DBB2052B00F2DD80DFE803F0F7
:10B1980003080D12171CD4F8E835A0785B6817E08F
:10B1A800D4F8E835A0789B6812E0D4F8E835A078A0
:10B1B800DB680DE0D4F8E835A0781B6908E0D4F81E
:10B1C800E835A0785B6903E0D4F8E835A0789B6996
:10B1D8000DF1060198470146BDF80630002B00F036
:10B1E800B680EA88002A00F0B2809A4228BF1A4640
:10B1F800ADF806205CE08B88002B40F0A480CB885B
:10B20800002B40F0A08094F812214B88032A00F00C
:10B218009A8003F07F05204684F813512946FFF7EA
:10B2280053F82046FFF79AFE0DB1022300E00123F0
:10B2380084F812318BE08978464E0129317100F289
:10B24800828094F81231022B02D0032B7BD108E0C4
:10B25800002962D00121032384F8101184F81231E7
:10B2680013E041B9022384F8123184F81011204602
:10B27800FFF7E4FD51E094F81011012920464DD064
:10B28800FFF7DCFD317984F810112046FFF7CAFD7D
:10B2980043E0CA88012A56D194F81231022B02D011
:10B2A800032B50D102E020462B4913E004F58871A6
:10B2B80020460FE094F81231023B012B43D8D4F812
:10B2C80014312449002B0CBF0123032341F80C3F00
:10B2D80020460122FFF710FE39E04B88012B29D0C8
:10B2E800022B34D18B8813F0FF0F30D121691B0A50
:10B2F800013B4A68042B0FD8DFE803F00305070970
:10B308000B00012306E0022304E0032302E00423E8
:10B3180000E0052363F306124A602046FFF71EFE8D
:10B3280015E094F81231023B012B0CD84B88012B05
:10B338000DD10023C4F81431D4F8E03520469B68B9
:10B3480029469847E9E720462946FFF74DFE0020A1
:10B358007CBD00BF800D0020880D002030B5C8B12D
:10B368000023DDB20133C41814F8014C002CF8D1C5
:10B378006B1C5B0013800B7003234B70022305E0EA
:10B38800CA545A1CD2B202338C54DBB210F8012BC7
:10B39800002AF5D130BD00BF70477047704770472D
:10B3A800704770477047000008B5FCF781FA094BF1
:10B3B8005A78187002435A701AB19A7801329A7002
:10B3C80030B99B78034A012B02D90023537093703C
:10B3D80008BD00BF900D00202DE9F84F394B1A78B1
:10B3E800394B2DED028B22B91A68802392FBF3F3B7
:10B3F80000E01B68354A5361354B1A8892B2002A1F
:10B40800FBD0334B00221A80FDF790FD10EE105A46
:10B41800FDF792FD284610EE104A06F06DFC8046B6
:10B428002046894606F068FC41EC100B41EC180BED
:10B4380008F01EFD57EC106BB0EE480AF0EE680AF3
:10B4480008F016FE32463B46404649465BEC10ABD8
:10B4580006F0A6FC06F086FF9FED1E8A07EE100A8E
:10B46800DFED1D7A57EE087A184C52465B46C4ED5C
:10B47800007A4046494606F093FC06F073FF07EE53
:10B48800900A27EE888A84ED018AFDF767FD84ED2E
:10B49800020AFDF769FD84ED030AFCF717F90F4B63
:10B4A80062691B68D31A0E4A07EE100A1268F8EE92
:10B4B800C77A93FBF2F3C4ED047A2383BDEC028BC5
:10B4C800BDE8F88FF40D0020102C0020BC370020B8
:10B4D800400D00200000F04200008C4210260020A1
:10B4E8009C25002007B50420012105F053F84FF4EE
:10B4F8006043009301238DF8043002238DF8053052
:10B508000448002369468DF806308DF8073004F0AA
:10B5180099FC0EBD00080240084B1A684FF47A7374
:10B52800B2FBF3F2064B013A5A60064AF02182F860
:10B53800231000229A6007221A607047D001002069
:10B5480010E000E000ED00E0034B5A6812B15A68C1
:10B55800013A5A60704700BF900D0020024B5860B6
:10B568005A68002AFCD17047900D002030B585B08C
:10B5780004460D4601A85C490A220BF071F95B4BA1
:10B588001B78032B10D8DFE803F00205080B01A88D
:10B59800574907E001A8574904E001A8564901E0C6
:10B5A800564901A80BF046FA04AA131913F80C3CE3
:10B5B8005D19EDB22F2D01D80A3502E0392D01D9D8
:10B5C8000A3DEDB204AB1C194FF6FF7004F80C5C91
:10B5D800FAF730FB0020FAF72FFC0DF103050F24D2
:10B5E800204623345A21002315F8012FA4B2FAF774
:10B5F8003DFCB4F5A57FF3D164205A212C22002309
:10B60800FAF734FC0023CD205A212C22FAF72EFC1D
:10B618000020FAF70FFB354B1B78032B62D8DFE8C5
:10B6280003F002284B5601A931480BF003FA0A220D
:10B6380000212F480CF026FB314A324B1278186053
:10B64800012A06D1304A904201DC01321A602F4AA1
:10B6580006E0B0F5FA5FBCBF4FF4FA521A602C4A04
:10B668001B689342C4BF274B1A602A4B1A682A4B9F
:10B6780020E001A91F480BF0DDF90A2200211D482E
:10B688000CF000FB1E4A254B12781860012A06D1DF
:10B698001D4A904201DC01321A601C4A06E0B0F5EE
:10B6A800FA5FBCBF4FF4FA521A60194A1B689342FA
:10B6B80018DD1A4B1A6015E001A90F480BF0BAF90A
:10B6C8000D4800210A220CF0DDFA154B09E001A90A
:10B6D8000A480BF0AFF9094800210A220CF0D2FA07
:10B6E800104B186005B030BD47AA05080F2600208A
:10B6F800E025002004260020162C0020CC25002060
:10B70800F40D0020182600201FA1070080D1F008A2
:10B7180050DA110010260020102C0020302C0020B8
:10B728000C2C0020C825002010B50D4B0D4C1A68B4
:10B738000D4821460BF056F90C4B0D481A68214666
:10B748000BF050F90B4B0C481A6821460BF04AF9DC
:10B758000A4B0B481A682146BDE810400BF042B965
:10B768001826002056A00508E0250020302C0020CF
:10B77800042600200C2C0020162C0020C8250020B0
:10B78800CC2500209FED010A704700BF0000000093
:10B798009FED010A704700BF000000009FED010AFD
:10B7A800704700BF0000000018B1012801D1034B09
:10B7B80000E0034B1868FDF73DBD00BF00260020E0
:10B7C8001026002010B9034B18687047024B186800
:10B7D800704700BF182600201026002010B9034B20
:10B7E80018687047024B1868704700BF302C00205B
:10B7F8000026002008B54FF49570FBF77BFF40F258
:10B808006523C31A584240EB030008BD08B5C6209B
:10B81800FBF770FF40F28D13C21A504240EB020052
:10B8280008BD4FF4957040F26521FBF755BFC6205F
:10B8380040F28D11FBF750BFDCE760EEA00AB7EECF
:10B84800007AF0EE606A70EE077A40EE006A47EE22
:10B85800A70A36EEC77A08B5C7EE200A10EE900A96
:10B8680006F04AFA0022084B06F09AFA0022074B23
:10B8780006F0E4F806F076FD07EE900AFDEEE77AAA
:10B8880017EE900A9F3008BD000059400000E03FC5
:10B8980038B52DED028BF7EE008AB0EE608A70EEB7
:10B8A800288A10EE900A28EE088A06F025FA08EE93
:10B8B800A88A00220F4B06F073FA044618EE100A05
:10B8C8000D4606F019FA02460B462046294606F0B0
:10B8D80091FB0022084B06F0B1F806F043FD07EE95
:10B8E800900AFDEEE77A17EE900A7730BDEC028BEE
:10B8F80038BD00BF000069400000E03F2DE9F04F6F
:10B90800894F2DED068B97E80F0091B00CAC1037DE
:10B9180084E80F000FCF05AE0FC697E807004FF673
:10B92800FF7386E807009F2077216422F7F727FE38
:10B93800A020772164224FF6FF73F7F720FE9E20A0
:10B94800772164224FF6FF73F7F719FE9F207621BF
:10B9580064224FF6FF73F7F712FE4FF6FF73782154
:10B9680064229F20F7F70BFE0020F9F722FA9F20A8
:10B9780077216522FAF7A0F90C349F2077216422F9
:10B98800FAF79AF90DF12C0A0394F7EE009A4FF0A2
:10B998000F0B00E04D460AF1040AF7EE008A9AED13
:10B9A800009A0024B0EE68AA01E0B846354618EEC1
:10B9B800900A06F0A1F95AA3D3E9002306F0F0F99A
:10B9C80006F0D0FC08EE900A38EEE98AB0EE490A93
:10B9D800F0EE480AFFF731FFB0EE490AF0EE480AE8
:10B9E8000646FFF755FFB2B2074683B22CB9104698
:10B9F80019460F22F9F7A8FA06E0A8B21FFA88F14B
:10BA0800CDF800B0FAF7A2F80134B4F5967FCCD19E
:10BA18003D46F7EE008A002401E045464E4618EE02
:10BA2800900A06F069F93EA3D3E9002306F0B8F9B5
:10BA380006F098FC08EE900A39EEE88AB0EE490A5A
:10BA4800F0EE480AFFF7F9FEB0EE490AF0EE480AB0
:10BA58008146FFF71DFF1FFA89F2804683B22CB991
:10BA6800104619460F22F9F76FFA05E0B0B2A9B2ED
:10BA7800CDF800B0FAF76AF80134B4F5967FCCD166
:10BA8800039B9A4586D104AD0DF12C0B4FF0000AAB
:10BA980001E0B846B146043595ED009AF7EE008A04
:10BAA800002401E0B846B14618EE900A06F024F9E1
:10BAB8001BA3D3E9002306F073F906F053FC08EE44
:10BAC800900A38EECA8AF0EE490AB0EE480AFFF743
:10BAD800B4FEB0EE480AF0EE490A0646FFF7D8FE73
:10BAE800B2B2074683B22CB9104619462246F9F776
:10BAF8002BFA07E01FFA89F01FFA88F1CDF800A0A9
:10BB0800FAF724F80134B4F5C87FCBD15D45C0D12C
:10BB180011B0BDEC068BBDE8F08F00BFAFF300801D
:10BB2800295C8FC2F528F03F24A50408121A06EEF6
:10BB3800902A081AB8EEE67A06EE900AF8EEE67A47
:10BB480008B5C7EE277A17EE900A06F0D5F807A3CE
:10BB5800D3E9002306F024F90022034B05F06EFF19
:10BB680006F0B8FB08BD00BF0000E03F0000000081
:10BB780000F073408A1A06EE902A081AB8EEE67AA0
:10BB880006EE900AF8EEE67A08B5C7EE277A17EEC1
:10BB9800900A06F0B1F807A3D3E9002306F000F9EC
:10BBA8000022034B05F04AFF06F094FB08BD00BFD6
:10BBB8000000E03F0000000000E0684070B5064665
:10BBC8000D460024610704D5A0B231462A46F9F78C
:10BBD800BBF90134B4F5A07FF4D170BD70B5064649
:10BBE8000D460024600704D5A1B230462A46F9F76D
:10BBF800ABF90134C82CF5D170BD114B11481B7835
:10BC08001149124A0068012B114B09D112680860CA
:10BC18001A60104B1A68104B1A60104B1A680CE027
:10BC28001268D2011A600B4B1A680B4BD2011A60CA
:10BC38000A4B1A68C0010860D201094B1A607047A4
:10BC4800F40D00201826002010260020302C00209B
:10BC5800002600200C2C00209C250020EC2500202C
:10BC6800282C0020014B1868FDF7E4BA10260020A4
:10BC780008B5FFF7C2FFBDE80840F3E770B500213B
:10BC88000A222748274D284E284C0BF0FBFF00219D
:10BC98000A22286026480BF0F5FF00210A223060AE
:10BCA80024480BF0EFFF00210A22206022480BF005
:10BCB800E9FF224B326818602B682149D31A06EE37
:10BCC800903A2368B8EEE67A06EE903AF8EEE67A0D
:10BCD800C7EE277AFCEEE77A17EE903A9AB20B8015
:10BCE800531C07EE903AB8EEE77ADFED167A67EE66
:10BCF800277A154BFCEEE76A16EE901A8AB206EE22
:10BD0800902AB8EEE67A198077EEC77AF5EEC07A0F
:10BD1800F1EE10FA01DD01321A80BDE87040A7E7A4
:10BD2800E025002018260020302C00200C2C0020B4
:10BD380004260020162C0020CC250020C825002031
:10BD4800FC3900200000803D903A00200022F0B528
:10BD58001346202603254FF02C0C00E02646303EE3
:10BD6800F6B217460132092E10F8014B0AD897FB94
:10BD7800F5F605FB16772FB9CE1801F803C07470D5
:10BD8800023301E0CC540133092AE7D12022CA54F6
:10BD9800CB1848225A707A229A700022DA70F0BDC5
:10BDA800F0B51F46144B1E78012E8DB005460C4683
:10BDB80020D0A6F1030CDCF1000646EB0C06CEB948
:10BDC8000E4908A80AF00EFE08A86946FFF7BEFF4C
:10BDD8000B496A4604A80AF005FEBDF84800F9F7C1
:10BDE80029FF3846F9F73CFF2846214604AA33467E
:10BDF800FAF75AF80DB0F0BDA425002056A00508A2
:10BE080098A7050810B501210446F9F7C3F8014BB6
:10BE18001C8110BD900D002008B50021C620FBF73D
:10BE28005BFC4FF495700021BDE80840FBF754BC5B
:10BE3800014B9F221A817047900D00200020014677
:10BE4800C82240F23F13F9F7B9B907B50DF1070059
:10BE5800FEF775FE9DF807000EBD08B5FFF7F5FF64
:10BE68000028FBD108BD30B5044687B010EE100A93
:10BE78000D4605F041FF02460B4601A805490AF0A8
:10BE8800B1FD2046294601AA0023FAF70DF807B0AC
:10BE980030BD00BF51AA050808B5084803F034FAB8
:10BEA8000648022103F001FB0028F9D0034803F0FB
:10BEB80057FA07EE900AB8EE670A08BD002001405D
:10BEC80010B52DED028B9FED098A1924FFF7E4FFC9
:10BED800013CE4B238EE008A002CF7D19FED040A49
:10BEE80028EE000ABDEC028B10BD00BF0000000068
:10BEF800ACC868392DE9F04F2DED068B8E4B8F4C71
:10BF08008F495D695F68C1B00646324638A893ED2F
:10BF1800038AD3ED04AAD3ED028A93ED00AA93ED28
:10BF2800069A0AF05FFDA06805F0E6FE02460B4699
:10BF380028A884490AF056FDE06805F0DDFE0246AF
:10BF48000B462CA880490AF04DFD1AEE900A05F020
:10BF5800D3FECDE90801DDE908237C4930A80AF0C1
:10BF680041FD284605F0C8FECDE90401DDE90423BA
:10BF7800774934A80AF036FD18EE900A05F0BCFEA1
:10BF88008046894642464B46724910A80AF02AFD67
:10BF980018EE100A05F0B0FE82468B4652465B4604
:10BFA8006D4914A80AF01EFD1AEE100A05F0A4FE49
:10BFB800CDE90A01DDE90A23684918A80AF012FD4B
:10BFC800384605F099FE54A3D3E90023CDE90601CC
:10BFD80005F0E6FE02460B461CA861490AF002FD80
:10BFE80049EC118B4BEC10AB08F09EF84AA3D3E94F
:10BFF800002351EC100B05F0D3FE02460B4624A893
:10C0080058490AF0EFFC19EE100A05F075FE0246D1
:10C018000B4620A854490AF0E5FCD4ED047AFDEE5D
:10C02800E77A0CA817EE902A50490AF0DBFCB5EE27
:10C03800C08AF1EE10FADFED4E9A37D5304605F09A
:10C0480049FE37A3D3E9002305F0AAFEF1EE487AAA
:10C05800044617EE900A0D4605F04EFE02460B46C2
:10C068002046294605F09CFE02460B462EA1D1E942
:10C07800000105F0BFFF06F075F99FED3E7A07EE67
:10C08800900AF4EEC77AF1EE10FAC6BFC7EEA97AA5
:10C09800394C3A4CF4EEE97AF1EE10FA38DD9FEDBE
:10C0A800347A374D374CC7EE877A76E020A3D3E948
:10C0B80000235046594605F073FE044630460D46A7
:10C0C80005F008FE16A3D3E9002305F069FE024631
:10C0D8000B462046294605F08DFF06F043F907EE8A
:10C0E800900AB7EE007AF4EEC77AF1EE10FA46BF7E
:10C0F80067EEA97A244C254CF4EEE97AF1EE10FAB1
:10C108004ADD9FED1B7A224D224CC7EE877A44E028
:10C118001B4D42E0AFF300806666666666A64C403B
:10C128001F85EB51B81E1940000000A2941A6D42F9
:10C138000000000080842E41AC390020BC3700206C
:10C1480073AA05087DAA050888AA050893AA050800
:10C158009DAA0508A7AA0508B3AA0508BFAA050845
:10C16800CAAA0508D5AA0508E0AA0508ECAA050880
:10C1780000007A440024744962AA05085FAA0508E9
:10C1880003AA05086BAA050868AA050865AA050890
:10C198006EAA050870AA0508954D17EE900A05F0D5
:10C1A800ABFD2A46CDE900013CA8924902940AF069
:10C1B80019FC914B1A68914B1B689642CCBF002220
:10C1C80001229E428E4BD8BF0022DA608D4B1B782D
:10C1D800082B40F09C800220F9F72EFE4FF6FF70E6
:10C1E800F9F73EFD1F20F9F725FD19210023864A9E
:10C1F8002D20F9F759FE4FF6FF70F9F731FD0020B1
:10C208000024F9F717FD0F20B42132464FF6FF73CB
:10C218000094FFF7C5FD0F206E2128AA2346F9F7E1
:10C2280043FEB0206E210DEB00022346F9F73CFED9
:10C238000F20382118AA2346F9F736FEB0203821F6
:10C248001CAA2346F9F730FE0F205C2130AA2346AA
:10C25800F9F72AFEB0205C2134AA2346F9F724FE18
:10C268000F204A2110AA2346F9F71EFEB0204A21C2
:10C2780014AA2346F9F718FE0F209B2120AA23466B
:10C28800F9F712FE0F2084213CAA2346F9F70CFE89
:10C29800B020842124AA2346F9F706FE5B4B1B68CD
:10C2A800B3F57A7FCCBF4FF4FC604FF47840F9F7D0
:10C2B800D7FC0023A0209B210CAAF9F7F5FD544BCD
:10C2C8001B78012B08D14FF4FC60F9F7C9FC4FF437
:10C2D8008C7002214F4A07E04FF6E070F9F7C0FC76
:10C2E8004D4A4FF48C7002210023F9F7DDFD002040
:10C2F800F9F7B6FC4FF4FC60F9F79CFCFFF7E0FD9A
:10C308000F20DC21FFF7AFFD1F20F9F7A9FC3D4BFB
:10C318001B789A1FD2B2012A02D90B2B40F0258232
:10C328003E4B1B78023B052B00F21F82DFE813F01F
:10C3380006007E00E2003B01DE015801DFED387A9D
:10C348002AEE27AA1AEE100A05F0D6FC9DED060B78
:10C358008046894607F08CFD404653EC102B494631
:10C3680005F01EFD1EA3D3E9002305F067FB05F0C9
:10C37800B1FF9DED060B044607F07AFE404653ECEC
:10C38800102B494605F00CFD02460B4616A1D1E9D3
:10C39800000105F051FB05F09DFF4FF6E073009397
:10C3A800054600230520DC213246FFF7F9FC144B33
:10C3B800DB6853B11B4B18881B4B4FF4784719881F
:10C3C8000097A2B2ABB2F9F7C1FB164B1C60164B33
:10C3D8004FF6E0701D60F9F72DFCC6E1AFF3008061
:10C3E8000000000000E063400000000000C05D4065
:10C3F8006EAA0508F9AA0508302C00201826002086
:10C40800900D0020A425002006AB05084C1A00203A
:10C41800F40D002071A9050875A90508242C002031
:10C428000000C842F83700209C3A0020A04B18684A
:10C43800A04B9FEDA19A19683246FFF777FBF4EEFF
:10C44800498AF1EE10FAC8BFF0EE498AF5EE408A43
:10C45800DFED9A7AF1EE10FA48BFF0EE678AF4EE53
:10C46800C98AF1EE10FA04461ED8F4EEE78AF1EE16
:10C4780010FA19DBFDEEE88A002018EE902A4FF436
:10C48800FA71FFF777FB8E4BDB68054653B18D4B8E
:10C4980018888D4B4FF6FF7719880097A2B2ABB278
:10C4A800F9F754FB884B1D60B4EE498ADFED827AB8
:10C4B800F1EE10FAC8BFB0EE678ADFED847AB4EE09
:10C4C800678AF1EE10FA48BFB0EE678AB4EEC98AFF
:10C4D800F1EE10FA00F24981B4EEE78AF1EE10FAB3
:10C4E800C0F24381BDEEC88A794818EE102A4FF48D
:10C4F800FA71AEE06E4B18686E4B32461968FFF75A
:10C5080015FBF5EEC0AAF1EE10FA044627DDDDE9C9
:10C51800080159A3D3E9002305F0B4FEF8B158A3E4
:10C52800D3E90023DDE9080105F03AFC0B46024691
:10C538006849002005F080FA05F0CCFE604BDB6806
:10C54800054653B15F4B18885F4B4FF6FF77198844
:10C558000097A2B2ABB2F9F7F9FA5B4B1D60DDE9BF
:10C56800040149A3D3E9002305F0AAFE002800F03E
:10C57800FC80DDE9040140A3D3E9002305F082FE35
:10C58800002800F0F28042A3D3E90023DDE904018A
:10C5980005F006FC02460B4600204F4905F04CFA10
:10C5A80005F098FE57E0424B1868424B324619682E
:10C5B800FFF7BCFA38A3D3E900230446DDE90A01F2
:10C5C80005F07EFE50B19DED0A0B07F035FE002206
:10C5D80051EC100B414B05F0E3FBB1E0C825B2E08C
:10C5E8002FA3D3E90023DDE9060105F0D9FB2EA32B
:10C5F800D3E9002305F0FEFC05F0B4FE2C4B08EE51
:10C60800100A18682B4B32461968FFF78FFADFEDCE
:10C61800347A4AEE677A2A4BFDEEE77ADB6817EE42
:10C62800905A044625EAE57553B1264B1888264BDF
:10C638004FF6FF7719880097A2B2ABB2F9F786FADE
:10C64800BDEEC88A204B18EE102A1D606FF0B300AB
:10C65800B421FFF78FFA1A4BDB68054653B1194B23
:10C668001888204B4FF4FC6719880097A2B2ABB228
:10C67800F9F76CFA1B4B75E09A9999999999B93F12
:10C688000000000000409F409A9999999999B9BF74
:10C698000000000000408F4089B5F81400E3693FAE
:10C6A80000000000008076401F85EB51B81E19403D
:10C6B80018260020302C00200000FA43000000005B
:10C6C800900D0020F83700209C3A00200000FAC3A3
:10C6D8000CFEFFFF0000694000005940000054C0F4
:10C6E80000004843E83500200000C8425FED027AA8
:10C6F800B4EE679AF1EE10FAC8BFB0EE679AB4EEDE
:10C70800E79AF1EE10FA30D8214B1868214B3246DF
:10C718001968FFF70BFA044619EE100A05F0ECFA4F
:10C7280041EC100B07F088FD00221B4B51EC100B5D
:10C7380005F036FB02460B460020184905F07CF947
:10C7480005F0C8FD0546164BDB6853B1154B188834
:10C75800154B4FF6FF7719880097A2B2ABB2F9F7DD
:10C76800F5F9114B1D600F4B1C60104B1B78022B09
:10C7780009D043B14FF6FF7300930520DC21324600
:10C788000023FFF70DFB41B0BDEC068BBDE8F08F31
:10C7980018260020302C0020000059400000694075
:10C7A800900D0020F83700209C3A0020242C00200F
:10C7B80010B54FF4C770FAF79DFFDB2805D14FF489
:10C7C800C870FAF797FF84B219E041F2E1042146F4
:10C7D80044F20100FAF780FF44F20100FAF78AFFF9
:10C7E800A04214BF80244FF4007421B24FF4C870E3
:10C7F800FAF772FF4FF4C770DB21FAF76DFF204696
:10C8080010BD024B00221A60704700BF043600209A
:10C8180070EEA10A88B030EE010A08B0704770EED9
:10C82800E10A88B030EE410A08B07047F0EE407A6D
:10C8380020EEA10A60EE810A47EEA10A88B017EE41
:10C84800810A08B07047D0B561EEA17A41EE017A4D
:10C858002DED048B17EE900A88B0B0EE409AF0EEFA
:10C86800609AF0EE418AB0EE618A05F045FA00223E
:10C87800002306460F4605F0FBFCE8B969EE887A06
:10C8880049EE287A29EE088A17EE900A05F034FA5C
:10C8980032463B4605F0AEFB19EEA88A05F062FD6C
:10C8A800044618EE100A05F027FA32463B4605F012
:10C8B800A1FB05F057FD01E00448044600EE900A8C
:10C8C80000EE104A08B0BDEC048BD0BD0050C34741
:10C8D800F0B58D4B2DED068B93ED001AD3ED011AB3
:10C8E8008FB0F0EE408AB0EE608A8DED060ACDED8D
:10C8F800070A30EE410A70EEE10A38EE811A78EE46
:10C90800211A8DED0C1ACDED0D1A8DED0A0ACDED1B
:10C918000B0AFFF798FF8DED040ACDED050A04AA6E
:10C9280092E8030008AB83E80300DDED099A9DED6A
:10C9380008AA69EEA97A4AEE0A7A17EE900A05F073
:10C94800DBF941EC100B07F0FDFC51EC100B05F086
:10C9580009FD09EE100A19EE900A05F0CDF9044612
:10C968001AEE100A0D4605F0C7F945EC104B41ECDC
:10C97800110B07F0D9FB51EC100B05F0F3FC68EE36
:10C98800087A48EEA87AB1EE48AAC8EEA79A5F4B93
:10C998005F4D5A691B8B6860EA612B8404468AEEF6
:10C9A80027AA85ED009A19EE100AC5ED028A85EDD1
:10C9B800038AC5ED049A85ED05AA05F09DF94CA3F7
:10C9C800D3E9002305F07CFCDFED527A002818BF7C
:10C9D800B0EE679AB7EE007A79EE077A37EE497AC1
:10C9E8004D4BC7EE877A1B78033BC5ED067A042BBF
:10C9F80071D8DFE803F0032738664F0018EE100AF5
:10CA080005F07AF9044618EE900A0D4605F074F917
:10CA180006460F4647EC116B45EC104B07F084FBBC
:10CA280035A3D3E9002351EC100BCDE9004505F0FF
:10CA3800B7F93246CDE902013B463849384809F092
:10CA4800D1FF48E019EE900A05F056F904461AEEAF
:10CA5800100A0D4605F050F92246CDE900012B4693
:10CA68002F4830492AE019EE100A05F045F941EC43
:10CA7800100B07F0E1FB00222B4B51EC100B05F0DB
:10CA88008FF905F06FFC05F037F902460B4624488C
:10CA980026491EE019EE100A05F02EF90646204632
:10CAA8000F4605F029F916A3D3E9002305F078F914
:10CAB800CDE900011A481E4932463B4609F092FF6B
:10CAC80009E017EE900A05F017F902460B461448DC
:10CAD800184909F087FF124C00230220CA21224678
:10CAE800F9F7E2F9002323700FB0BDEC068BF0BD17
:10CAF800AE47E17A14AEEF3F6666666666A64C40BE
:10CB0800F6285C8FC2A54C402C360020BC3700208C
:10CB1800AC390020A4707D3F242C002025AB0508EB
:10CB2800C83500203FAB0508000034C04FAB0508EE
:10CB380061AB05087DAB050800B560EEA07A40EE54
:10CB4800007A2DED028B17EE900A87B0B0EE408A7E
:10CB5800F0EE608A8DED020ACDED030A05F0CCF8FF
:10CB680041EC100B07F0EEFB51EC100B05F0FAFB53
:10CB7800DFED117A07EE100A78EEA78A38EE078AF9
:10CB880068EEA87A48EE087AC7EE277A17EE900A78
:10CB980005F0B2F841EC100B07F0D4FB51EC100B88
:10CBA80005F0E0FB00EE900A20EE880A60EEA80A85
:10CBB80007B0BDEC028B00BD00000000F0B52DED04
:10CBC800028BDFED3A1A3A4B8DB030EEA17AF0EED7
:10CBD800407AB7EE001A8DED020A83ED001A30EEA6
:10CBE800010AC3ED011A31EE671A71EEE01ACDEDB4
:10CBF800030AF0EE470A8DED077A8DED081ACDEDA0
:10CC0800091A8DED060AFFF71EFE8DED000ACDED1F
:10CC1800010A9DE8030004AB83E803009DED058A43
:10CC2800DDED048A68EE087A48EEA87A17EE900AD5
:10CC380005F062F841EC100B07F084FB18EE100ABF
:10CC480057EC106B05F058F8044618EE900A0D469C
:10CC580005F052F845EC104B41EC110B07F064FA63
:10CC68003946304655EC104B05F07CFB05F044F88E
:10CC780041EC100B07F05AFA002251EC100B0D4B47
:10CC880005F08EF805F06EFB29460646204605F0AD
:10CC980069FB00EE900AF6EE007A60EEA70A00EE55
:10CCA800106A0DB0BDEC028BF0BD00BF00000000A3
:10CCB800043A00200000E03FF0EE407A86B020EE13
:10CCC800200A67EE810A06B070472DE9F04F2DED76
:10CCD800028B85B0FCF72AF910EE105AFCF72CF9F4
:10CCE800284610EE104A05F007F880462046894687
:10CCF80005F002F841EC100B41EC180B07F0B8F8FE
:10CD080057EC106BB0EE480AF0EE680A07F0B0F97D
:10CD180032463B46404649465BEC10AB05F040F8CE
:10CD280005F020FB9FED138A07EE100ADFED127A5B
:10CD380057EE087A114C5B46C4ED007A52464046DD
:10CD4800494605F02DF805F00DFB07EE900A27EE91
:10CD5800888A04AB84ED018A94E8030003E90300A0
:10CD6800DDED030A9DED020A05B0BDEC028BBDE8BE
:10CD7800F08F00BF0000F04200008C42943A00207F
:10CD880030B53F4B2DED088BD3ED008AD3ED019ADA
:10CD98003C4BD3ED00AAD3ED01BA3B4B93ED008A8F
:10CDA80093ED019A394B93ED00AA93ED01BA38EE51
:10CDB800EA0A79EEEB0A38EE4A1A79EE4B1A93B082
:10CDC8008DED0A0ACDED0B0A8DED0C1ACDED0D1A7D
:10CDD800FFF72CFD8DED000ACDED010A9DE803005B
:10CDE8003AEE6A0A7BEE6B0A04AB38EE681A79EE03
:10CDF800691A83E803008DED081ACDED091A8DED47
:10CE08000E0ACDED0F0AFFF711FD8DED000ACDEDED
:10CE1800010A9DE8030006AB83E803009DED040AC0
:10CE2800DDED050A9DED061ADDED071AFFF70BFD8E
:10CE38008DED000ACDED010A9DE8030002AD85E8FD
:10CE48000300134B9DED021A93ED000AD3ED010A7E
:10CE5800DDED031AFFF7EAFC8DED000ACDED010ABE
:10CE68009DE8030012AB03E903006C46DDED110AEF
:10CE780085E803009DED100A13B0BDEC088B30BDAA
:10CE8800C035002018360020883A0020183A0020C3
:10CE9800E0370020F7EE007A77EEC07A20EE022A1B
:10CEA80020EE210A07EEA00AF0EE420A47EE810AB8
:10CEB80088B008B070472DE9F0432DED028B924BF6
:10CEC8001B78012B89B08146884646D14FEAC009B4
:10CED80001291FFA89F92BD809F58065A8B2FAF754
:10CEE8004DFC8A4C0435A8B284ED000AFAF746FCDA
:10CEF80009F58645A8B284ED010AFAF73FFC844C8F
:10CF0800043584ED000AA8B2FAF738FCA9F5FC400C
:10CF180084ED010A80B2FAF731FC7E4CA9F5FA409B
:10CF2800FC3884ED000A80B2FAF728FC84ED010A87
:10CF380008F1FF385FFA88F8B8F1010F00F2DF80D6
:10CF4800A9F57C5080B2FAF719FC734CA9F57A5907
:10CF580084ED000AA9F17C09CBE0022B40F0CF80D8
:10CF68006E4B6F4A1B68012992ED007A00F2AC8083
:10CF780007EE900AF8EE676A07EE903A46EE877A6F
:10CF8800BDEEE77A17EE104AA4B207EE104A04F194
:10CF98008005ED00B8EE478AADB2284637EEC88A5C
:10CFA800FAF7ECFB0435A8B204F50665EE008DED42
:10CFB800020AFAF7E3FBB6B230468DED030AFAF738
:10CFC800DDFB043604F58257B0B28DED040AFE008D
:10CFD800FAF7D4FBB6B230468DED050AFAF7CEFB68
:10CFE8000436B0B281348DED060AE400FAF7C6FBC8
:10CFF800A4B220468DED070AFAF7C0FB434E04346D
:10D00800A0B286ED000AFAF7B9FB6C1CE400A4B2E2
:10D01800204686ED010AFAF7B1FB3D4D0434A0B273
:10D0280085ED000AFAF7AAFB7C1CE400A4B22046AE
:10D0380085ED010AFAF7A2FB364F0434A0B287ED5A
:10D04800000AFAF79BFBD6ED001A96ED012ADDEDF2
:10D05800020AF0EE408A87ED010A9DED031AB0EE50
:10D06800480AFFF717FF8DED000ACDED010A9DE88C
:10D078000300D5ED001A95ED012AB0EE480ADDED62
:10D08800040A86E803009DED051AFFF703FF8DEDFE
:10D09800000ACDED010A9DE80300D7ED001A85E8E6
:10D0A8000300B0EE480ADDED060A9DED071AB0EE62
:10D0B800682AFFF7EFFE8DED000ACDED010A9DE825
:10D0C800030087E803006C4608F1FF385FFA88F828
:10D0D800B8F1010F13D809F5C1594FEAC9091FFA68
:10D0E80089F94846FAF74AFB0B4C84ED000A09F126
:10D0F80004091FFA89F0FAF741FB84ED010A09B027
:10D10800BDEC028BBDE8F083B5010020883A002011
:10D1180018360020183A0020C0350020A02500202D
:10D12800D82500202DE9F04F2DED048B734BC7B0A7
:10D1380005464FF476701C78FAF7DCFA06464FF489
:10D148007570FAF7D7FA07464FF47470FAF7FAFAD7
:10D15800012C14BF10240024C0B2032D1D9040F0F0
:10D16800A080674A674924A809F03CFCC1B224A8FA
:10D17800FDF7E4FC33463A46634924A809F032FC3B
:10D18800C1B224A8FDF7DAFC604A5E4924A809F078
:10D1980029FCC1B224A8FDF7D1FC002C14BFD8206B
:10D1A800C820FAF7CFFA0746002C14BFDC20CC20A1
:10D1B800FAF7C8FA0646002C14BFE020D020FAF788
:10D1C800C1FA8046002C14BFE420D420FAF7BAFA3A
:10D1D800F31B06EE903AB8EEE67A06EE908AF8EE81
:10D1E800E67A3346C7EE277A3A4601904849CDF8A1
:10D1F800008024A8FDEEE77ACDED027A09F0F2FB73
:10D20800C1B224A8FDF79AFC424A3E4924A809F075
:10D21800E9FBC1B224A8FDF791FCE820FAF792FADD
:10D228000746EC20FAF78EFA0646F020FAF78AFA53
:10D238008046F420FAF786FAF31B07EE903A06EEDA
:10D24800908AB8EEE77AF8EEE67A3A46C7EE277A99
:10D2580001902F49CDF80080334624A8FDEEE77AE7
:10D26800CDED027A09F0BEFBC1B224A8FDF766FC39
:10D278001D9A022A08D124A8274909F0DBFB24A813
:10D288001421FDF75BFC29E11D9B012B40F0228155
:10D2980024A8224909F0CEFB24A81021FDF74EFC52
:10D2A80003E01D9A012A40F01581002C14BFD820F4
:10D2B800C820FAF747FA1B90002C14BFDC20CC20BA
:10D2C800FAF740FA0646002C14BFE020D020FAF7FF
:10D2D80039FA1B9B1C90F61A06EE906AB8EEE67AAD
:10D2E80006EE900AF8EEE67A1026C7EE277A0024B2
:10D2F800FDEEE77ACDED1F7AE7E000BFF40D0020E0
:10D308008DAB050888AB050897AB0508A4AB0508E5
:10D31800AAAB0508F4AB0508FAAB05080FAC05087D
:10D328001C9B1B9A2046012103FB042AFFF7C3FD1F
:10D33800944B954A18681768D3ED018A92ED019AC3
:10D34800924B934AD3F80090D3ED019A1368012DBC
:10D35800209392ED018A7ED1F5EEC08AF1EE10FAA3
:10D3680054BF4FF0000C4FF0010CB5EEC09ABCF161
:10D37800000F0CBF4FF02B084FF02D08F1EE10FAFC
:10D3880054BF4FF0000E4FF0010EF5EEC09ABEF1FB
:10D39800000F0CBF2B262D26F1EE10FA54BF0021EA
:10D3A8000121B5EEC08A00290CBF4FF02B0B4FF0BE
:10D3B8002D0BF1EE10FA54BF00220122002A0CBFF7
:10D3C8002B232D231E93BCF1000F01D0F1EE688AA8
:10D3D800BEF1000F01D0B1EE499A09B1F1EE699A98
:10D3E8000AB1B1EE488A04F087FCCDE9000118EED5
:10D3F800900ACDF8088004F07FFCCDE90401384696
:10D4080004F07AFCCDE9060119EE100A089604F03A
:10D4180073FCCDE90A01484604F06EFCCDE90C0125
:10D4280019EE900ACDF838B004F066FCCDE9100189
:10D43800209804F061FC1E9ACDE9120118EE100A3A
:10D44800149204F059FC5246CDE9160124A851491A
:10D4580009F0C8FA2FE0022D2ED1FFF791FC8DEDCF
:10D46800220ACDED230A22AB93E8030046AB03E979
:10D478000300DDED457AF5EEC07AF1EE10FA449836
:10D4880005D5F1EE677A17EE906A2D2702E017EEC0
:10D49800906A2B2704F030FC02460B463046CDE953
:10D4A8000023029704F028FC5246CDE9040124A881
:10D4B800394909F097FAC6B224A83146FDF73EFB70
:10D4C8000120FEF74BF80134A4B21F9BA342BFF61C
:10D4D80027AF70E11D9A022A40F06D81E820FAF723
:10D4E80031F91B90EC20FAF72DF90646F020FAF7EF
:10D4F80029F91B9B1C9006EE900AF61AB8EEE68AEC
:10D5080006EE906AF8EEE67A002C14BFD820C82000
:10D51800C7EE887AFDEEE77ACDED1E7AFAF712F9B2
:10D528000646002C14BFDC20CC20FAF70BF907467E
:10D53800002C14BFE020D020FAF704F9BF1B07EE37
:10D54800100A06EE907AF8EEC77AB8EEE67A1B9AD9
:10D558001F9087EE277A931B012D06EE903ABDEEB9
:10D56800C77A88EE278A0D4B8DED207AB8EEE67AD9
:10D5780087EE277A83ED007A094B83ED008A40F025
:10D58800D0808FE0883A002018360020183A002012
:10D59800C035002020AC05085BAC0508A02500209C
:10D5A800D82500201F9A002102FB04622046219200
:10D5B800FFF781FC95ED018AD8ED018AB5EEC08AA6
:10D5C800F1EE10FA54BF4FF0000C4FF0010CF5EEDD
:10D5D800C08A9AED019ABCF1000F0CBF2B272D27AA
:10D5E800F1EE10FA54BF4FF0000E4FF0010EB5EEF9
:10D5F800C09ABEF1000F0CBF4FF02B0B4FF02D0B54
:10D60800F1EE10FA54BF002101212868D8F80090E3
:10D61800DAF8003000290CBF2B222D22BCF1000FB4
:10D6280001D0B1EE488ABEF1000F01D0F1EE688A50
:10D6380009B1B1EE499A19921A9304F05DFBCDE94C
:10D64800000118EE100A029704F056FBCDE9040118
:10D65800484604F051FBCDE9060118EE900ACDF8D2
:10D6680020B004F049FB1A9BCDE90A01184604F0E2
:10D6780043FB199ACDE90C0119EE100A0E9204F039
:10D688003BFB219ACDE910014F4924A809F0AAF9DA
:10D69800C1B224A8FDF752FA01340120FDF75EFF5C
:10D6A800A4B205E0494DDFF83481DFF834A1002445
:10D6B800209BA342BFF676AF0024454D2DE01C9B6E
:10D6C8001B9A2046022103FB0426FFF7F4FB95ED85
:10D6D800018AB5EEC08AF1EE10FA286803D5B1EEDA
:10D6E800488A2D2700E02B2704F006FBCDE900012E
:10D6F80018EE100A029704F0FFFA3246CDE9040149
:10D70800344924A809F06EF9C1B224A8FDF716FA25
:10D718000120FDF723FF0134A4B21E9BA342CEDAF9
:10D7280049E0022D43D046E01C9B1B9A012120466C
:10D7380003FB0425FFF7BFFBFFF722FB8DED220A51
:10D74800CDED230A22AB93E8030046AB03E90300BF
:10D75800DDED457AF5EEC07AF1EE10FA449806D57B
:10D76800F1EE677A17EE908A4FF02D0903E017EE75
:10D77800908A4FF02B0904F0BFFA06460F46404640
:10D78800CDE90067CDF8089004F0B6FA2A46CDE94D
:10D798000401104924A809F025F9C1B224A8FDF70D
:10D7A800CDF901340120FDF7D9FEA4B200E0002430
:10D7B8001E9BA342B8DA084B1D9A1A7047B0BDECFD
:10D7C800048BBDE8F08F00BF6FAC0508883A0020D5
:10D7D800C03500209DAC0508B50100201836002092
:10D7E800183A0020F0B52DED028B04468DB00028C4
:10D7F80000F0D480724B18890419A4B222B2002A0E
:10D8080005DB40F23F139A42C8BF1C4600E00024E3
:10D81800F7F7AEFBA0B24EF29C71F7F7BBFB684B73
:10D828001C81684B186804F067FA5FA3D3E90023EA
:10D8380004F0B6FA04F096FD634B1860634B1B784E
:10D848000A2B054624B23DD107EE104AF8EEC77AF6
:10D8580017EE900A04F050FA5D4B064618680F461A
:10D8680004F038FA02460B4651A1D1E9000104F050
:10D87800C1FB02460B463046394604F091FA06468B
:10D8880028460F4604F038FA02460B463046394619
:10D8980004F086FA00224F4B04F0ACFB04F062FD62
:10D8A80004F02AFA02460B4604A84B4909F09AF8F4
:10D8B8000020F8F7C1FA0520D72104AA0023F8F7B9
:10D8C800F3FA6BE0454B1888604304F003FA3AA377
:10D8D800D3E9002304F08EFB04F044FD404B08EE2E
:10D8E800100A1B68FCEEC87A07EE103A17EE905A39
:10D8F800F8EEC77A3B4B68EE277A1B68FDEEE77AAD
:10D90800ADB217EE906A28460121F618FFF7D3FA50
:10D91800FFF736FA8DED020ACDED030A02AC94E862
:10D92800030008AB83E80300681C80B20121FFF7FD
:10D93800C2FAFFF725FA8DED020ACDED030A94E845
:10D9480003000CAB07EE105A03E90300B8EEC70A50
:10D95800DDED080A38EE400A9DED091ADDED0A1AD8
:10D968009DED0B2AFFF796FA8DED020ACDED030A1D
:10D9780094E8030006AB83E803004FF6FF730093B7
:10D9880005200023DC213246FEF70AFA164B9DEDEE
:10D99800060A1878DDED070AFEF79AFF0DB0BDEC10
:10D9A800028BF0BDAFF300807B14AE47E17A843F71
:10D9B800000000A0D954BD410000000000F07340F1
:10D9C800900D0020080300207C3A0020A4250020A8
:10D9D800302C00200000F43FB0AC0508FC390020D2
:10D9E8000C2C002018260020242C00202DE9F843B8
:10D9F800461F8846B6B200250D4F12E008EB040119
:10DA080089B23046F7F768FA29F814000A20013479
:10DA1800FBF718F8062CF1D116350136F22DB6B2FF
:10DA280004D06FF0040407EB0509E7E7BDE8F883C5
:10DA3800383A00202DE9F04F85B00B1A0193431EA8
:10DA48009BB20293431C441F00F1060901F1FF3AFF
:10DA580001F1010B9BB20F461646A4B21FFA89F9D1
:10DA68001FFA8AFA1FFA8BFB039380462046514619
:10DA78003246F7F769FA204639463246F7F764FA2C
:10DA8800204659463246F7F75FFA019B0298E51897
:10DA9800ADB229463246F7F757FA4046294632468C
:10DAA800F7F752FA0134039829463246F7F74CFA49
:10DAB800A4B20A20FAF7C6FF4C45D7D105B0BDE895
:10DAC800F08F2DE9F843461F8846B6B200250E4F61
:10DAD80012E008EB040139F8142089B23046F7F750
:10DAE80033FA01340A20FAF7ADFF062CF1D11635C6
:10DAF8000136F22DB6B204D06FF0040407EB050925
:10DB0800E7E7BDE8F88300BF383A00202DE9F04385
:10DB18002DED068B70EE007A8DB017EE900AB0EE00
:10DB2800408A10EE904A20EE009A04F0E5F8064686
:10DB380020460F4604F0E0F8F7EE008A41EC100B9F
:10DB480041EC1A0B06F094F979EE287A55EC104B53
:10DB580017EE900A04F0D0F82246804689462B46F4
:10DB68003046394604F01CF902460B464046494601
:10DB780003F062FF04F0F6FBB0EE4A0AF0EE6A0A20
:10DB880009EE900A38EEC99ADFED377A89EE299ABC
:10DB980029EE279A06F06CFA304653EC102B3946DA
:10DBA80004F0FEF8044619EE900A0D4604F0A4F8B5
:10DBB80002460B462046294604F01CFA00222B4B4D
:10DBC80004F0EEF804F0CEFBB4EE688ADFED287AB4
:10DBD800284BF1EE10FA044619EE100A08BFB0EE11
:10DBE800678A1D6804F088F802460B4603A8224994
:10DBF80008F0F8FE204604F07FF802460B4606A817
:10DC08001E4908F0EFFE78EE287A38EEC88A87EECB
:10DC1800888A18EE100A04F06FF802460B4609A825
:10DC2800174908F0DFFE0520014603AA0023F8F78C
:10DC38003BF90520142106AA0023F8F735F9C82076
:10DC4800052109AA0023F8F72FF94FF6E07300938E
:10DC58000520DC212A460023FEF7A2F80DB0BDEC12
:10DC6800068BBDE8F08300BF000048420000494031
:10DC7800A4707D3FD8370020B9AC0508C1AC0508B1
:10DC8800C9AC05082DE9F04F494B2DED048B1D78E3
:10DC9800022D85B080467BD1464E348A012120462C
:10DCA800FFF709F9FFF76CF88DED000ACDED010AD1
:10DCB8009DE8030004AB03E9030028469DED020A32
:10DCC800DDED030AFEF704FE3B4B1A683B4B1B686D
:10DCD80002FB04343A4B1C603A4BDFED3B7A93ED80
:10DCE800008A68EE277A5F6817EE900A04F004F855
:10DCF800824638468B4603F0FFFF41EC100B41EC9F
:10DD0800190B06F0B5F8504653EC102B594604F0A1
:10DD180047F823A3D3E9002303F090FE04F002FBA5
:10DD2800B0EE490AF0EE690A054684B206F0A0F999
:10DD3800504653EC102B594604F032F80B46024675
:10DD480019A1D1E9000103F077FE04F0EBFAB37CE6
:10DD580081461FFA80FA1BB9B08AF18AFFF7B1FE33
:10DD6800002320465146B374FFF740FE2046514633
:10DD78001F22FFF75FFEB0EE480A00EE907AFFF729
:10DD8800C5FE338AB5829844A6F81080A6F8169086
:10DD980005B0BDEC048BBDE8F08F00BFAFF3008089
:10DDA8000000000000E063400000000000C05D408B
:10DDB800242C0020900D00200C2C00201826002078
:10DDC800D8370020AC3900200000C842124B1B781D
:10DDD800022B10B50CD1114B1B78022B08D1104C1B
:10DDE8002078C0B140B2FFF74DFF0023237010BD6B
:10DDF8000C4C237E23B99F20F7F794F80123237650
:10DE0800064B1B78022B06D1054C94F90000FFF74E
:10DE1800E9FC0023237010BD242C002004380020C6
:10DE2800591A0020900D0020034B00201860034B66
:10DE38001870FDF7B9BC00BF043600200438002074
:10DE4800034B00201860034B02221A70FDF7ACBC8C
:10DE5800043600200438002037B500242546A0B237
:10DE680028213223024601340095F7F76FFEB4F5F6
:10DE7800A07FF4D13EBD2DE9F04F2DED088B02288F
:10DE880097B080468DED070AB34B05D0032805D01F
:10DE9800012805D10C2202E0092200E00B221A70A9
:10DEA8001878F2F719FE042103914FF00009F3EEF8
:10DEB8000EAA9FEDAABADFEDAABA7DE1A94B1A68AE
:10DEC800A94B1B6802FB093307EE103A01211FFA20
:10DED80089F0B8EEC78AFEF7EEFFFEF751FF8DED29
:10DEE800080ACDED090A08AD95E803000AAB83E8F6
:10DEF80003009E4B1A6802EBC9030EAF19689C4BCE
:10DF080019600399521812685A60FEF739FF8DEDAF
:10DF1800080ACDED090A95E803000CAB83E8030075
:10DF2800DDED0A9A9DED0BAADDED0C8A9DED0D9AAB
:10DF3800B0EE690AF0EE4A0AB0EE681AF0EE491A35
:10DF4800FEF774FC8DED080ACDED090A95E803008B
:10DF5800B0EE691AF0EE4A1A87E80300B0EE680AD4
:10DF6800F0EE490AFEF76FFC8DED080ACDED090ABF
:10DF780095E8030010AB83E803009DED0E0ADDED84
:10DF88000F0AFEF7D9FD8DED080ACDED090A95E8CF
:10DF9800030016AA02E903009DED100ADDED110A3F
:10DFA800149EFEF7C9FD8DED080ACDED090A95E826
:10DFB800030087E80300DDED0F0AF5EEC00AF1EE75
:10DFC80010FA48BFF1EE600A9DED0E0ACDED0F0A7A
:10DFD800FEF7F4FD8DED080ACDED090A08AA92E8CE
:10DFE800030012AB83E803000798129D03F084FE38
:10DFF8005D4B139FD3F800B05E4BBDEEC87AD3F8E3
:10E0080000A0CDE9040117EE102A58465146FDF745
:10E018008DFD07EE10AAF8EEC77A07EE10BAB4EE37
:10E02800E78AF8EEC77AF1EE10FAB4EEE78A8CBF09
:10E0380000220122504B0690F1EE10FAD4BF0022C4
:10E0480002F00102B8F1020FDA6012D0B8F1030F42
:10E058003ED0B8F1010F68D1304603F04DFE36A32B
:10E06800D3E9002303F09CFE0022444B03F0E6FCB6
:10E078002AE0284603F040FEDDE9042304460D4665
:10E088002FA1D1E9000103F0B5FF02460B46204657
:10E09800294603F085FE2CA3D3E9002303F080FE74
:10E0A80004F060F907EE900AC7EEAA7A17EE900A14
:10E0B80003F022FE41EC100B06F0BEF8002251ECF2
:10E0C800100B2F4B03F06CFE04F004F904462CE00F
:10E0D80018EE100A03F010FE044638460D4603F009
:10E0E8000BFE17A3D3E9002303F05AFEDDE904234E
:10E0F80003F080FF04F036F903F0FEFD14A3D3E922
:10E10800002303F04DFE02460B462046294603F045
:10E1180071FF04F027F907EE900AB0EE6B7A07EE6C
:10E128008B7AFDEEC77A17EE904A002C2ADBC72CB3
:10E13800A8BFC72427E000BF8716D9CEF753F5BF7D
:10E148008FC2F5285CAF434000000000009070408B
:10E1580000000080DBC48641242C00200000C8C3D6
:10E168000000C8430C2C002018260020F0350020A1
:10E17800C0350020302C0020900D002000006940A0
:10E18800000049C00024114BDB685BB1104B1888B4
:10E19800104B1988069B4FF6FF759AB2A3B20095EB
:10E1A800F7F7D4FC0B4B039A1C600699084B08320E
:10E1B800196009F101090392074B1B884B45BFF60B
:10E1C8007DAE17B0BDEC088BBDE8F08F900D002038
:10E1D800F83700209C3A0020FC3900202DE9F04354
:10E1E8002D4B85B01878F2F777FC2C4B0B221A7060
:10E1F8002B4B1C782B4B1B78012C14BF10240024AC
:10E20800012B0BD1002C14BFD820C820F9F79AFA9B
:10E218000646002C14BFE020D02004E0E820F9F7DF
:10E2280091FA0646F020F9F78DFA00240746DFF840
:10E2380084901D4DDFF8808020E007FB04632046B2
:10E2480001216B61A8F82040FEF735FEFEF798FD26
:10E258008DED000ACDED010A9DE8030004AB03E94A
:10E2680003000D4B9DED020A1878DDED030AFEF759
:10E278002FFB6869FDF73EFE0134A4B2B9F80030FF
:10E28800A342DADA094B02221A70094B00221A76E5
:10E2980005B0BDE8F08300BF242C0020A425002091
:10E2A800F40D0020B5010020BC3700200438002000
:10E2B800900D0020FC390020AC3900207FB5FDF717
:10E2C8008BF8274A274B1168526819605A60264C08
:10E2D800264B22681B68264DD31A06EE903AB8EEF4
:10E2E800E67AD5ED006AF8EEE67A0021C7EE277ADD
:10E2F800FCEEE77A17EE906AB0B2FEF7DCFDFEF7A7
:10E308003FFD8DED000ACDED010A9DE8030004AB49
:10E3180003E90300174B9DED020A1878DDED030AA7
:10E32800FEF7D6FA144B1868144B1B6836B200FB7C
:10E338000630FDF7DFFD124B226893F900102868BC
:10E3480000FB01200F4A126890421C4605DCFAF7D0
:10E3580071FF0D4B1868FDF701F9002323707FBD8D
:10E36800BC370020C0350020F835002010260020DA
:10E378009C250020242C00200C2C0020182600208E
:10E38800C325002000260020C825002008B5FFF777
:10E3980095FF0C4B1A680C4B1B689A4210DB4FF028
:10E3A8008040002102F057FD084B1868FAF742FF39
:10E3B800074B02221A70074A00231370064A137685
:10E3C80008BD00BFF83500200026002010260020D8
:10E3D80004380020C3250020900D002010B500212E
:10E3E8004FF0804002F037FD0A4B00241C700A4BA6
:10E3F80020461C70F7F74AFC084B1868FAF71AFF12
:10E40800074B084801221A70074B1C70BDE81040E2
:10E41800F3F793BAC3250020083600201026002001
:10E42800242C0020D4170020A425002007EE100A71
:10E43800034BF8EE477A0022C3ED007A5A60704722
:10E448002C36002007EE100A034BF8EE477A00221C
:10E45800C3ED007A5A607047E03700200F4B10492F
:10E468001A68104B1B68D31A06EE903A0E4B1B68BD
:10E47800B8EEE67A06EE903AF8EEE67AC7EE277A34
:10E48800FCEEE77A17EE903A9AB20B80074B1888A1
:10E4980090422CBF00200120704700BF302C002084
:10E4A800FC390020182600200C2C002014260020FF
:10E4B80013B502AB011D23ED010A054A89B213F811
:10E4C800014B1454013080B28842F8D11CBD00BF02
:10E4D8003A3700202DE9F8431F4F0740002F044624
:10E4E8000D4603DA013F67F00F070137BFB2DFF8C7
:10E4F80074804FEAC7091FFA89F9484698ED000A5F
:10E5080009F10409FFF7D4FF1FFA89F098ED010A11
:10E51800FFF7CEFF114B10261B8894FBF6F6F60189
:10E528009C42B6B20CD1701980B20D498022FAF71C
:10E5380029FB00B1FEE721B24FF47F70F9F7CCF860
:10E548000F2F07D17519A8B205498022FAF71AFBCF
:10E5580000B1FEE7BDE8F8830F000080FC39002019
:10E568003A370020BC3700202DE9F043744B2DEDDD
:10E57800028B1888FF2898BF4FF4807093B0C000B2
:10E5880007F0BEFE6F4B0546186028B90520B42178
:10E598006D4A2B46F7F788FC0024694F6B4E4FF005
:10E5A80000086AE0FCF718FF20464FF44141FFF7E6
:10E5B80091FF674B1A685B683260002173602046E0
:10E5C800FEF779FCFEF7DCFB8DED020ACDED030AC0
:10E5D8000DF1080999E803000AAB83E803005D4BD5
:10E5E8009DED0A1A93ED007AD3ED017ADDED0B1A51
:10E5F80031EE470A71EEE70A31EE071A71EEA71AF3
:10E608008DED0E0ACDED0F0A8DED101ACDED111A14
:10E61800FEF719F98DED020ACDED030A99E803001A
:10E628000CAB83E80300FF2C4FEAC4032B4404D946
:10E63800C3F80080C3F8048003E00C9A1A600D9AAE
:10E648005A603B8840F23F10604390FBF3F080B281
:10E658004FF4FC630246282100933223F7F776FA39
:10E668003D4B18683D4B1B68C018FAF7E3FD3C4B5F
:10E678001868FCF773FF0134A4B23B88A34291DA0F
:10E68800012213464FF4807105A804F0E5FE354ECB
:10E69800DFF8F880294605A805F0C0F9082333708B
:10E6A800314B01241C700020F6F7BEFD2F48F3F70C
:10E6B80044F93078F2F710FA2D4B9FED2E8ADFEDF2
:10E6C8002E8A1C700024D5ED007AB0EE687A07EE29
:10E6D800C87A2046FCEEC77A17EE906A03F0FAFA79
:10E6E800264B002203F05CFB03F01CFEB6B2A3B27B
:10E6F800C72E28BFC72687B253B1214BB8F80000F0
:10E7080019884FF6FF7300933A463346F7F71EFA17
:10E718001B4BC8F8007001340835B4F5807F1E60C3
:10E72800D1D1184B1868FAF785FD114B02221A70DF
:10E73800154B00221A7613B0BDEC028BBDE8F083AE
:10E74800FC390020F0350020BEA40508C0350020A3
:10E75800BC3700202C360020F83500209C250020EE
:10E76800C8250020242C0020510D0020301700203F
:10E7780004380020000016430000C8420000F43F9F
:10E788009C3A002010260020900D0020F837002029
:10E79800F0B5294B294F2A4D2A4E012285B01A700F
:10E7A80000243AE0284B1A68336802FB04336B6193
:10E7B800264B1C84FCF710FE20464FF44141FFF71E
:10E7C80089FE234B2A681A606A6820465A6000212D
:10E7D800FEF771FBFEF7D4FA8DED000ACDED010AC4
:10E7E8009DE8030004AB03E903001A4B9DED020A00
:10E7F8001878DDED030AFEF76BF86869FDF77AFB18
:10E80800154B1868154B1B68C018FAF713FD144B05
:10E818001868FCF7A3FE0134A4B23B88A342C1DA0E
:10E82800104B1868FAF706FD034B02221A700E4BBC
:10E8380000221A7605B0F0BD04380020FC3900200B
:10E84800BC370020182600200C2C0020AC390020F2
:10E85800C0350020242C0020F83500209C250020FD
:10E86800C825002010260020900D002038B5FDF79F
:10E87800F9F9124B124D9F221A81124B0124187874
:10E888002C70F2F729F9104B00221A600F4B1B78F5
:10E89800072B04D00B2B0DD0062B0ED102E0BDE8C0
:10E8A800384075E74FF0804021462C70BDE838406D
:10E8B80002F0D1BABDE8384090E438BD900D002090
:10E8C80004380020242C002004360020A425002031
:10E8D8002DE9F743002581462C46154E154FDFF8E4
:10E8E8005C801FE0FCF778FD49462046FFF7F2FD03
:10E8F800D8F800303868C018FAF79CFC0E4B186836
:10E90800FCF72CFE308895FBF0F080B24FF4FC63E6
:10E918000093282102463223F7F718F905F59E756A
:10E92800013403353388A342DCDABDE8FE8300BF37
:10E93800FC390020F8350020C82500209C2500203F
:10E9480010B5104C4FF47570B4F90010F8F7C4FE08
:10E958000D4B4FF47670B3F90010F8F7BDFE40F296
:10E96800D230F8F7C7FEB02804D040F2D230B02138
:10E97800F8F7B2FE2088FFF759FD034B1888BDE869
:10E9880010405FE5B0010020AC01002000210A2200
:10E9980008B509F077F9D0F1010038BF002008BDAB
:10E9A80073B5041D0E46A4B20C2200234FF6E07581
:10E9B800204601360095F7F76DF900230C22B1B215
:10E9C80020460095F7F766F90D4B1B78012B16D1F9
:10E9D8000C4E0D4D308829880024043080B20C225A
:10E9E80023460094F7F756F93088298800940430B4
:10E9F800013180B289B20C222346F7F74BF97CBD6E
:10EA0800E43500202A360020DC37002008B54FF610
:10EA1800FF70F7F70FF90020F7F70EFAE12023212E
:10EA28002C4A0023F7F740FAE1204621294A00231F
:10EA3800F7F73AFAE1206921264A0023F7F734FA72
:10EA4800E1208C21244A0023F7F72EFA2348FFF708
:10EA58009DFF20B121482249012207F0C3FF4B2026
:10EA680023211E4A0023F7F71FFA1E48FFF78EFFDF
:10EA780020B11C481A49012207F0B4FF4B20462157
:10EA8800184A0023F7F710FA1748FFF77FFF20B15D
:10EA980015481349012207F0A5FF4B206921124AA6
:10EAA8000023F7F701FA1148FFF770FF20B10F486C
:10EAB8000B49012207F096FF4B208C2100230B4ABB
:10EAC800F7F7F2F90A4B18880A4B1988BDE808408D
:10EAD80066E700BFCEA20508D5AC0508E0250020F2
:10EAE80056A0050804260020162C0020CC2500205E
:10EAF800143A0020DC39002070B5044600200D4689
:10EB08001646F7F799F90020F7F7AAF84FF4FC60D2
:10EB1800F7F790F82046294656BB1E4A3346F7F7C2
:10EB2800C3F91D48FFF732FF20B11B481B490122DA
:10EB380007F058FF04F17006B6B230462946164A67
:10EB48000023F7F7B1F91648FFF720FF20B1144862
:10EB58001249012207F046FF3235ADB22046294658
:10EB6800104A0023F7F7A0F9304629460C4A07E077
:10EB78000D4A0023F7F798F932350B4AA9B2204617
:10EB88000023F7F791F9094B1888094B1988BDE854
:10EB9800704005E7DAAC0508803A002069A405084A
:10EBA800F0390020E2AC050809A50508143A002050
:10EBB800DC39002030B5144D9DF80C402C70134DF5
:10EBC8002880134D02FB04002980124D80B2288052
:10EBD800114D2980114D2A80114A1380114B18803C
:10EBE800114B1980114B1249E2B21A7000230B70B5
:10EBF80010490A709DF810200134013254430E4A1E
:10EC080014700E4A137030BD983B0020783A0020EB
:10EC1800BA370020143A0020DC39002038370020A9
:10EC2800A43A00202A360020DC370020DE390020F4
:10EC380009360020163A0020E5350020E43500208A
:10EC480038B5054600200C46F7F7F6F80020F7F728
:10EC580007F84FF4FC60F6F7EDFF0B48FFF796FE58
:10EC680028B1094809490A4B002207F0BBFE28468B
:10EC780021460023044AF7F717F9064B1888064B74
:10EC88001988BDE838408BE62036002008A9050819
:10EC98000000F03F143A0020DC390020114B1B68BB
:10ECA800002B70B505460C4604DA5B420E480F4946
:10ECB8002D2202E00C480D49202207F093FE002087
:10ECC800F7F7BAF80020F6F7CBFF4FF4FC60F6F739
:10ECD800B1FF054A284621460023BDE87040F7F7F2
:10ECE800E3B800BF103A0020E8370020EAAC050876
:10ECF8000F4B10B519684FF4E170F8F70AFD40F2B0
:10ED08003D114FF4E070F8F7E7FC0020F7F794F8AE
:10ED18000020F6F7A5FF4FF4FC60F6F78BFF054AD5
:10ED2800192064210023BDE81040F7F7BDB800BFE3
:10ED3800103A0020F2AC050808B54FF4E070F8F777
:10ED4800D9FC40F23D13984205D14FF4E170BDE87B
:10ED58000840F8F7F7BC002008BD38B50546002084
:10ED68000C46F7F769F80020F6F77AFF4FF4FC60D5
:10ED7800F6F760FF0B48FFF709FE28B109480A4972
:10ED88000A4B002207F02EFE284621460023054A9A
:10ED9800F7F78AF8064B1888064B1988BDE83840FB
:10EDA800FEE500BFFC35002008A905080000F03F7B
:10EDB800143A0020DC39002038B5C501ADB2002472
:10EDC800601980B2F9F786FC0134C0B2FBF7A6FEE1
:10EDD800A4B24FF47A70F9F735FE802CF0D138BD23
:10EDE80073B5104D00240E20FBF798FE002609E0AD
:10EDF8000DF10700FBF7A3FE20B19DF80730AB55D6
:10EE08000136F6B23306F3D5E00180B20549802217
:10EE1800F9F7B8FE00B1FEE70134A4B2B4F5007FFB
:10EE2800E1D17CBD3A37002007EE100AF8EE477AA8
:10EE38007FB517EE900A02F05FFF02460B4601A865
:10EE4800054907F0CFFD0A20962101AA0023F7F70C
:10EE58002BF807B000BD00BFF9AC0508AFF3008080
:10EE68000EB403B070470A2810B5044602D10D202D
:10EE7800FFF7F9FF064A13681BB103F8014B13604B
:10EE880010BD044B1B680BB12046984710BD00BF4E
:10EE9800B00D00209C3B002010B5044601E0FFF7B0
:10EEA800E2FF14F8010B0028F9D110BD2DE9F04F4D
:10EEB800044685B00D464FF00A0A00E03546207832
:10EEC800002800F0C480252801D0013467E060786C
:10EED800302803D1A0780123033407E02D2802D07D
:10EEE8000234002302E0A078022303344FF0000824
:10EEF80005E00AFB080814F8010BA8F13008A0F196
:10EF08003002D2B2092AF4D96C2801D04C2803D196
:10EF180014F8010B43F00403002800F098806028DF
:10EF280086BFA0F12002D2B202464F2A3DD006D8B1
:10EF3800432A2DD0442A09D0422A30D133E0552A19
:10EF480004D0582A29D0532A29D101E00A272DE0D4
:10EF58002E1D2F68002500E001357A5D002AFBD1BF
:10EF680004E02020FFF77FFF4D4601E0980704D416
:10EF7800454505F10109F4D34D463846FFF78CFFA6
:10EF880003E02020FFF76FFF01354545F9D395E7EA
:10EF980028782E1DFFF767FF90E7102706E0FFF798
:10EFA80062FF2E468AE7022700E008272E1D442A22
:10EFB800296804D1002902DA494243F008030022F3
:10EFC80000E02A46B1FBF7FE07FB1E11CDB2092D62
:10EFD800714607D9782814BF4FF0070C4FF0270C5B
:10EFE8006544EDB230350DF80250551CBEF1000FE6
:10EFF80002D0102DE5D10F22190705D504A94D1906
:10F008002D2105F8101C951C13F0010F0CBF4FF0B3
:10F01800200B4FF0300B9B072F4604D508E05846CD
:10F02800FFF721FF4F46474507F10109F7D34F4640
:10F03800013D1DF80500FFF716FF002DF8D103E08C
:10F048002020FFF710FF01374745F9D336E705B011
:10F05800BDE8F08F70B5064D0C462E68286001E0BB
:10F06800FFF701FF14F8010B0028F9D12E6070BDDD
:10F078009C3B00200FB407B504A951F8040B01917B
:10F08800FFF714FFBDE80E4004B070470EB417B583
:10F0980005A9084C51F8043B206018460191FFF778
:10F0A80005FF2268002313702360BDE81E4003B0EB
:10F0B800704700BFB00D00200EB433B505A9074C4A
:10F0C80051F8043B2568206018460191FFF7EEFED1
:10F0D8002560BDE83C4003B0704700BF9C3B002062
:10F0E80070B51E4604461C481546FFF7C3FF022E9E
:10F0F8001FD0042E25D0012E2AD105E0A15D174886
:10F10800FFF7B8FF013600E00026AE42F6DB20200C
:10F11800FFF7A9FE002609E0A05DA0F12003DBB2FD
:10F128005E2B88BF2E20FFF79EFE0136AE42F3DB32
:10F138000EE034F8021B0A48FFF79CFF013DF8D1A6
:10F1480006E054F8041B0748FFF794FF013DF8D187
:10F158000A20BDE8704086E600AD050807AD050841
:10F168000DAD050813AD050808B501214FF48070F1
:10F1780001F07CFA4FF480700021BDE8084001F0EE
:10F1880075BA43680A6823F0407323F48073134305
:10F198000A7943EA02234360CA680B6930B51A4307
:10F1A80084688D68084B2A43234013434A7943EA0D
:10F1B800420383600B7DC26A013B22F47002DBB21A
:10F1C80042EA0353C36230BDFDF7FFC0002303606A
:10F1D800037143718360C360036101230375704742
:10F1E800074A084B516810B50B4090E812002143BC
:10F1F8008468C068214301430B43536010BD00BFBE
:10F2080000230140E030FCFF00230360436083607B
:10F21800C3607047836811B143F0010301E023F034
:10F22800010383607047436823F4400323F40073A9
:10F238000B4343607047416282627047436823F022
:10F248001F030B4343607047044B5A6810B142F4E4
:10F25800000201E022F400025A60704700230140D6
:10F26800044B5A6810B142F4800201E022F4800293
:10F278005A60704700230140092970B50CB20CD9B7
:10F2880004EB44041E3CC6680725A54026EA05058C
:10F29800A34045EA0304C4600AE0066904EB440499
:10F2A8000725A54026EA050513FA04F42C43046152
:10F2B800062A0CD80523013A5A43446B1F2393406E
:10F2C80024EA0303914043EA0102426370BD0C2A19
:10F2D80012B20CD802EB8202233A046B1F2393402C
:10F2E80024EA0303914043EA0102026370BD02EB82
:10F2F8008202413AC46A1F23934024EA03039140DF
:10F3080043EA0102C26270BD836843F080438360B0
:10F3180070478068C0F380507047836811B143F428
:10F32800806301E023F4806383607047836811B1D0
:10F3380043F0020301E023F002038360704743684F
:10F34800013923F4604343EA41334360704743681B
:10F3580011B143F4006301E023F400634360704794
:10F36800C06C80B27047014B186870470823014091
:10F37800836811B143F4807301E023F480738360E0
:10F388007047836811B143F4007301E023F40073FC
:10F3980083607047044B5A6810B142F4005201E090
:10F3A80022F400525A60704700230140092970B5C1
:10F3B8000CB20CD904EB44041E3CC6680725A540D2
:10F3C80026EA0505A34045EA0304C4600AE0066985
:10F3D80004EB44040725A54026EA050513FA04F4BE
:10F3E8002C430461836BC3F30154121B0232D2B263
:10F3F80002EB82021F24944023EA040391400B434A
:10F40800836370BD836B013923F4401343EA0153CE
:10F418008363704782B0002301930190019BCB184E
:10F428000193019B1A6002B07047836823F470232C
:10F438000B4383607047836823F440130B43836056
:10F448007047836843F48003836070478068C0F323
:10F4580080507047436811B143F4806301E023F49E
:10F46800806343607047436811B143F4805301E0FF
:10F4780023F480534360704782B0002301930190C6
:10F48800019B28335B180193019B186880B202B076
:10F4980070470123C9B213FA01F143680AB119434D
:10F4A80001E023EA010141607047036819420CBF7B
:10F4B800002001207047C943016070474368006815
:10F4C80010EA112007D00122C9B212FA01F119423B
:10F4D8000CBF0020012070476FEA112101607047BE
:10F4E800036823F001030360002303604360836023
:10F4F800C3600361212343612C4B98421CD02C4BE1
:10F50800984220D02B4B984225D02B4B98422AD09A
:10F518002A4B98422FD02A4B984233D0294B9842F5
:10F5280037D0294B984204D14FF03D5243F8AC2CC8
:10F538007047264B984203D13D2243F8082C704768
:10F54800234B984204D14FF4746243F8202C70473F
:10F55800204B984204D14FF4741243F8382C70476A
:10F568001D4B984204D14FF0746243F8502C7047F9
:10F578001A4B984203D11A4A43F8642C7047194B26
:10F58800984203D1184A43F87C2C7047174B98428D
:10F5980003D1174A43F8942C7047164B984204BF7E
:10F5A8004FF03D5243F8AC2C704700BF106002404A
:10F5B800286002404060024058600240706002408B
:10F5C80088600240A0600240B860024010640240B7
:10F5D800286402404064024058640240706402405B
:10F5E8003D00002088640240400F0020A0640240D3
:10F5F80000003D20B86402400268134B10B5134068
:10F60800CC680A6822434C6922438C692243CC693E
:10F6180022430C6A22434C6A22438C6A22434C6B75
:10F6280022438C6B22431343036042690C6BCB6A01
:10F6380022F007022343134343610B6943604B687D
:10F6480083608B68C36010BD3F801CF0002303609B
:10F6580043608360C360036143618361C361036284
:10F6680043628362C36203634363836370470368CF
:10F6780011B143F0010301E023F001030360704777
:10F68800036811B143F4004301E023F4004303602D
:10F698007047036811B143F0200301E023F0200311
:10F6A8000360704741607047406880B270470368E4
:10F6B80012B143F4002301E023F400230360016145
:10F6C8007047036811B143F4802301E023F48023D9
:10F6D800036070470AB101617047C16070470068F4
:10F6E800C0F3C0407047006800F0010070474069EF
:10F6F80000F0380070470A4A0A4B10B50A4CA0427D
:10F7080088BF13468A004CBF5B681B6821F0F02154
:10F7180021F0821119420CBF0020012010BD00BF4A
:10F7280000640240006002400F64024010B5084BBC
:10F73800084A094CA04288BF134611F0005F21F027
:10F74800F02121F0821114BFD960996010BD00BF6B
:10F7580000600240006402400F6402400B0607D5B7
:10F76800436912B143F0800301E023F08003436151
:10F77800802909D001F01E01036812B11943016004
:10F78800704723EA010101607047124B124A10B515
:10F79800124CA0428CBF14461C4621F0F02323F0E3
:10F7A800C3132BB1026802F01E0202EAD12202E062
:10F7B800426902F0800288004CBF6368236821F028
:10F7C800F02121F08210184002D0101C18BF01202F
:10F7D80010BD00BF00600240006402400F64024098
:10F7E80010B5084B084A094CA04288BF134611F0CF
:10F7F800005F21F0F02121F0821114BFD9609960D7
:10F8080010BD00BF00600240006402400F64024067
:10F81800044B00221A605A609A60DA60024A5A6100
:10F82800704700BF003C0140FFFF7F00837910B59F
:10F83800002B29D01A4B01681C68CA4314401C606D
:10F848005C6822405A60027902F1804202F59E32D9
:10F8580014682143116002689C68D1430C409C6085
:10F86800DC682140D9604179102906D19968114393
:10F878009960D9680A43DA6010BD01F1804303F545
:10F888009E3319680A4308E00379016803F180434D
:10F8980003F59E331A6822EA01021A6010BD00BF00
:10F8A800003C014000230C22036003714271837104
:10F8B8007047024B1A6902431A617047003C0140C5
:10F8C800034B5B6918420CBF00200120704700BF42
:10F8D800003C0140014B5861704700BF003C0140AB
:10F8E800054B1A685B69034004D010420CBF002026
:10F8F8000120704718467047003C0140014B586191
:10F90800704700BF003C01404FF0204318B943F254
:10F91800DB021A6003E043F2D20243F820204FF0E2
:10F928002042411C6FF0704342F8213002F5827288
:10F9380042F82030704770B584684568C368C16A6A
:10F94800026825431D4303691D4343691D438369B9
:10F958001D43C3691D43036A1D43436A1D43836AEC
:10F968001D43036B0D431D434FF02043082C43F800
:10F97800225005D153F8224044F0400443F8224075
:10F98800436B9E691D6835435E6845EA06159E68A7
:10F9980045EA0625DE6845EA06451E695B6945EACB
:10F9A8000655541C45EA03654FF02043B1F5804FD6
:10F9B80043F8245010D1836B98691968014358683B
:10F9C80041EA0011986841EA002118695B6941EA37
:10F9D800005141EA036101E06FF07041014B43F8C7
:10F9E800221070BD040100A0022242604FF4805230
:10F9F8004262416B4FF4005210B5826200230F221D
:10FA0800FF2403608360C360036143618361C36152
:10FA18000362C36203630A604A608C60CA600A6159
:10FA28004A618B61816B0A604A608C60CA600A61B6
:10FA38004A618B6110BD4FF0204321B153F820205B
:10FA480042F0010203E053F82010024A0A4043F84A
:10FA580020207047FEFF0F0010280CBF064B074BF5
:10FA68004FF040024FF0180119605A604FF0FC3215
:10FA78009A60DA60704700BF600000A0800000A0B4
:10FA880030B5836844681C43C36844F008041C43C9
:10FA980003691C43436944EA4324836944EA4334C1
:10FAA800C36999685A68090441EA02211A68DB683F
:10FAB800114341EA0361036A9A685D68120442EAE5
:10FAC80005221D68DB682A4342EA03620368102B9B
:10FAD8000CBF034B034B1C609960DA6030BD00BF5C
:10FAE800600000A0800000A010230360C26900230A
:10FAF80043608360C360036143618361FC231360D7
:10FB080053609360D360026A136053609360D3605C
:10FB1800704741B110280CBF074B084B1A6842F0D8
:10FB280004021A60704710280CBF034A034A044BAA
:10FB380011680B4013607047600000A0800000A0AF
:10FB4800FBFF0F0041B110280CBF084B084B1A6887
:10FB580042F040021A60704710280CBF034A044A5A
:10FB6800044B11680B401360704700BF600000A091
:10FB7800800000A0BFFF0F00102802D1024B586977
:10FB88007047024B58697047600000A0800000A0D1
:10FB9800054B18221A6000225A604FF0FC329A6016
:10FBA800DA601A61704700BFA00000A002684368CD
:10FBB80042F0100242EA4322836842EA4332144B7D
:10FBC80010B51A60C26891685468090441EA0421B2
:10FBD8001468D268214341EA02629A600269916816
:10FBE8005468090441EA04211468D268214341EAAF
:10FBF8000262DA60426991685068090441EA0021AA
:10FC08001068D268014341EA02621A6110BD00BF60
:10FC1800A00000A0C2680023036043608360FC2347
:10FC2800136053609360D3600269136053609360FC
:10FC3800D3604269136053609360D3607047054B8B
:10FC480018B11A6842F0040202E01968024A0A4030
:10FC58001A607047A00000A0FBFF0F0062B11028D7
:10FC680001D10E4B03E0B0F5807F03D10C4B5A68ED
:10FC7800114311E00B4BFAE7102804D1074B5A68DF
:10FC880022EA010108E0B0F5807F0CBF044B054B68
:10FC98005A686FEA0101114059607047600000A07E
:10FCA800800000A0A00000A0102801D1064B04E0AD
:10FCB800B0F5807F0CBF054B054B5B680B420CBF52
:10FCC80000200120704700BF600000A0800000A055
:10FCD800A00000A0102804D1074B5A6822EA0101AD
:10FCE80008E0B0F5807F0CBF044B054B5A686FEAFB
:10FCF8000101114059607047600000A0800000A019
:10FD0800A00000A0102801D1084B04E0B0F5807FC6
:10FD18000CBF074B074B5B6813EA010004D013EADA
:10FD2800D1010CBF00200120704700BF600000A077
:10FD3800800000A0A00000A0102804D1084B5A6839
:10FD480022EAD10109E0B0F5807F0CBF054B064BD4
:10FD58005A684FEAD10122EA01015960704700BF91
:10FD6800600000A0800000A0A00000A008B52C4BF7
:10FD7800984205D10120014600F048FC012048E0E6
:10FD8800284B984205D10220012100F03FFC0220B7
:10FD98003FE0254B984205D10420012100F036FCB4
:10FDA800042036E0214B984205D10820012100F0BB
:10FDB8002DFC08202DE01E4B984205D11020012172
:10FDC80000F024FC102024E01A4B984205D1202092
:10FDD800012100F01BFC20201BE0174B984205D1A5
:10FDE8004020012100F012FC402012E0134B984201
:10FDF80005D18020012100F009FC802009E0104B8A
:10FE080098420BD14FF48070012100F0FFFB4FF4B2
:10FE180080700021BDE8084000F0F8BB08BD00BFB5
:10FE2800000002400004024000080240000C0240AA
:10FE3800001002400014024000180240001C02405A
:10FE4800002002402DE9F0470023D1F800801A462F
:10FE58004FF0010C03270CFA02F404EA0805A54246
:10FE68002ED1066817FA03F4E443264006600E799B
:10FE7800D0F8009006FA03FA013E4AEA0909012E71
:10FE8800C0F8009014D8866891F8059026408660DE
:10FE9800866809FA03F949EA06068660466826EA8A
:10FEA800050545608D7946689540ADB23543456096
:10FEB800C5682C40C460CC79C5689C402C43C4609C
:10FEC80001320233102AC6D1BDE8F0874FF6FF731E
:10FED80003600023037143718371C371704782B05B
:10FEE8004FF480330193019B0B430193019BC36142
:10FEF800C161019BC361C3690193C369019302B0E6
:10FF08007047036919420CBF00200120704700693F
:10FF180080B27047436919420CBF00200120704726
:10FF2800406980B2704701837047418370470AB1C6
:10FF380001837047418370474161704743694B4073
:10FF48004361704701F00703C908083130B59B00C9
:10FF580050F821500F249C4025EA040440F8214021
:10FF680050F8214012FA03F31C4340F8214030BDF9
:10FF780008B5134B984207D14FF40010012100F047
:10FF880069FB4FF4001014E00E4B984207D14FF470
:10FF98008000012100F05EFB4FF4800009E00A4B6D
:10FFA80098420BD14FF40000012100F053FB4FF4AD
:10FFB80000000021BDE8084000F04CBB08BD00BFB0
:10FFC8000054004000580040005C00407FB50446E3
:10FFD800868868460D4600F06DFA02992C482B6811
:10FFE80026F03F063604B1FBF0F0360C80B206432B
:08FFF800A680228822F001021C
:020000040801F1
:100000001204120C2280254A93420AD85B00B1FBED
:10001000F3F301309BB280B22084032B98BF0423FA
:1000200021E0EE884BF6FF72964205D1032253433E
:10003000B1FBF3F39BB206E019225343B1FBF3F398
:100040009BB243F480431A054FF4967208BF43F005
:10005000010350434FF47A7290FBF2F0013080B20A
:1000600043F400432084A38323886989AA889BB230
:1000700043F001032380238823F4816323F00203E8
:100080001B040A431B0C13439BB223802A89AB89B0
:1000900013439BB223817FBD40420F00A086010025
:1000A00041F288330360002383804BF6FF720381A3
:1000B00043814FF48043C28083817047038819B124
:1000C0009BB243F0010303E023F001031B041B0C6C
:1000D00003807047038819B19BB243F4807303E037
:1000E00023F480731B041B0C03807047038819B131
:1000F0009BB243F4007303E023F400731B041B0C56
:100100000380704712B141F0010101E001F0FE01EE
:1001100001827047038819B19BB243F4806303E006
:1001200023F480631B041B0C0380704783899BB2FC
:1001300001F0FE0123F0FE030B43838170478389A6
:1001400019B19BB243F0010303E023F001031B0448
:100150001B0C83817047038819B19BB243F04003A5
:1001600003E023F040031B041B0C0380704703884B
:1001700029B16FEA43436FEA53439BB201E05B044A
:100180005B0C03807047038819B99BB243F080036E
:1001900003E023F080031B041B0C03807047B1F5C0
:1001A000804F838B04D023F480431B041B0C02E09C
:1001B0009BB243F4804383837047B1F5006F03889B
:1001C00003D19BB243F4006303E023F400631B04F8
:1001D0001B0C03807047B1F5005F038803D19BB20D
:1001E00043F4005303E023F400531B041B0C03806F
:1001F0007047038819B19BB243F0100303E023F06A
:1002000010031B041B0C0380704701827047008A97
:10021000C0B27047038819B19BB243F4805303E026
:1002200023F480531B041B0C03807047B1F5006F4F
:10023000038803D19BB243F4006303E023F400631B
:100240001B041B0C03807047038819B19BB243F059
:10025000200303E023F020031B041B0C03807047E2
:10026000008BC0F307207047838819B19BB243F419
:10027000006303E023F400631B041B0C83807047BE
:10028000838819B19BB243F4805303E023F4805375
:100290001B041B0C8380704782B0002301930190E4
:1002A000019BCB180193019B188880B202B0704764
:1002B00083889BB20AB1194301E023EA01018180DE
:1002C0007047838A008B9BB243EA0040084020F0CD
:1002D0007F40431A584240EB03007047838A008BEB
:1002E0009BB243EA004020F07F40704782B0002379
:1002F000009301930B0F01900093009B21F07F412D
:1003000013B1019B143302E0019B090C18330193D4
:10031000019B1B6819420CBF0020012002B07047EE
:10032000C94389B2818270478388808A80B208403D
:100330009BB206D001F0E06113EA11410CBF00202E
:1003400001207047C94389B2818270470A4B1A68FD
:1003500042F001021A6000229A60196821F084714B
:1003600021F48031196005495960196821F4802110
:100370001960DA60704700BF003802401030002476
:10038000024B00221A701870704700BF02380240FA
:10039000034B1A6822F0F80242EAC0021A60704762
:1003A00000380240014B1860704700BF0000474210
:1003B000064B002201281A701A7002D0042804D1BA
:1003C00001E01870704705221A70704770380240BB
:1003D000014B1860704700BF800E4742014341EA5D
:1003E000821200995B08013B42EA016141EA034144
:1003F000014B5960704700BF00380240014B186044
:10040000704700BF600047428001034B40EA017122
:10041000C3F88410704700BF00380240014B1860D9
:10042000704700BF68004742014B1860704700BF2B
:100430004C004742034B9A6822F0EC6202430A43A5
:100440009A60704700380240034B9A6822F0784265
:1004500002430A439A60704700380240034B9A688F
:1004600022F0030202439A60704700BF0038024046
:10047000024B986800F00C00704700BF0038024043
:10048000034B9A6822F0F00202439A60704700BF63
:1004900000380240034B9A6822F4E05202439A600B
:1004A000704700BF00380240034B9A6822F4604254
:1004B00042EAC0029A607047003802401E4B9A68B8
:1004C00002F00C02042A10B503D0082A03D01B4BFB
:1004D00018E01B4B16E059685A6811F4800F5968F0
:1004E00014BF174B154B02F03F02B3FBF2F3124A55
:1004F0005268C2F30142C1F3881101324B435200EA
:10050000B3FBF2F30C4903608B680E4A0468C3F333
:100510000313D35C34FA03F343608C68C4F382247E
:10052000145D33FA04F484608968C1F34231525C8B
:10053000D340C36010BD00BF003802400024F40067
:1005400000127A001003002000F44073B3F5407FDE
:10055000084B08D1996820F0704221F4F81122F478
:1005600040720A439A601A6F000542EA10501867F9
:10057000704700BF00380240014B1860704700BF51
:100580003C0E4742014B1860704700BF400E474287
:10059000014B1860704700BF5C014742044B1A6B67
:1005A00009B1104301E022EA00001863704700BF60
:1005B00000380240044B5A6B09B1104301E022EAB3
:1005C00000005863704700BF00380240044B9A6B2C
:1005D00009B1104301E022EA00009863704700BFB0
:1005E00000380240044B1A6C09B1104301E022EAC2
:1005F00000001864704700BF00380240044B5A6C7A
:1006000009B1104301E022EA00005864704700BFBE
:1006100000380240044B1A6909B1104301E022EA94
:1006200000001861704700BF00380240044B5A694F
:1006300009B1104301E022EA00005861704700BF91
:1006400000380240044B9A6909B1104301E022EAE4
:1006500000009861704700BF00380240044B1A6ADE
:1006600009B1104301E022EA00001862704700BFA0
:1006700000380240044B5A6A09B1104301E022EAF3
:1006800000005862704700BF00380240044B1A6DEA
:1006900009B1104301E022EA00001865704700BF6D
:1006A00000380240044B5A6D09B1104301E022EAC0
:1006B00000005865704700BF00380240044B9A6D37
:1006C00009B1104301E022EA00009865704700BFBD
:1006D00000380240044B1A6E09B1104301E022EACF
:1006E00000001866704700BF00380240044B5A6E85
:1006F00009B1104301E022EA00005866704700BFCC
:1007000000380240044B1A7809B1104301E022EA94
:1007100000001870704700BF0D3802404309012BDC
:10072000074A01D1136803E0022B0CBF136F536F0C
:1007300000F01F0033FA00F000F00100704700BF26
:100740000038024007B5002301933120FFF7E6FF90
:10075000019B01330193019BB3F5A06F01D00028E9
:10076000F3D03120FFF7DAFF003018BF01200EBDB3
:10077000024B5A6F42F080725A677047003802404D
:10078000034BDB6818420CBF00200120704700BFFC
:1007900000380240014B1870704700BF0E3802400D
:1007A00008B5154B98420BD101214FF48050FFF74B
:1007B00061FF4FF480500021BDE80840FFF75ABFA9
:1007C0000E4B984207D14FF480400121FFF746FFBE
:1007D0004FF4804009E00A4B98420BD14FF400409F
:1007E0000121FFF73BFF4FF400400021BDE8084026
:1007F000FFF734BF08BD00BF0030014000380040A3
:10080000003C00400B88028810B54C8823438C883C
:100810002343CC8823430C8923434C8923438C896D
:100820002343CC8902F44152234313439BB20380F8
:10083000838B23F400631B041B0C83830B8A0382CA
:1008400010BD838B23F47B6323F00F031B041B0C6D
:100850008383022303848B68F0B5858B022BADB2B2
:1008600038D0294A8E889468002E14BF02260126AB
:10087000240203D5946824F400049460D2F88440E0
:10088000D2F884705268DFF884C002F03F02BCFBEB
:10089000F2F2C4F388145443C7F30272B4FBF2F4C7
:1008A000CA88B2F5007F4FF00A0201D1240A02E0A3
:1008B0007601B4FBF6F46243B2FBF3F305330A228C
:1008C0009BB2B3FBF2F303F001021202C3F34F0336
:1008D00092B200E000229C1EA4B2FE2C28BF00228F
:1008E000CC8828BF0223134323439BB203840B8885
:1008F0004A882B4343F4006313438A8813438A894D
:1009000013439BB28383F0BD0038024000127A008B
:100910000023038043808380C380038143818381DC
:10092000C381072303827047002302220380438090
:100930008380C380826083817047038819B19BB232
:1009400043F0400303E023F040031B041B0C03802F
:100950007047838B19B19BB243F4806303E023F4A7
:1009600080631B041B0C83837047038823F400639C
:100970001B041B0C038003889BB20B43038070474E
:10098000B1F5804F038803D19BB243F4804303E069
:1009900023F480431B041B0C038070474FF6FF6356
:1009A0009942038803D09BB243F4807303E023F49D
:1009B00080731B041B0C03807047838819B19BB2A2
:1009C00043F0040303E023F004031B041B0C8380A7
:1009D0007047838819B19BB243F0100303E023F002
:1009E00010031B041B0C83807047838B23F47B63F1
:1009F00023F00F031B041B0C8383022303840B8847
:100A0000828BB3F5007F10B592B205D0002B0CBFDE
:100A10004FF48073002301E04FF480734C8822432D
:100A20008C88898942F4006222430A4392B21343BC
:100A3000838310BD808980B27047818170470388AD
:100A400019B19BB243F4005303E023F400531B0499
:100A50001B0C0380704703889BB243F480530380D0
:100A60007047012902D0008B80B27047808A80B223
:100A70007047008A80B2704783889BB20AB11943DD
:100A800001E023EA010181807047090901238B40BD
:100A90009BB21AB1828892B2134303E0828892B269
:100AA00022EA030383807047038919420CBF0020A8
:100AB00001207047C94389B20181704710B584880D
:100AC0000089012301F00F0280B213FA02F21040F4
:100AD000A4B205D009098B401C420CBF00200120A4
:100AE00010BD01F00F0101238B40DB439BB203815A
:100AF000704700BF08B501214FF48040FFF7BAFDF1
:100B00004FF480400021BDE80840FFF7B3BD014B22
:100B1000186070470038014001F0030289080A4B51
:100B2000023130B5920053F821500F24944025EA49
:100B3000040443F8214053F8214010FA02F2144310
:100B400043F8214030BD00BF00380140014B186020
:100B5000704700BFDC002742014B1860704700BFA0
:100B600000042742024B186AC0F30020704700BF00
:100B70000038014030B5048C24F001042404240C16
:100B80000484058B048CADB2A4B225F0F3051543A3
:100B900024F00A0445EA031544F00104ADB20C4305
:100BA0000583048430BD30B5048C24F01004240483
:100BB000240C0484048B058C24F44074ADB2240509
:100BC000240D25F0A00544EA022445F0100544EA6E
:100BD000033445EA0115A4B2ADB20483058430BDE7
:100BE00008B5474B984205D101200146FFF742FD69
:100BF00001203DE0B0F1804F05D101200146FFF713
:100C00002DFD012076E03F4B984205D102200121C5
:100C1000FFF724FD02206DE03B4B984205D10420F4
:100C20000121FFF71BFD042064E0384B984205D1F9
:100C300008200121FFF712FD08205BE0344B9842A9
:100C400005D110200121FFF709FD102052E0314BA2
:100C5000984205D120200121FFF700FD202049E026
:100C60002D4B984209D102200121FFF703FD0220FC
:100C70000021BDE80840FFF7FDBC284B984207D192
:100C80004FF480300121FFF7F5FC4FF48030EFE79F
:100C9000234B984207D14FF400300121FFF7EAFCC3
:100CA0004FF40030E4E71F4B984207D14FF4802007
:100CB0000121FFF7DFFC4FF48020D9E71A4B98425F
:100CC00005D140200121FFF7C9FC402012E0174B5D
:100CD000984205D180200121FFF7C0FC802009E067
:100CE000134B98420BD14FF480700121FFF7B6FCF3
:100CF0004FF480700021BDE80840FFF7AFBC08BD8D
:100D0000000001400004004000080040000C0040CA
:100D10000010004000140040000401400040014069
:100D2000004401400048014000180040001C004001
:100D3000002000401C4A038890429BB212D002F56A
:100D4000806290420ED0B0F1804F0BD0A2F580327D
:100D5000904207D002F58062904203D002F5806293
:100D6000904203D14A8823F0700313430F4A904204
:100D700008D002F58062904204D023F440730A89BF
:100D80009BB2134303804B68C3620B880385064BF9
:100D9000984203D003F58063984201D18B7A038691
:100DA00001238382704700BF000001400010004013
:100DB0004FF0FF334360002303800381438083723D
:100DC0007047018582827047038823F070031B04FB
:100DD0001B0C0B430380704741627047C162704730
:100DE000406A7047008D80B27047038819B19BB28A
:100DF00043F0020303E023F002031B041B0C0380F7
:100E00007047038819B19BB243F0040303E023F059
:100E100004031B041B0C03807047038819B19BB2A9
:100E200043F0800303E023F080031B041B0C0380CA
:100E30007047038823F008031B041B0C03800388FE
:100E40009BB20B4303807047038823F440731B0459
:100E50001B0C038003889BB20B43038070470388FD
:100E600019B19BB243F0010303E023F001031B041B
:100E70001B0C03807047038C23F001031B041B0C25
:100E8000038470B5038C8488028B0D884E8822F011
:100E900073021204120C2A438D8923F002031B04EF
:100EA00035431B0CADB22B430E4DA842A4B203D068
:100EB00005F58065A8420ED1CD894E8A23F008033E
:100EC0002B438D8823F004032B430D8A354324F4F0
:100ED0004074ADB22C43848002838A6842630384E9
:100EE00070BD00BF00000140038C23F010031B0401
:100EF0001B0C0384038C828830B5048B0D8824F48A
:100F0000E6442404240C23F0200344EA05241B04B3
:100F10008D891B0C43EA05134D8843EA0513134DD5
:100F2000A84292B2A4B29BB203D005F58065A84254
:100F300015D1CD8923F080039BB243EA05134FF608
:100F4000BF751D408B8845EA03130D8A22F4406269
:100F500042EA85024D8A42EA85029BB292B28280C1
:100F60008A6804838263038430BD00BF00000140AF
:100F7000038C23F480731B041B0C0384038C828872
:100F800030B5848B0D8824F073042404240C23F4DE
:100F900000731B042C438D891B0C43EA05234D88E9
:100FA00043EA0523124DA84292B29BB203D005F545
:100FB0008065A84215D1CD8923F400639BB243EA32
:100FC00005234FF6FF351D408B8845EA03230D8A24
:100FD00022F4405242EA05124D8A42EA05129BB2BF
:100FE00092B282808A688483C263038430BD00BF6A
:100FF00000000140038C23F480531B041B0C03846A
:10100000038C30B58488828B0D8822F4E64212046A
:10101000120C23F4005342EA05221B048D891B0C99
:1010200043EA05334D8843EA05330B4DA842A4B289
:1010300092B29BB203D005F58065A84205D10D8A16
:1010400024F4804444EA8514A4B2848082838A68AC
:101050000264038430BD00BF000001400023038010
:101060004380838083608381C3810382438270478E
:1010700030B5058C0124ADB28C4025EA040400F1A2
:101080001803048409B1082907D149084FF68F7065
:10109000CC582040C850C8580AE00439C1F34E016A
:1010A00048F6FF70CC582040C8501202C85892B27F
:1010B0000243CA5030BD4163704781637047C163CA
:1010C000704701647047038B23F070031B041B0CF3
:1010D0000B4303837047038B23F4E0431B041B0C77
:1010E00043EA01239BB203837047838B23F0700391
:1010F0001B041B0C0B4383837047838B23F4E04357
:101100001B041B0C43EA01239BB283837047038BB0
:1011100023F008031B041B0C0B4303837047038B52
:1011200023F400631B041B0C43EA01239BB20383DB
:101130007047838B23F008031B041B0C0B43838332
:101140007047838B23F400631B041B0C43EA0123C9
:101150009BB283837047038B23F004031B041B0C97
:101160000B4303837047038B23F480631B041B0C26
:1011700043EA01239BB203837047838B23F004036C
:101180001B041B0C0B4383837047838B23F4806306
:101190001B041B0C43EA01239BB283837047038B20
:1011A00023F080031B041B0C0B4303837047038B4A
:1011B00009025B0441EA53439BB203837047838B6C
:1011C00023F080031B041B0C0B4383837047838B2A
:1011D00009025B0441EA53439BB283837047038C4B
:1011E00023F002031B041B0C0B4303847047038C86
:1011F00023F008031B041B0C0B4303847047038C70
:1012000023F020031B041B0C43EA01139BB203844D
:101210007047038C23F080031B041B0C43EA01136B
:101220009BB203847047038C23F400731B041B0CD4
:1012300043EA01239BB203847047038C23F40063C9
:101240001B041B0C43EA01239BB203847047038CED
:1012500023F400531B041B0C43EA01339BB20384A9
:10126000704710B5048C01238B40A4B224EA030319
:101270000384038C12FA01F10B439BB2038410BD6B
:1012800010B5048C04238B40A4B224EA0303038426
:10129000038C12FA01F10B439BB2038410BD0023AF
:1012A0000122038043808280C38003817047406BAA
:1012B0007047806B7047C06B7047006C7047038B42
:1012C00023F00C031B041B0C0383038B9BB20B4307
:1012D00003837047038B23F440631B041B0C0383BD
:1012E000038B9BB243EA01239BB203837047F8B59B
:1012F0000C464988A288B4F800E0238905460029F5
:101300000CBF02270027012A14BF01260226BEF1C6
:10131000000F10D1FFF72EFC2846E188FFF7CFFF22
:101320002846394632462389FFF73DFCE1882846A6
:10133000BDE8F840CEE7FFF736FC2846E188FFF726
:10134000C9FF2846394632462389FFF713FCE18856
:101350002846BDE8F840B2E7838B23F00C031B045A
:101360001B0C8383838B9BB20B4383837047838BDC
:1013700023F440631B041B0C8383838B9BB243EADF
:1013800001239BB283837047F8B50D460B88AA886A
:10139000498804463BB92B89FFF7ECFBE9882046D6
:1013A000BDE8F8408BE7042B07D12B89FFF7FBFB47
:1013B000E9882046BDE8F8408CE7082BB5F808C05E
:1013C000078C1DD127F480773F043F0C0784868B60
:1013D000038CB6B29BB226F0F30623F4206346EAF0
:1013E0000C1C43EA01211FFA8CFC89B24CEA020270
:1013F00041F4807182830184E988BDE8F840ABE75D
:1014000027F480573F043F0C0784868B038C26F417
:10141000407623F4005336055B04360D5B0C46EA38
:10142000022243EA013342EA0C329BB2E98892B2CB
:1014300043F4805382830384BDE8F84097E74A88E9
:101440000B8813438A881343CA8813430A891343BA
:101450004A8913438A8913439BB2A0F844307047EA
:101460000023038043808380C38003814381838181
:101470007047B0F8443029B16FEA43436FEA5343F1
:101480009BB201E05B045B0CA0F84430704783889A
:1014900019B19BB243F0040303E023F004031B04DF
:1014A0001B0C83807047838819B19BB243F0010302
:1014B00003E023F001031B041B0C83807047838926
:1014C0009BB20AB1194301E023EA0101818170470F
:1014D00081827047038A19420CBF002001207047A7
:1014E000C94389B201827047038A828911EA0300E5
:1014F00092B203D011420CBF002001207047C943B3
:1015000089B2018270470A43A0F848207047838956
:101510009BB20AB1194301E023EA010181817047BE
:10152000838819B19BB243F0080303E023F008035A
:101530001B041B0C83807047038923F007031B04E3
:101540001B0C03817047038923F070031B041B0CE1
:101550000B43038103899BB243F007030381704768
:1015600038B50D4611460122602D044602D1FFF721
:101570001AFB01E0FFF7FEFA238923F070031B0436
:101580001B0C1D43258123899BB243F00703238154
:1015900038BD038923F070031B041B0C0B4303812C
:1015A0007047838823F070031B041B0C838083889F
:1015B0009BB20B4383807047038923F007031B040E
:1015C0001B0C038103899BB20B4303817047038982
:1015D00023F080031B041B0C038103899BB20B4384
:1015E0000381704710B50489E4B20C43144344EA04
:1015F0000324A4B2048110BD10B50446FFF7F2FF26
:1016000023899BB243F48043238110BD10B5044667
:10161000FFF7E8FF238923F077031B041B0C43F03B
:101620007703238110BD70B50489068B058C26F4E1
:101630004076ADB226F0030624F00704360425F008
:1016400022052404360C1543240C46F4807645EA22
:101650000315214346F00106ADB2018106830584DE
:1016600070BD838819B19BB243F0800303E023F07F
:1016700080031B041B0C83807047A0F85010704738
:1016800008B5234B984205D110200121FEF7F2FF47
:10169000102037E01F4B984207D14FF40030012152
:1016A000FEF7DCFF4FF4003009E01B4B98420BD1F2
:1016B0004FF480200121FEF7D1FF4FF4802000215C
:1016C000BDE80840FEF7CABF144B984207D14FF45B
:1016D00000200121FEF7C2FF4FF40020EFE7104B7E
:1016E000984207D14FF480100121FEF7B7FF4FF465
:1016F0008010E4E70B4B984209D120200121FEF72E
:10170000B9FF20200021BDE80840FEF7B3BF08BDA7
:10171000001001400044004000480040004C0040E0
:101720000050004000140140038ACA889BB223F491
:10173000405330B513430D46038283890989AA8833
:1017400023F4B0530A43698923F00C031B040A43B2
:101750001B0C92B213438381838AAA899BB223F420
:101760004073134385B0838204466846FEF7A6FEA5
:101770001A4B9C4203D003F580639C4201D1039B2A
:1017800000E0029BA28912B2002A4FF019012A68D8
:1017900001FB03F101DA520000E092006423B1FB87
:1017A000F2F1B1FBF3F21201100903FB1011A08951
:1017B00000B2002806DAC9003231B1FBF3F303F0BE
:1017C000070305E009013231B1FBF3F303F00F0326
:1017D0001A4392B2228105B030BD00BF0010014013
:1017E0004FF4165303600C2200238380C3800381CF
:1017F0004281838170470B88028A10B54C8823434D
:101800008C88C988234392B20B4322F470629BB246
:101810001343038210BD0023038043808380C38071
:101820007047838919B19BB243F4005303E023F45A
:1018300000531B041B0C83817047038B03F47F430D
:101840000383038B9BB20B4303837047838929B1C6
:101850006FEA43436FEA53439BB201E05B045B0CC6
:1018600083817047838A19B19BB243F4006303E01C
:1018700023F400631B041B0C83827047C905C90D48
:10188000818070478088C005C00D7047038A23F0AF
:101890000F031B041B0C0382038A9BB20B430382BE
:1018A0007047838919B19BB243F0020303E023F030
:1018B00002031B041B0C83817047838923F400639C
:1018C0001B041B0C838183899BB20B43838170476C
:1018D000038A23F020031B041B0C0382038A9BB2A0
:1018E0000B4303827047038A19B19BB243F48043D0
:1018F00003E023F480431B041B0C0382704783899D
:101900009BB243F0010383817047838A19B19BB274
:1019100043F0080303E023F008031B041B0C83823D
:101920007047038BDBB20383038B9BB243EA012333
:1019300003837047838A19B19BB243F0200303E00D
:1019400023F020031B041B0C83827047838A19B188
:101950009BB243F0100303E023F010031B041B0CA5
:1019600083827047838A23F004031B041B0C838249
:10197000838A9BB20B4383827047838A19B19BB2DF
:1019800043F0020303E023F002031B041B0C8382D9
:101990007047838A9BB20AB1194301E023EA01012F
:1019A00081827047C1F3421310B501F01F01012479
:1019B00014FA01F1A34201D10C3004E0022B01D151
:1019C000103000E0143003680AB1194301E023EA43
:1019D0000101016010BD038819420CBF00200120E5
:1019E0007047C94389B201807047012210B501F0E8
:1019F0001F03C1F342149A40012C01D1838903E0F3
:101A0000022C0CBF038A838A9BB21340028892B2D5
:101A100043B1090A012313FA01F111420CBF00205E
:101A2000012010BD184610BD090A01238B40DB437D
:101A30009BB20380704700BF81F0004102E000BF0D
:101A400083F0004330B54FEA41044FEA430594EA7E
:101A5000050F08BF90EA020F1FBF54EA000C55EAB9
:101A6000020C7FEA645C7FEA655C00F0E2804FEA8A
:101A70005454D4EB5555B8BF6D420CDD2C4480EA6C
:101A8000020281EA030382EA000083EA010180EA9C
:101A9000020281EA0303362D88BF30BD11F0004FEA
:101AA0004FEA01314FF4801C4CEA113102D0404220
:101AB00061EB410113F0004F4FEA03334CEA13335B
:101AC00002D0524263EB430394EA050F00F0A78073
:101AD000A4F10104D5F1200E0DDB02FA0EFC22FA6E
:101AE00005F2801841F1000103FA0EF2801843FA62
:101AF00005F359410EE0A5F120050EF1200E012A53
:101B000003FA0EFC28BF4CF0020C43FA05F3C01890
:101B100051EBE37101F0004507D54FF0000EDCF109
:101B2000000C7EEB00006EEB0101B1F5801F1BD3B2
:101B3000B1F5001F0CD349085FEA30004FEA3C0CB6
:101B400004F101044FEA445212F5800F80F09A80AC
:101B5000BCF1004F08BF5FEA500C50F1000041EBB0
:101B6000045141EA050130BD5FEA4C0C404141EBB4
:101B7000010111F4801FA4F10104E9D191F0000FDB
:101B800004BF01460020B1FA81F308BF2033A3F15E
:101B90000B03B3F120020CDA0C3208DD02F1140C55
:101BA000C2F10C0201FA0CF021FA02F10CE002F190
:101BB0001402D8BFC2F1200C01FA02F120FA0CFC89
:101BC000DCBF41EA0C019040E41AA2BF01EB0451D2
:101BD000294330BD6FEA04041F3C1CDA0C340EDCD0
:101BE00004F11404C4F1200220FA04F001FA02F313
:101BF00040EA030021FA04F345EA030130BDC4F1D1
